:100000000040002051B2000091B2000093B2000005
:1000100000000000000000000000000000000000E0
:1000200000000000000000000000000095B2000089
:10003000000000000000000097B2000099B200002C
:100040009BB20000F18300003DB600009BB20000AF
:100050009BB2000000000000A9B700009BB20000A6
:100060007D4D0000D9BB00009BB200009BB2000098
:100070009BB200009BB200009BB200009BB200004C
:100080009BB2000089B800009BB200009BB2000048
:100090009BB200009BB200009BB200009BB200002C
:1000A0009BB200009BB200000000000000000000B6
:1000B0000000000000000000000000000000000040
:1000C00010B5064C2378002B07D1054B002B02D02E
:1000D000044800E000BF0123237010BD8C02002003
:1000E000000000004C600100044B10B5002B03D051
:1000F0000349044800E000BF10BDC04600000000F6
:10010000900200204C600100164B002B00D1144BD4
:100110009D46402292029A1A924600218B460F4633
:100120001348144A121A10F099FB0F4B002B00D001
:1001300098470E4B002B00D0984700200021040068
:100140000D000D48002802D00C4800E000BF10F060
:1001500025FB200029000BF0A7FB10F0F9FAC046A0
:100160000000080000400020000000000000000027
:100170008C020020F02F0020000000000000000092
:10018000024B1868431E984180007047E00200202F
:100190000020704710B5034B02220349092008F0E4
:1001A0002DFA10BDE8360100F83601000020704736
:1001B00000207047002070470020704710B5034BA7
:1001C000042203490D2008F019FA10BD1C37010064
:1001D0003C37010002000120104013D1002A10D04A
:1001E000042A0ED01368180980B2002809D00138FB
:1001F0008000031D11180979002902D001309842AE
:10020000F8D170470020FCE770B5002204000D0013
:10021000411C092005F066FD002806D0012362007C
:10022000134343600023A34200DB70BD9A00A9582A
:10023000821891600133F6E7F8B54D680F00EB07BF
:1002400006D4042D04D90F232E683340092B03D084
:100250000B2001F035FFF8BD6B683609B6B25C10B3
:10026000731EA3420FD8032120000DF0DBFB642195
:10027000642803DC0100032800DA0321280089191F
:1002800005F062FD05002B6800201B099BB2013BB5
:100290009C42E0D23A68A31C9B005A5101230134CE
:1002A00064001C436C60D6E710B505F041FB4300C9
:1002B0000120184310BD0000C30713D4002811D03B
:1002C00004280FD00F2302681340032B0AD11940D2
:1002D0000133591AC0234907DB051940024B1A4064
:1002E000114301607047C046FFFFFF9F70B50028B3
:1002F00005DC1C2001F0E4FE0500280070BD012291
:100300000C68144201D10D20F4E701281CD04B6881
:100310001342F8D05B101320FF2BEBD81A061904F8
:100320000A431A431B0213436410E243D2171440DA
:10033000E11C89101A00032005F0D4FC051EDCD056
:100340002100FFF7B9FFD8E70023EDE7F7B50191EA
:10035000002804DC1C2001F0B3FE040015E0019B22
:1003600001271D682E003E4011D03D41FF2D01D9CF
:100370001320F0E700223900032005F0B3FC041E2F
:1003800003D03900FFF798FF25712000FEBD042D32
:10039000EED90F232A681340042B1BD12800FFF746
:1003A00019FFC31C07000320D9170140C918891081
:1003B000320005F097FC041EE7D03900FFF77CFF00
:1003C000280005F0D1FA231D01003A00180010F0B2
:1003D00029FADAE7092B21D103206D6832006D106C
:1003E000EB1CD9170140C918891005F07BFC041ECD
:1003F000CBD0019B29001B680193FFF75DFFAE4244
:10040000C3DA019AB300D3189B683B4204D05B1057
:10041000FF2BADD8A21913710136F0E7032BA7D13A
:100420002C00B2E7030001220220134207D1100082
:10043000002B04D0042B02D018680F2318407047FB
:1004400010B588B0002806DC1C2001F039FE04003D
:10045000200008B010BD0C682000FFF7E3FF013852
:10046000082822D80DF02CFA050D18F4212121219D
:1004700018001048042C00D00F48012105F0B0FCF2
:10048000E5E70E496210684611F0CEF8684611F0B3
:1004900011F901006846F1E7200005F065FA040053
:1004A00011F008F901002000E8E7002005F08CFCBD
:1004B000CDE7C0466E45010026380100D843010053
:1004C00010B57F2902DC0170013010BD1A4B994232
:1004D0000CDC40238A115B42134303703F230B4023
:1004E00080214942194341700230EEE7134B994293
:1004F00010DC20230A135B4213433F248022037045
:100500008B1152422340214013430A4343708270AF
:100510000330DAE70A4B9942D7DCF0230370603BE3
:100520004370113B8A11FF3B1A4382703F221140F6
:100530001943C1700430C8E7FF070000FFFF000047
:10054000FF0F010010B5094C002220600221092094
:1005500005F0C8FB2368002803D10A3001F0B0FD84
:1005600010BD032283604260FAE7C046D00B002032
:1005700070B5C30710D544101320FF2C07D80022F4
:100580000121032005F0AEFB051E09D10A2001F070
:1005900097FD0500280070BD0400601E8441EEE751
:1005A0000121FFF789FE2C71F4E710B50124044006
:1005B00002D04410200010BD042810D90F23026877
:1005C0001340042B07D105F0CFF921000A2211F0C6
:1005D00039F90400EEE7032B01D10430F5E70D20D3
:1005E00001F06EFDE6E70000F0B50E0085B00028D2
:1005F00003DC1C2001F064FD17E00F6801243D00BE
:10060000254006D1042F1ED90F233A681340042B2E
:100610000DD13800FFF7C9FF02AC01002000FFF741
:100620004FFF011B200005F0DBFB040032E0092B2B
:1006300009D17B685B100193019B9C4205DD01F0B1
:1006400045FD002819D02A20D4E70134A300F8582A
:10065000FFF7ABFF01237F280DDD154ADB18904221
:1006600009DD144A0133904205DD0021124AC30F0F
:1006700082424B419B00ED18DEE7280005F0A4FB09
:10068000041E07D0376805F06FF901250600019BAD
:100690009D4202DD200005B0F0BD0135AB00F858E9
:1006A000FFF783FF01003000FFF70AFF0600EEE7C7
:1006B000FF070000FFFF0000FF0F0100F7B5030078
:1006C00001900E001C20012B11DD0868FFF76DFF63
:1006D00007007068FFF769FF019B05000124022BEA
:1006E00008D0B068FFF761FF041E03DC292001F089
:1006F000E7FCFEBDAF421CDCE81B21000DF092F9C7
:10070000451C691C0022092005F0ECFA0028F0D0F5
:1007100001226B00134343609440002379009D4203
:10072000E7DD17009E000F438619B76001330919F2
:10073000F5E7781B21000DF075F96442451CE0E7F0
:1007400010B504000120084010D104290DD90F2351
:100750000A681340042B08D1080005F005F90100D0
:10076000200010F09DFF4342584110BD0020FCE7DF
:10077000F7B50E00012803DC1C2001F0A1FCFEBD32
:100780004D68EB0706D4042D04D90F222B681A40BC
:10079000092A01D00B20F0E76A681B099BB25410AC
:1007A000A34200D85C1E012731680F404810002F7B
:1007B00035D12648FFF7C4FF01230190002813D14B
:1007C00031682348FFF7BCFF002811D0002C0DD062
:1007D0000122631C013C94409B005A5114436C60FD
:1007E00004E00137BA00AB50BC42FADA0020C6E799
:1007F00001233068184223D1042821D902680E331E
:100800001340042B1CD1FFF7D0FE002807D131681C
:100810001048FFF795FF002812D01220ADE70028FE
:10082000FBDD8442F9DB8300EB180433844209DCEE
:100830000123621C013C9C40920053511C43CEE7B3
:1008400011209AE75A6801301A60EEE71D3801005E
:100850002138010026380100002310B50C000B7070
:10086000C30705D50D494210200010F0DDFE08E059
:100870000B49002802D0042804D10A49200010F0B6
:10088000F3FE10BD0428FCD90F2302681340042B8B
:10089000F7D105F069F804490200E5E7D843010003
:1008A000263801006E45010028380100F0B593B0EC
:1008B000060002911C20012E1DDD029B01251B68F4
:1008C0001C002C4000D0ADE0042B00D8E6E01A68F4
:1008D0000F231A40092A4AD10394039A02999200DD
:1008E0008A5817002F4005D1042A03D910681840F0
:1008F000092806D0222001F0E3FB0190019813B0F3
:10090000F0BD52685210A418039A01320392964225
:10091000E3D1611C012205F0E5F90190002802D124
:1009200000230193EAE7019B6400190025435D6001
:100930000831029ABB00D05802684368120992B28B
:100940005B109A4200D8531E0022934209DCDA431E
:10095000D21713409B00C918039B01379F42E8DB65
:10096000CCE794000519AD6801320D51EDE7270081
:10097000032A59D10193029ABB00D3582B42B9D113
:10098000042BB7D9186801990140032939D102090C
:1009900092B2430F92000B40D31A1C190137BE428A
:1009A000E9D10320E31CD9170140C918891000229E
:1009B00005F098F901900028B2D000252100FFF73A
:1009C0007BFC019B1E1D029AAB00D45801231C42E4
:1009D0001FD1042C1DD90F2123681940032918D1D8
:1009E000180980B25B0F80000B40C01A00238342BD
:1009F00013DBC343DB17184001353618BD42E2DB79
:100A00007CE7042900D075E71800FFF7E3FB241802
:100A1000C4E72000FFF7DEFBE8E7E2181279F254A2
:100A20000133E4E700273C000F25029ABB00D358AE
:100A30000122134239D1042B32D919680800284009
:100A400004283AD11800FFF7C5FB24180137BE422D
:100A5000EBD1200005F0B8F90190002800D15FE744
:100A6000029FB600BB19051D029301233C681C427E
:100A700032D1042C2CD90F2623681E40042E40D1DD
:100A80002000FFF7A7FB0600200004F06DFF010027
:100A9000280032000FF0C6FEAD192BE02700C3E797
:100AA000002B02D0042B00D024E7180005A9FFF783
:100AB000D3FE05A810F0FEFDC7E7032800D019E714
:100AC0000B099BB2490F9B0001405A1A1419BDE74C
:100AD000002C01D0042C0DD105A92000FFF7BCFE8D
:100AE00005A810F0E7FD05A90400020028000FF09A
:100AF00099FE2D19029B0437BB42B6D100232B70FF
:100B0000FCE6032EF6D11A0992B25B0F92001E404A
:100B1000961B211DBCE70000F0B50D0097B0002822
:100B200006DC1C2001F0CCFA0700380017B0F0BD3D
:100B30000C68012123000B40009306D1042C04D93A
:100B400022680F331A40092A01D00B20EAE76268B5
:100B500052100392002A03DC009805F035F9E3E710
:100B6000524A019201280BD06868084208D1042833
:100B700006D902681340042B02D104F0F5FE01905F
:100B8000019810F097FD06000F27039B0834013BE6
:100B900005935E43039B02909B00E318049301239B
:100BA0002068184277D1042871D901680A003A40B8
:100BB000042A03D1FFF70EFB361808E0032A71D18F
:100BC0000B099BB2490F9B0011405A1A9619049BBE
:100BD0000434A342E3D1300005F0F6F8071EA4D098
:100BE0002B680793029B002B03D0686804F0BCFEBF
:100BF0000190380004F0B8FE0400009B079A9B00A7
:100C0000D3189D68280004F0AFFE01232B40060096
:100C10000693002B03D1002D01D0042D04D109A986
:100C20002800FFF719FE09AE300010F043FD069BC7
:100C30000490002B0ED1042D0CD90F212B681940E4
:100C4000032907D11A0992B25B0F92000B40D31A05
:100C50002E1D04932000049A31000FF0E3FD049B45
:100C6000E418029B002B0AD0059B009A934206DDF4
:100C70002000029A01990FF0D5FD029BE418009B19
:100C800001330093009A039B9342B6D14DE70028AD
:100C900001D0042806D109A9FFF7DEFD09A810F04C
:100CA00009FD89E704F060FEF9E7C046EB43010067
:100CB0000378002B03D05AB2002A01DB01307047C1
:100CC0003F229343C03B59424B41C01803789343A2
:100CD000802BF4D10130F9E7F0B585B0012803DCB1
:100CE0001C2001F0EDF912E001254B682A00009369
:100CF000022806D08B682B4203D05D10002D00DC4B
:100D000015000122009B134203D00120404205B090
:100D1000F0BD009B042BF8D91B680F271E000C6840
:100D20003E40042E30D101231C4205D1042C03D9AE
:100D300023681F40042F01D00E20D2E70098FFF750
:100D400049FAA842E1DB009804F00EFE06002000FC
:100D500004F00AFE03780100002BD6D0681E30187C
:100D600010F0D4FC0125041ECFD03378002B01D025
:100D7000A64203D3680001252843C8E73000FFF7E7
:100D800097FF01350600F0E7092E40D1009B5B6814
:100D900001935E10B542B8DC01231C422DD1042C16
:100DA0002BD923683B40042B27D1200004F0DCFD25
:100DB00001230290019303976F1C009ABB00D05847
:100DC000844204D1019B6800034318009FE7019B04
:100DD00018420ED104280CD90368039A1340042B3F
:100DE00007D104F0C1FD0100029810F059FC002861
:100DF000E8D03D00B742DFDD87E76B1C00999A0021
:100E00008A58A242B6D01D00B342F6DD7DE7032E1C
:100E100000D07AE71A0992B25B0F92001E40961B2F
:100E2000B54200DD71E701231C4227D1042C36D9DD
:100E300022681740032F17D1100980B2520F231DCB
:100E400080003A400193801A019B361A1F18009BBC
:100E5000681E0433B04200DD57E7019A1918BA4200
:100E60001FD326D1013018E0042F18D1200004F040
:100E70007BFD01902000FFF7ADF9E5E76410681EE7
:100E8000FF2C01D928202CE7B04200D13DE7009B80
:100E90001B181B790130A342F6D140006BE70F20ED
:100EA0001FE70C78A4461478A44502D10131013221
:100EB000D5E70130CEE710B500240378002B01D12F
:100EC000200010BDFFF7F4FE0134F6E7F7B5070088
:100ED0000E001C20012F06DD4C68012322001A4061
:100EE000009203D10D2001F0EBF853E0022F02D065
:100EF0008A681A42F6D0012335681D4200D0A9E065
:100F0000042D00D8A6E01C41002C00DC1C000F20A2
:100F100029680840092828D16B685B100093022FCC
:100F200005D0B368009A5B109A4200DD0093009BE5
:100F300001221D1B0135EB43DB171D40691C0920F5
:100F400004F0D0FE071E09D001236D001D430300ED
:100F50003268083345600099A14201DA3800FEBDCD
:100F60000134A100515802C3F5E7042845D12800F7
:100F700004F0FAFCFFF79FFF0190022F04D0B36842
:100F80005B10984200DD0193019BA34204DA00202C
:100F900004F01AFF0700E1E7280004F0E5FC070071
:100FA000009BA34221DB2800009704F0DDFC050034
:100FB0003800FFF77DFE019B01340700A342F7DAFA
:100FC000009BC41A200004F0FFFE071EC6D004F0E8
:100FD000CBFC0190306804F0C7FC2200009B591B39
:100FE000411801980FF01EFCB8E73800FFF760FECB
:100FF000009B070001330093D2E703282AD10B0995
:101000009BB2490F9B000140591A022F04D0B268CD
:101010005210914200DD1100A14205DA00220320A6
:10102000110004F05FFEB5E703200E1B331DD91736
:101030000140C9188910002204F054FE071E00D197
:101040008CE7013631000334FFF736F9381D2919D2
:101050003200C7E7212046E7F0B506008DB00D004D
:101060001C20012E0BDD01230868184206D104283C
:1010700004D90F2102680A40042A04D00E2001F08E
:101080001FF80DB0F0BD6A6813400493F6D1042A2E
:10109000F4D913680B40042BF0D104F065FC040074
:1010A000686804F061FC039010F004FB0290022ECB
:1010B00004D0AB68043B5A425A410492029B002B75
:1010C0000FD12000FFF7F7FE0190019B0122591C70
:1010D000092004F007FE514F3860002815D1002088
:1010E000CFE70399200010F011FB001B434243415E
:1010F00020000193019B5E1C0028E6D0029B03990F
:10110000C01810F003FB0196F4E7019B029E5A0001
:10111000012313434360049B1E4319D12000FFF7B2
:10112000C7FD019B0500B34202DC3C4B1868A8E7F1
:10113000291B200004F054FE0028D0D0B31C3A68CC
:101140009B0098502800FFF7B3FD01362C00E8E71C
:10115000019B012B02D12B688360E6E7200010F091
:10116000A9FA23180593029B651C002B04D0039950
:10117000200010F0CBFA05000127002DD5D0019BEF
:10118000BB42D2DB049A291B2300002A06D120008F
:1011900004F026FE002826D1A1E701339D42F6D9AE
:1011A0001A78202AF9D92D2A02D101339D42EED98D
:1011B0001A009D422AD8A54202D92378202B2BD988
:1011C0002E1B132E00DD13263200210007A810F07D
:1011D00089FA002107AB18000A22995510F032FB5A
:1011E0000123400018430D4B01371B68BA00D05053
:1011F000029BEC180135002B04D00399200010F05D
:1012000085FA0500002DB8D1059DB6E712780133A7
:10121000303A092ACCD9BAE70134CCE7D00B002008
:1012200070B50D0004F0A0FB0400012D0EDCFFF7EB
:101230003FFD061B300004F0C7FD051E0ED004F074
:1012400093FB320021000FF0EDFA07E02378013D17
:10125000002B05D1122000F033FF0500280070BDDF
:101260002000FFF725FDDFE7020000787F2809DD79
:10127000DF2808DCF8238001DB00184053783F2288
:10128000134018437047EF280BDCFC215378090109
:101290009B010007000C0B40034390783F22104055
:1012A000EFE7F72812DCFC21537889021B030B407F
:1012B000E0218004490308403F210343D0780840DF
:1012C00003439078FC2280011201E8E701204042AC
:1012D000D8E770B5012803DC1C2000F0F1FE70BDDA
:1012E00001230C6811201C42F7D04868184206D12F
:1012F000042804D90F2302681340042B01D00E20C8
:10130000EBE704F031FB64100500002C03DDFFF770
:10131000D2FDA04205DA1220DFE7FFF7C9FC050085
:10132000013C2800012CF8D1FFF79EFF400020432C
:10133000D5E70000F0B50D008BB0012806DC1C20BD
:1013400000F0BEFE040020000BB0F0BD0C682000D1
:10135000FFF768F80600686804F006FBB04907006C
:1013600010F09EF9012500281FD1AE49380010F079
:1013700097F9002800D10225AB49380010F090F908
:10138000002800D10425A949380010F089F9002867
:1013900000D10925A649380010F082F9002800D1B3
:1013A000B0E16B1C03D13020CAE76D42DDE7701E4F
:1013B0000828C8D80CF098FA09001F004F01400017
:1013C000C7FFC7FFC7FFC7FFAF00A81E0728BAD8CF
:1013D0000CF076FA042E09B9B9B9B92A042C00D157
:1013E0008EE10124AFE79348042C00D092480121FC
:1013F00004F0F6FCA6E7681E0828A4D80CF060FAF2
:1014000005A31809A3A3A3A3140064102BD00424DC
:1014100099E78A49621002A810F006F902A810F0B4
:1014200049F9010002A8E3E72000FFF78BF889E7FC
:101430002000FFF79DF885E7681E082800D982E79D
:101440000CF052FA09001300480081FF81FF81FF70
:1014500081FF81FF1A00200004F086FA764910F01F
:101460001FF90028D3D100246DE72000FFF79DF875
:1014700001244000044366E7200004F075FAFFF7FA
:101480001AFD6F4D411C0600002209202C6004F05B
:1014900029FC041E01D10A2052E7012273001343E4
:1014A0002868636004F060FA0123070000250193B7
:1014B000AE4200DC47E73800FFF7D6FE019AAB00EA
:1014C00040001043E31898603800FFF7F1FB013546
:1014D0000700EDE7200004F047FA10F0EBF8584E53
:1014E000C11C0500891000220320346004F0FAFBBF
:1014F000041ED0D036682900FEF7DEFE300004F06E
:1015000033FA00239D4200DC1DE7C15CE218117133
:101510000133F7E703256368681E5F10032800D9CD
:1015200011E70CF0D7F9020D5835012F06D1A46848
:101530002000FEF777FF012800D104E72D20FFE609
:10154000012F03D1A4683C4200D0FCE62C20F7E632
:101550000136B300E058FFF728F801237F280CDD9F
:10156000384ADB18904208DD374A0133904204DDE7
:10157000364A2B00904200DD0023019AD3180193D4
:10158000B742E5DA00F0A2FD002804D02A20D7E611
:1015900001260023F3E72A4D01982C6004F014FC87
:1015A000041E00D15FE72E6804F0DEF90125AF428A
:1015B00000DAC8E60135AB00F1580123194201D128
:1015C0002720BDE6224B4910994201D93120B7E6C8
:1015D000FEF776FFEBE70320FB1CD9170140184DFF
:1015E000C918891000222C6004F07CFB041E00D175
:1015F00051E739002D68FEF75FFE002301219F426D
:1016000000DCA0E69A00AA1892680A42D8D05210CC
:10161000FF2A01D9132093E6E01802710133EEE7A7
:10162000F7370100FF370100063801000D380100CF
:10163000123801006E45010026380100D843010030
:10164000D00B0020FF070000FFFF0000FF0F01008C
:10165000FFFF100035002368681E1E09B6B25B004C
:10166000B6009B0FF61A082800D96CE60CF03CF97E
:10167000090012006BFE19006BFE6BFE6BFE6BFE29
:101680002C00012E00D059E723790424002B00D030
:1016900059E6E8E6012E00D058E724796400344387
:1016A00051E6204D30002C6004F08EFB29680400C8
:1016B0000423002800D1EEE61A1F964200DC42E621
:1016C000CA5CE2540133F7E7164D711C0022092071
:1016D0002C6004F007FB041E286800D1DBE601251E
:1016E00073002B43636000239E4200DC2BE6C2188C
:1016F00012799900520061182A438A600133F3E796
:10170000032420E6701E082800D91CE60CF0ECF833
:1017100090FE90FEA2FFE2FE1BFE1BFE1BFE1BFEC8
:1017200002FFC046D00B002010B501220024002883
:101730000BDD0B681A40141E03D05C10E343DB176B
:101740001C400122904200D04A68611C092004F02C
:10175000C9FA002803D0012364001C43446010BD73
:101760000123F7B500254E680C0033400193AB42CE
:101770000ED11D00042E0BD90F2233681A40092AFE
:1017800014D172681B099BB25510AB4200D85D1E84
:1017900027687C10FB074CD439003E48FEF7D0FF89
:1017A000002829D0002D12D112203EE0042A04D1B5
:1017B0003000FEF70FFD0500EAE7019D032AE7D19F
:1017C0001D09ADB25B0FAD001340ED1AE0E70FF05D
:1017D000B5FE29000CF00CFA4C1C019B002B56D1D5
:1017E000042E54D932680F331340092B28D1013409
:1017F000A400A4592000FEBD39002748FEF7A0FF31
:1018000000281BD1042F0FD90F233A681340042B53
:101810000AD13800FEF7C9FE041E0AD139001F485C
:10182000FEF78EFF0028BFD1112000F049FC040014
:10183000E0E7002CB8DDA542CFDAB5E72C00CCE715
:10184000042B1CD1300004F08FF80500012C0EDCB5
:10185000FFF72EFA461B300004F0B6FA041EC9D07A
:1018600004F082F8320029000EF0DCFFC2E72B788A
:10187000013C002B98D02800FFF71AFAE5E7032B6C
:1018800005D13419E37801245B001C43B2E70B2037
:10189000CBE7C046F03701002138010026380100AF
:1018A000F7B54D680E002A0001210A402FD1042D02
:1018B0002DD90F242B68B7681C40092C14D16968F6
:1018C0001B099BB24C100192A34200D85C1E3168E8
:1018D0003448FEF735FF00282DD00F232A68134027
:1018E000092B1DD1012317E0032C10D10F4203D186
:1018F000132000F0E5FBFEBD7A100192FF2AF7D815
:101900001A0992B25B0F92001C40141BDFE70B20F8
:10191000EFE701339A00AF509C42FADA0020EAE781
:10192000032BFBD12B0001335A1BA242F6DC6A4683
:101930001279DA70F7E736687010F30719D43100BE
:101940001948FEF7FDFE002822D1042E1ED90F23D0
:1019500032681340042B19D13000FEF726FE002810
:1019600007D131001148FEF7EBFE00280ED01220FF
:10197000BFE70028FBDD8442F9DB0F232A68134010
:10198000092B07D1013080004751C7E71120B0E78C
:101990002000F2E7032BC1D16B461B792D18EB70A9
:1019A000BCE7C0461D38010021380100263801007F
:1019B00070B501240868204207D1042805D90F25F5
:1019C00001680D40092D02D14468200070BD032D2F
:1019D00008D10A0992B24B0F92002B40D31A5B0038
:1019E0001C43F2E7042DF0D103F0BEFFFFF763FACA
:1019F00040000443E9E7000010B5034B10220349FF
:101A0000012006F0FBFD10BD703701006B370100AF
:101A1000024A1368013313607047C046A8020020D1
:101A2000024AD3680133D3607047C046A802002041
:101A3000024A9369013393617047C046A8020020AF
:101A4000024A536A013353627047C046A80200201D
:101A500010B5002802DD0B68DA0703D4112000F06E
:101A60002FFB10BD5B10013B0020032B03D80C2281
:101A70005343034A9858430001201843F1E7C046F6
:101A8000A802002010B5002802DD0B68DA0703D495
:101A9000112000F015FB10BD5B10013B0020032B53
:101AA000F9D80C225343014A9850F4E7A8020020C9
:101AB00010B50400807909F04BFEE07909F048FE8A
:101AC00001235B42E3800023236010BDF7B50300D0
:101AD00001900F001C20012B07DD01230C681C4224
:101AE00002D04868184203D1112000F0E9FAFEBD87
:101AF000401003F06BF8019B6410013C05000026C8
:101B0000022B04D0BB6801361E4000D05E10002DB1
:101B100001DA3520E9E7032CFBD80C206043144F91
:101B2000EBB23818EDB20193FFF7C2FF0021280095
:101B300003F028F8631E0F49022B02D80E4A9B00BF
:101B400099580322012E03D03200022E00D0042225
:101B5000280009F089FD0C235C436B4600201B79AB
:101B600038513F19BB71FF233872FB71BFE7C04684
:101B7000A8020020111A0000D438010010B5002876
:101B800002DD0868C30705D4112000F099FA0400AB
:101B9000200010BD4010013800240328F8D80C2381
:101BA00043430248C018FFF783FFF1E7A802002073
:101BB000F0B5070085B00E001C20022F0ADD0123BE
:101BC0000C681C4205D04868184202D08A681A4244
:101BD00004D1112000F074FA05B0F0BD401002F0FD
:101BE000F5FFB3680500581002F0F0FF00230190E4
:101BF0000093032F05D0F368043B5A425341DBB2F4
:101C00000093002D02DB019B002B01DA3520E1E778
:101C10006410661E032EF9D8EBB202930C206B46BB
:101C2000FF271B79704303931A4B3D401818FFF7A9
:101C30003FFF019B00213B401F00280002F0A2FF54
:101C40000021380002F09EFFA31E134C022B02D885
:101C50009C00124BE45802222100280009F004FDE8
:101C6000009B002B04D002222100380009F0FCFC6C
:101C70000C2300205E43074B98519E196B461B7A3C
:101C80003071B3716B461B7B7071F3716B461B78BF
:101C90003372A1E7A8020020391D0000C8380100F6
:101CA00070B5040080790AF017F8451EA841C5B246
:101CB000E0790AF011F8431E9841237AC0B2002B54
:101CC00019D02379DBB2AB4209D0236801228542C7
:101CD00003D09B182360257170BD5242F9E76279E9
:101CE0008242F9D022680121834200D00239521881
:101CF00022606071F0E723680122854202D09B18C0
:101D00002360E9E75242FAE710B502482430FFF7B2
:101D1000C7FF10BDA802002010B502481830FFF719
:101D2000BFFF10BDA802002010B502480C30FFF71D
:101D3000B7FF10BDA802002010B50248FFF7B0FFA2
:101D400010BDC046A802002010B5034B0522034970
:101D50000F2006F053FC10BDE038010008390100E7
:101D60000122034B5242DA805A82DA835A85704745
:101D7000A80200200020704704207047012070470F
:101D800010B5002004F020F810BD0020704700209E
:101D900070470020704700207047002070470020E7
:101DA00070470020704700207047002070470020D7
:101DB00070470120704710B5002004F005F810BDF1
:101DC00010B5034B10220349072006F017FC10BD85
:101DD0003C390100BC3901007047002070470020E9
:101DE0007047002070470020704700207047002097
:101DF00070470020704700207047000010B5034B6B
:101E0000082203490C2006F0F9FB10BD603A0100DE
:101E1000A03A0100704770470022014B1A607047DA
:101E2000DC0200200020014B18607047DC0200201B
:101E300070B5074C060020000D0009F0A7FA02005B
:101E4000A84200DD2A003100200009F044FA70BDEC
:101E5000601A002010B5521A4118024809F098F98A
:101E600010BDC046601A002010B5054C200009F0D6
:101E70005BFAE1212000490209F041FA10BDC04699
:101E8000601A0020F8B50127060014000800394246
:101E900027D104293FD90F230A681A40042A3AD1CE
:101EA0003C4213D1042C11D922681340042B0DD1CC
:101EB00003F05AFD0500200003F056FD0100280044
:101EC0000FF0EEFB00282EDB1FD127E0E30722D521
:101ED00003F04AFD0A2200210FF0B4FC0500601057
:101EE00010E0174015D1042A15D90F2312681340AA
:101EF000042B10D120004D1003F036FD0A223900CA
:101F00000FF0A0FC85420EDB08DD002E09DC00206E
:101F10000CE04D10E3E70F22054B1A700136022E3C
:101F2000F5D8042002E0042076173040F8BDC04602
:101F30000803002002000120104007D1002A04D02D
:101F4000042A02D01068000980B270470020FCE724
:101F500070B50E000400FFF7EDFF05003000FFF73D
:101F6000E9FF0023854206D10434AD00043665192B
:101F7000AC4202D30123180070BD207832780028CB
:101F800001D1002AF6D0013401369042F0D000236E
:101F9000F1E7000010B50124044002D044102000F5
:101FA00010BD042810D90F2302681340042B07D159
:101FB00003F0DAFC21000A220FF044FC0400EEE7F3
:101FC000032B01D10430F5E70D22014B1A70E6E72F
:101FD00008030020F7B50700009101932E492F4B0D
:101FE000002A02D002220A70013A00261A601B68F9
:101FF000CE54BE4200DBF7BD009AB300D058274B49
:10200000254D1C68FA239B0065191C1B01231842EF
:1020100006D0234A4310210028000FF0D3FA09E02C
:10202000204A002802D004281BD11F4A2100280082
:102030000FF0C8FA184C20000FF03CFB174A019B28
:102040001060002B0BD07B1EB34208DD174B98426B
:1020500005D8431C1360202222540022E25401368A
:10206000C7E70F2301680B40042B04D103F07CFC6D
:102070000F4A0300CFE7092B03D143680D4A5B10D9
:10208000C9E70D4A032BC6D10A0992B2490F920043
:102090000B40D31A094ABEE709030020F4060020CA
:1020A000D8430100FC3C0100023D0100E7030000B1
:1020B00044550100073D0100213D0100163D01008E
:1020C000014B18700020704708030020024B18785D
:1020D000431E98417047C04608030020FA239B0026
:1020E0005843044B1860044B1A78002A01D1FF3280
:1020F0001A707047FC06002008030020002310B56A
:102100001A00FFF767FF034B0348196806F0FEFF4C
:10211000002010BDF40600200903002010B502F0D5
:10212000F7FC014B186010BD0007002070B502F0ED
:1021300023FD094C0100251D1F2228000FF0D2FAB3
:1021400028000FF0B7FA0423043080080001184378
:102150002060200070BDC046E4020020F8B50400F5
:102160000FF0A8FA0022154DD3005B191979032945
:102170000ED11B6819005B6808319B00013BCB182E
:10218000994202D21E78002E08D01B1A994207D914
:102190000132FF2AE8D1013AFF3A06E0013BEFE7BE
:1021A00019780029F4D1884201DC1000F8BD5E18CE
:1021B0007778665CB742EBD10131F4E71025002057
:1021C00010B5040006F026FA002806D12000FFF71B
:1021D000C5FF002802DB044B184310BD1B22012061
:1021E000024B40421A70F8E700FFFFFF080300208F
:1021F000C368F0B55F00836889B0DF190300183346
:1022000001930369019A9900019B00905C1843694E
:1022100002939B00D3180393C64B1B78002B0DD160
:102220000022BB5E7F2289101D1201611340C2494A
:102230009B005B58023702929F461400BD4B00255D
:102240001978FF292BD11D70BC4D2B68002B46DD62
:102250000123009A137002F051FC2B681818009BA0
:1022600058603CE014000700E8E714000700E5E7C9
:102270001400E3E71400E1E71400DFE71400DDE7F2
:102280003400DBE7049CD9E73400D7E73400D5E716
:1022900014000700D2E7049FD0E7079FCEE7FE298E
:1022A00002D11D7009B0F0BD009B9B680293FA1A21
:1022B000009B52109B7812021A43009B587806F03C
:1022C00074FCF022009B9E491D700B689D48013BE9
:1022D0005A43125C002A00D10B60964B1D70009B84
:1022E000009A9B680293FB1A5B10D360019BE41A6F
:1022F000A4101461039B019A9B1A009A9B105361CE
:10230000D0E7009B587806F048FC0023009A8C49DF
:102310001370F0220B688B48013B5A43125C002A71
:10232000DDD10B60DBE7ECE7824BAD001B78641B73
:10233000002B00D082E70022BB5E019A0099A21A0E
:1023400092100A61029A1D1213407B4A9B009B580F
:10235000023771E7019B221DD11A764BD82902DD85
:102360001A221A706AE71B782560002B00D064E7F8
:1023700000203B5E00988910016102991D120B40FC
:102380006D499B005B581400023755E7019B221DE5
:10239000D11AD82903DD1A22664B1A704EE700269F
:1023A000BB5FEDB21B021D43624BB81C1B7825605E
:1023B000002B00D056E702203B5E00988910016197
:1023C00002991D120B405C499B005B5814000437B6
:1023D00032E7019B221DD11AD82903DD1A22554B61
:1023E0001A702BE700257B5FB81C5B00FB1823608D
:1023F000504B1B78002B00D037E702203B5E009843
:102400008910016102991D120B404B499B005B58DA
:102410001400043710E7019B221DD11AD82903DDCF
:102420001A22444B1A7009E7474BAD00EB58236062
:10243000404B1B78002B00D01AE700203B5E009831
:102440008910016102991D120B403B499B005B58AA
:1024500014000237F0E6043C3B4B2268AD00EA5022
:10246000344B1B78002B00D0E8E60022BB5E019ABB
:102470000099A21A92100A61029A1D1213402E4A64
:102480009B009B580237D7E62F4BAE00F058FFF762
:1024900081FD284B05001B78002B09D1043C2068E6
:1024A000FFF778FD451901206D00274B0543F550D6
:1024B000204B1B78002B00D0C0E60022BB5E019AA7
:1024C0000099A21A92100A61029A1D1213401A4A28
:1024D0009B009B580237AFE6019B221DD11A154B7A
:1024E000D82902DD1A221A70A8E6019D039E012058
:1024F000B54202D230000C3800681B782060002BF7
:1025000000D0B7E600203B5E009889100161029977
:102510001D120B4008499B005B58140002378BE6E4
:10252000019B221DD11A034BD8290FDD1A221A70E4
:1025300084E6C04608030020FC3A0100FC060020A7
:10254000F8060020B01B0020082D00200198039EF3
:10255000B0421CD233000C3B1B68D2485B102D18D4
:10256000ED1AAD00AB592360CF4B1B78002B00D088
:1025700082E600203B5E00988910016102991D12DD
:102580000B40CA499B005B581400023754E61820E0
:1025900018700023E7E7019B039A93421FD21300B0
:1025A0000C3B1B68BF4A5B10AD18043CED1A226857
:1025B000039BAD00EA50BC4B1B78002B00D03DE6DE
:1025C0000022BB5E019A0099A21A92100A61029A37
:1025D0001D121340B54A9B009B5802372CE6182267
:1025E000B14B1A70E7E7019B039A93422ED2AD4B91
:1025F000043CEE1815000C3D2B685B10F31A9B0091
:102600009858FFF7C7FC04902068FFF7C3FC2D68BB
:10261000049B6D10751B1E1801207600039BAD00F6
:102620000643EE50A04B1B78002B00D006E600229C
:10263000BB5E019A0099A21A92100A61029A1D12B9
:1026400013409A4A9B009B580237F5E51822964B97
:102650001A70E7E7019B221DD11A934BD82902DD9E
:102660001A221A70EAE50398AD0028581B782060FA
:10267000002B00D002E600203B5E0098891001612B
:1026800002991D120B4089499B005B5814000237C8
:10269000D2E5043C039B2268AD00EA50824B1B78D4
:1026A000002B00D0CAE50022BB5E019A0099A21A55
:1026B00092100A61029A1D1213407C4A9B009B589B
:1026C0000237B9E5039BAD005D192B68043C206817
:1026D0005E10FFF75FFC36180120734B76001B7805
:1026E00006432E60002B00D0A8E50022BB5E019AB5
:1026F0000099A21A92100A61029A1D1213406B4AA5
:102700009B009B58023797E5019BAD00641B664D0B
:10271000A34212D82B78002B00D08FE50022BB5E9D
:10272000019A0099A21A92100A61029A1D1213408E
:102730005E4A9B009B5802377EE55D4803F004F932
:102740002B78002B00D079E50022BB5E019A00991E
:10275000A21A92100A61029A1D121340534A9B005A
:102760009B58023768E5002D02D10023FD5E023739
:102770006B00FF18002D00DAB1E54B4B1B78002BE6
:1027800000D05BE50022BB5E019A0099A21A92106C
:102790000A61029A1D121340444A9B009B5802375B
:1027A0004AE5002D02D10023FD5E02376D007F193E
:1027B000BB1E1B88029A1340132B14D10C3C3A4BBE
:1027C0001B78002B00D039E50022BB5E019A0099EE
:1027D000A21A92100A61029A1D121340334A9B00FA
:1027E0009B58023728E51A2BE9D1043CE7E7002D76
:1027F00002D10023FD5E0237043C2368042B04D180
:102800006B00FF18002D00DA69E5274B1B78002BC1
:1028100000D013E50022BB5E019A0099A21A921023
:102820000A61029A1D121340204A9B009B580237EE
:1028300002E5002D02D10023FD5E0237043C23682F
:10284000042B04D06B00FF18002D00DA47E5164B6F
:102850001B78002B00D0F1E40022BB5E019A0099A6
:10286000A21A92100A61029A1D1213400F4A9B008D
:102870009B580237E0E4002D02D10023FD5E0237B1
:10288000261F3068C3070AD540100138002811DB25
:10289000012340006D0018437F1930601FE5FFF7EA
:1028A00079FBF2E7FDFFFF3F08030020FC3A01003F
:1028B000333D0100DB4B34001B78002B00D0BDE41E
:1028C0000022BB5E019A0099B21A92100A61029A24
:1028D0001D121340D44A9B009B580237ACE40023DE
:1028E000F85E023703129C46DBB2DB000493049AC5
:1028F000CE4BCC499B181B79032B02D002230B70C3
:102900009CE42500019B0C35EE1AD82E02DD1A231B
:102910000B7093E4FF2301225B004000184010433A
:10292000009B20609B6800980693FB1A13418078F7
:102930001B0203439340134363600198039B039579
:102940001B1A9B1093401A43A2606246009B9A7028
:10295000049AB64BD358009A93600A78002A03D0A1
:1029600008331F002C0069E41F0008229B5E009AB8
:10297000B6101661029A1D121340AB4A9B000A372B
:102980009B58039C58E4231F1D68039A019B9342A4
:1029900032D10A20EB0711D4042D18D90F232A684D
:1029A0001340042B16D1280002F0DEFF0EF082FE49
:1029B000C8239B00984200D918000630643005F007
:1029C000F3FE00280FD1023F019B039387E4072009
:1029D000042DF3D02800431E9841FA234042FF33D0
:1029E00018400730EAE7009B2900587806F0EFF816
:1029F0000023009A1370E7E7039B039A0C3B1B68C4
:102A000000995B109B00D31A0C3B1D601C1D13002A
:102A1000083B1B685A108A70D2B28449D2005B000E
:102A200057589B0A009A5B009760FF18039B019A16
:102A3000043B1B685B109B00D3180393794B1B78F6
:102A4000002B01D0FFF7FAFB0022BB5E019A009930
:102A5000A21A92100A61029A1D121340724A9B0038
:102A60009B580237FFF7E8FB231F1868FFF792FA1D
:102A7000AD000600641B1E2837DC002815DC694BFE
:102A80001B78002B01D0FFF7D9FB0022BB5E019A17
:102A90000099A21A92100A61029A1D121340624A0A
:102AA0009B009B580237FFF7C7FB02F027F8033E55
:102AB000361802F023F85E4B801B9842F9D8594B28
:102AC0001B78002B01D0FFF7B9FB0022BB5E019AF7
:102AD0000099A21A92100A61029A1D121340524ADA
:102AE0009B009B580237FFF7A7FB0123009A137046
:102AF00002F004F8009B073886195E60FFF7EFFBD1
:102B0000231F1868FFF746FAAD000600641B002873
:102B100015DC444B1B78002B01D0FFF78FFB002204
:102B2000BB5E019A0099A21A92100A61029A1D12C4
:102B300013403D4A9B009B580237FFF77DFB3D4BFE
:102B4000984204DD1D22374B1A70FFF777FB0123F3
:102B5000009A137001F0D2FFFA239B005E43073EF8
:102B60003018FFF77CFBAB00E41A002328001A00A2
:102B70002100FFF72FFA304E304D3168280003F066
:102B80002FF92F4B31681860280006F06BF9316877
:102B9000280006F0BBFA234B1B78002B01D0FFF76F
:102BA0004DFB0022BB5E019A0099A21A92100A61A5
:102BB000029A1D1213401C4A9B009B580237FFF7D4
:102BC0003BFB184BAD001B78641B002B01D0FFF7BB
:102BD00035FB0022BB5E019A0099A21A92100A618D
:102BE000029A1D121340104A9B009B580237FFF7B0
:102BF00023FB009805F052FE0A4B1B78002B01D0F6
:102C0000FFF71CFB0022BB5E019A0099A21A9210EA
:102C10000A61029A1D121340034A9B009B58023717
:102C2000FFF70AFB08030020FC3A010010250020F2
:102C30007F96980080EE3600F406002009030020FD
:102C400004000020231F1868002840D1083B1968A1
:102C50004810CB0708D4042934D90F23086803404F
:102C6000092B1ED148684010220001234100083A78
:102C70000B431360002867DD01234200211F1A4324
:102C80000A602200083A1168043A19411268091AC8
:102C90001A421FD0C8189840AD001843039BE85053
:102CA00025E0042B05D1080002F05EFEFEF703F9D3
:102CB000DAE7032B06D1010989B2400F89001840D9
:102CC000081AD1E71922DC4B1A70FFF7B7FA401047
:102CD0000138CFE7042A32D90F201668304009287E
:102CE0001BD1881C80008358039AAD00AB50D24B97
:102CF0001B78002B01D0FFF7A1FA0022BB5E019ADE
:102D00000099A21A92100A61029A1D121340CB4A2E
:102D10009B009B580237FFF78FFA042808D1039BCA
:102D2000AD00013110005D19FEF77AFA2860DEE788
:102D3000032804D152181079AD004000ADE71922E4
:102D4000BD4B1A70FFF77AFA0437D0E7AB00019A4F
:102D5000E3189B1AD82B18DC0123002D1ADCB64B84
:102D60001B78002B01D0FFF769FA0022BB5E019AA5
:102D70000099A21A92100A61029A1D121340AF4ADA
:102D80009B009B580237FFF757FA1A22AA4B1A707A
:102D9000FFF754FA2360013D0434DEE7019A231D56
:102DA0009B1AA54ED82B03DD1A233370FFF746FA82
:102DB000019B039AAD00934230D2231F1868FFF79E
:102DC000E9F8011E27DD039B0C3B1A685210824272
:102DD00021DB9007801A9A4B4018C018039B800093
:102DE000C258631B1A60944B641B1B780434002B7D
:102DF00001D0FFF723FA0022BB5E019A0099A21AC4
:102E000092100A61029A1D1213408C4A9B009B5833
:102E10000237FFF711FA20233370E4E71823FBE7AA
:102E2000884BAD001A68631B1C001A60824B043487
:102E30001B78002B01D0FFF701FA0022BB5E019A3C
:102E40000099A21A92100A61029A1D1213407B4A3D
:102E50009B009B580237FFF7EFF9002D02D10023AA
:102E6000FD5E0237231F1A68042A17D16D007F19EF
:102E7000714B1B78002B01D0FFF7E0F90022BB5EFD
:102E8000019A0099A21A92100A61029A1D12134027
:102E90006A4A9B009B580237FFF7CEF91C00E7E710
:102EA000002D02D10023FD5E0237231F1A68042A79
:102EB00019D000226D001A607F195F4B1B78002B20
:102EC00001D0FFF7BBF90022BB5E019A0099A21A5C
:102ED00092100A61029A1D121340584A9B009B5897
:102EE0000237FFF7A9F91C00E7E7A900661A002DD1
:102EF0001CDC1C22504B1A70002333604E4B641AAA
:102F00001B780434002B01D0FFF798F90022BB5E38
:102F1000019A0099A21A92100A61029A1D12134096
:102F2000464A9B009B580237FFF786F93368350005
:102F30005A108B199C4601232868034003D10D20A9
:102F40003D4A1070D9E74010824200DD020004358E
:102F5000AC45F0D1012352001343CEE7A900661A15
:102F6000002D1CDC1C22344B1A7000233360324BC2
:102F7000641A1B780434002B01D0FFF75FF900229C
:102F8000BB5E019A0099A21A92100A61029A1D1260
:102F900013402A4A9B009B580237FFF74DF93368CC
:102FA00035005A108B199C4601232868034003D131
:102FB0000D20214A1070D9E74010824200DA020049
:102FC0000435AC45F0D1012352001343CEE7230072
:102FD0000122083B1968AE00114223D0231F1B6851
:102FE00013421FD0114113410022994200DA0432EA
:102FF000A31B1A60104BA41B1B780434002B01D0B8
:10300000FFF71CF90022BB5E019A0099A21A9210E8
:103010000A61029A1D121340084A9B009B5802370E
:10302000FFF70AF90220231F1A684042FEF72AFF21
:10303000A51B2860DEE7C04608030020FC3A01001B
:10304000FCFFFF3F040000202300083B1968012318
:10305000AE00194224D0221F12681A4220D0194112
:103060005010CB0FD21788425341A21B9B00136014
:10307000E24BA41B1B780434002B01D0FFF7DEF8D1
:103080000022BB5E019A0099A21A92100A61029A6C
:103090001D121340DA4A9B009B580237FFF7CCF809
:1030A0000120231F1A684042FEF7ECFEA51B286092
:1030B000DEE72300083B1868231F1968AE00A61B33
:1030C0000423814202D0042802D80023336016E092
:1030D00001231842F9D10F2302681A40042AF4D1BF
:1030E000033A1142F1D10429EFD90A681340042BA5
:1030F000EBD1FEF72DFF431E984180003060BF4B9F
:10310000AD001B78641B0434002B01D0FFF796F848
:103110000022BB5E019A0099A21A92100A61029ADB
:103120001D121340B64A9B009B580237FFF784F8E4
:103130002300083B1868231F1968AE00A61B002354
:10314000814202D0042802D80423336016E0012310
:103150001842F9D10F2302681A40042AF4D1033A25
:103160001142F1D10429EFD90A681340042BEBD1A5
:10317000FEF7EEFE43425841800030609F4BAD00A9
:103180001B78641B0434002B01D0FFF757F8002292
:10319000BB5E019A0099A21A92100A61029A1D124E
:1031A0001340974A9B009B580237FFF745F82300CE
:1031B0000122083B1968AE00114224D0231F1B686E
:1031C000134220D05B104A10D80FC9179A424141D0
:1031D000A31B89001960894BA41B1B780434002BA6
:1031E00001D0FFF72BF80022BB5E019A0099A21ACA
:1031F00092100A61029A1D121340814A9B009B584B
:103200000237FFF719F8231F1A680120FEF73AFE6C
:10321000A51B2860DFE723000122083B1968AE00E8
:10322000114223D0231F1B6813421FD011411341A9
:103230000022994200DD0432A31B1A606F4BA41BCD
:103240001B780434002B01D0FEF7F8FF0022BB5E90
:10325000019A0099A21A92100A61029A1D12134053
:10326000674A9B009B580237FEF7E6FF231F1A6848
:103270000220FEF707FEA51B2860DFE7231F1B685F
:10328000AD00043B5A1E9341621B14009B00136067
:103290005A4B04341B78002B01D0FEF7CFFF0022DD
:1032A000BB5E019A0099A21A92100A61029A1D123D
:1032B0001340534A9B009B580237FEF7BDFF230083
:1032C000083B1868FEF766FE231F06001868FEF725
:1032D00061FE36180120AD00631B1C00760006431A
:1032E0001E60464B04341B78002B01D0FEF7A6FF6E
:1032F0000022BB5E019A0099A21A92100A61029AFA
:103300001D1213403E4A9B009B580237FEF794FF64
:103310002300083B1868FEF73DFE231F06001868CF
:10332000FEF738FE361A0120AD00631B1C00760044
:1033300006431E60314B04341B78002B01D0FEF78E
:103340007DFF0022BB5E019A0099A21A92100A61C9
:10335000029A1D1213402A4A9B009B580237FEF71F
:103360006BFF2300083B1868FEF714FE231F0600BE
:103370001868FEF70FFE46430120AD00631B1C00DA
:10338000760006431E601D4B04341B78002B01D0D1
:10339000FEF754FF0022BB5E019A0099A21A921018
:1033A0000A61029A1D121340154A9B009B5802376E
:1033B000FEF742FF231F1868FEF7ECFD061E21D121
:1033C0001F230E4A1370AD00631B1C001E600B4BC5
:1033D00004341B78002B01D0FEF730FF0022BB5EC7
:1033E000019A0099A21A92100A61029A1D121340C2
:1033F000034A9B009B580237FEF71EFF080300207C
:10340000FC3A01002300083B1868FEF7C3FD3100B9
:103410000AF008FB012640000643D4E7AD00661B16
:103420003068FEF7B7FD06907068FEF7B3FD002820
:103430001BD11F22E44B1A70E34B641B1B783060D6
:103440000434002B01D0FEF7F9FE0022BB5E019A86
:103450000099A21A92100A61029A1D121340DB4AC7
:103460009B009B580237FEF7E7FEC21783185340B4
:103470001900069804930AF0BBFB002901DA049BAB
:10348000C918012049000843D6E7231F1868FEF732
:1034900081FDC217801850400122AD00631B1C0043
:1034A000400010431860C84B04341B78002B01D037
:1034B000FEF7C4FE0022BB5E019A0099A21A921088
:1034C0000A61029A1D121340C04A9B009B580237A2
:1034D000FEF7B2FEAB00E31A06950493012D07D167
:1034E0001868FEF757FD061E0EDA01256D420BE047
:1034F000022D35D1049B1868FEF74CFD049B050096
:103500005868FEF747FD0600B54202DC33002E0086
:103510001D000135AD1B0EF011F829000AF068FB03
:103520008E190121049B76000E431E60069B9B00B2
:10353000E41AA54B04341B78002B01D0FEF77EFE65
:103540000022BB5E019A0099A21A92100A61029AA7
:103550001D1213409D4A9B009B580237FEF76CFEDC
:1035600064250126D5E7AB00E61A31002800049354
:1035700002F07DFC049B3060E41A934B04341B780A
:10358000002B01D0FEF75AFE0022BB5E019A009983
:10359000A21A92100A61029A1D1213408B4A9B00D4
:1035A0009B580237FEF748FE2300083B1868FEF7D9
:1035B000F1FC231F06001868FEF7ECFC0640012012
:1035C000AD00631B1C00760006431E607E4B043476
:1035D0001B78002B01D0FEF731FE0022BB5E019A62
:1035E0000099A21A92100A61029A1D121340774A9A
:1035F0009B009B580237FEF71FFE2300083B18680C
:10360000FEF7C8FC231F06001868FEF7C3FC06433C
:103610000120AD00631B1C00760006431E606A4B50
:1036200004341B78002B01D0FEF708FE0022BB5E9D
:10363000019A0099A21A92100A61029A1D1213406F
:10364000624A9B009B580237FEF7F6FD2300083BB9
:103650001868FEF79FFC231F06001868FEF79AFC07
:1036600046400120AD00631B1C00760006431E602F
:10367000554B04341B78002B01D0FEF7DFFD0022F0
:10368000BB5E019A0099A21A92100A61029A1D1259
:1036900013404E4A9B009B580237FEF7CDFD231F77
:1036A0001868FEF777FCC0430122AD00631B1C00C5
:1036B000400010431860444B04341B78002B01D0A9
:1036C000FEF7BCFD0022BB5E019A0099A21A92107F
:1036D0000A61029A1D1213403C4A9B009B58023714
:1036E000FEF7AAFD2300083B1868FEF753FC231FD2
:1036F00006001868FEF74EFC86400122AD00631BF1
:103700001C00760016431E602F4B04341B78002BE0
:1037100001D0FEF793FD0022BB5E019A0099A21A28
:1037200092100A61029A1D121340284A9B009B586E
:103730000237FEF781FD2300083B1868FEF72AFCDC
:10374000231F06001868FEF725FC06410122AD0084
:10375000631B1C00760016431E601B4B04341B7851
:10376000002B01D0FEF76AFD0022BB5E019A009992
:10377000A21A92100A61029A1D121340134A9B006A
:103780009B580237FEF758FDAB00E31A9C46012D0B
:1037900054D11A6813002B4050D1042A52D90F205B
:1037A00011680840190009284AD111000831049114
:1037B0002E001900526852100692069A8A4207DCBF
:1037C00001225B001A430CE008030020FC3A0100D0
:1037D00004988A008058020032401DD12721DB4B1B
:1037E000197063461A60D94BAD001B78641B043412
:1037F000002B01D0FEF722FD0022BB5E019A00994A
:10380000A21A92100A61029A1D121340D04A9B001C
:103810009B580237FEF710FD40101B180131CCE712
:1038200040101B1801318D42CADD60468A00805865
:1038300002003240F4D1C54B0D21D1E700210B002D
:103840000126F0E71900FBE723000C3B1868FEF7A0
:10385000A1FB2300083B06001868FEF79BFBF1174D
:103860000200C31730000AF059FA231F0490059193
:103870001868FEF78FFB0200049805990AF0BEF95C
:1038800043000120AE00A51B2C001843AF4B28605D
:103890001B780434002B01D0FEF7D0FC0022BB5E65
:1038A000019A0099A21A92100A61029A1D121340FD
:1038B000A74A9B009B580237FEF7BEFCAB00E61AF6
:1038C000310028000493FDF72FFF049B3060E41AB9
:1038D0009E4B04341B78002B01D0FEF7AFFC002276
:1038E000BB5E019A0099A21A92100A61029A1D12F7
:1038F0001340974A9B009B580237FEF79DFCAB0094
:10390000E61A310028000493FDF72AFF049B30607B
:10391000E41A8E4B04341B78002B01D0FEF78EFC8A
:103920000022BB5E019A0099A21A92100A61029AC3
:103930001D121340864A9B009B580237FEF77CFC01
:10394000AB00E41A21002800FDF7AAFF7F4B1B788B
:10395000002B01D0FEF772FC0022BB5E019A009999
:10396000A21A92100A61029A1D121340784A9B0013
:103970009B580237FEF760FCAB00E61A31002800C6
:103980000493FEF715F8049B3060E41A6F4B04347F
:103990001B78002B01D0FEF751FC0022BB5E019A80
:1039A0000099A21A92100A61029A1D121340684AE5
:1039B0009B009B580237FEF73FFC231F186801F05D
:1039C000D3FF2200083A12680300AD00D10731D4BA
:1039D000002A0ED0042A0CD010680F2210400138A3
:1039E00008280FD809F076FF05262C280E0E0E0E9B
:1039F0002A00584918000DF053FE43425841631BFA
:103A000080001860514B641B1B780434002B01D0DC
:103A1000FEF714FC0022BB5E019A0099A21A9210D4
:103A20000A61029A1D121340494A9B009B580237B3
:103A3000FEF702FC4849DDE74849DBE74849D9E79A
:103A40004849D7E7019B261DF31A0493D82B04DDC0
:103A50001A223E4B1A70FEF7F1FB01F07DF8FA22B4
:103A6000002392000AF03AF93F4B4000184001232E
:103A70001843364B20601B78002B01D0FEF700FC6A
:103A80000022BB5E049A009992100A61029A1D12EC
:103A900013402F4A9B009B5834000237FEF7CCFBA3
:103AA000019A231D04939E1AD82E04DD1A22274B57
:103AB0001A70FEF7C3FB01F021F82B4B40001840B1
:103AC00001231843214B20601B78002B01D0FEF707
:103AD000D9FB0022BB5E009AB6101661029A1D1235
:103AE00013401B4A9B009B58049C0237FEF7A4FB23
:103AF000019B261DF31A0493D82B04DD1A22134BC5
:103B00001A70FEF79BFB01F003F8184B1A68831A32
:103B1000904201D2164A9B1801205B0003432360A8
:103B20000A4B1B78002B01D0FEF7AEFB0022BB5ED8
:103B3000049A009992100A61029A1D121340044AD5
:103B40009B009B5834000237FEF776FB08030020E9
:103B5000FC3A0100F7370100FF3701000638010089
:103B60000D38010012380100FEFFFF7F0007002022
:103B700037894100FEF7D2FAF34BAD001B78641B86
:103B8000002B01D0FEF75AFB0022BB5E019A009980
:103B9000A21A92100A61029A1D121340EB4A9B006E
:103BA0009B580237FEF748FB05F082F8AE0000286C
:103BB00016D1E54BA41B1B78002B01D0FEF73EFB72
:103BC0000022BB5E019A0099A21A92100A61029A21
:103BD0001D121340DD4A9B009B580237FEF72CFB59
:103BE0000123A61B28001A003100FEF7F3F9D84D77
:103BF0002868643004F0D8FD002802D1023FFEF7A7
:103C00006EFB009B29685A78D24804F0E7FF012335
:103C1000009A3400137000F071FFCF4B2A681B68C4
:103C2000063253431818009B5860FEF758FB05F006
:103C30003FF8AE00002816D1C34BA41B1B78002B05
:103C400001D0FEF7FBFA0022BB5E019A0099A21A8E
:103C500092100A61029A1D121340BC4A9B009B58A5
:103C60000237FEF7E9FAA61B2800012300223100E3
:103C7000FEF7B0F9B64D2868643004F095FD0028D1
:103C8000BCD0B44804F06DFFC1E7AD00661BFEF781
:103C90004DFA3400AC4B30601B780434002B01D05B
:103CA000FEF7CCFA0022BB5E019A0099A21A92108C
:103CB0000A61029A1D121340A44A9B009B580237C6
:103CC000FEF7BAFAA04EAA00012D1BDC1C2300212E
:103CD0003370A31A19603378A41A0434002B01D06E
:103CE000FEF7ACFA0022BB5E019A0099A21A92106C
:103CF0000A61029A1D121340944A9B009B58023796
:103D0000FEF79AFA231F18680399019BA51A8B42A4
:103D100001D32860DFE72300083B1B685B10002B02
:103D2000F7DD03990C39096849108B42F1DC8B48A7
:103D30001B18591A039B8900C858EAE7AD00661B97
:103D4000300000F048FF34007F4B30601B780434B3
:103D5000002B01D0FEF772FA0022BB5E019A009997
:103D6000A21A92100A61029A1D121340774A9B0010
:103D70009B580237FEF760FAAD00661B300000F07A
:103D80002CFF3400704B30601B780434002B01D0C2
:103D9000FEF754FA0022BB5E019A0099A21A921013
:103DA0000A61029A1D121340684A9B009B58023711
:103DB000FEF742FAAB00E61A31002800049300F047
:103DC0002DFD049B3060E41A5F4B04341B78002BFC
:103DD00001D0FEF733FA0022BB5E019A0099A21AC5
:103DE00092100A61029A1D121340584A9B009B5878
:103DF0000237FEF721FAAD00641B200000F0F0FE50
:103E0000514B1B78002B01D0FEF718FA0022BB5E45
:103E1000019A0099A21A92100A61029A1D12134087
:103E20004A4A9B009B580237FEF706FAAB00E61A97
:103E300031002800049300F0C9FC049B3060E41AB0
:103E4000414B04341B78002B01D0FEF7F7F9002218
:103E5000BB5E019A0099A21A92100A61029A1D1281
:103E600013403A4A9B009B580237FEF7E5F9AD0034
:103E7000641B200000F01EFF334B1B78002B01D089
:103E8000FEF7DCF90022BB5E019A0099A21A92109B
:103E90000A61029A1D1213402C4A9B009B5802375C
:103EA000FEF7CAF90121280000F0DEFE264B1B7840
:103EB000002B01D0FEF7C2F90022BB5E019A0099E7
:103EC000A21A92100A61029A1D1213401F4A9B0007
:103ED0009B580237FEF7B0F90021280000F0C4FE1D
:103EE000194B1B78002B01D0FEF7A8F90022BB5E0E
:103EF000019A0099A21A92100A61029A1D121340A7
:103F0000124A9B009B580237FEF796F9AD00661BDC
:103F1000300000F0FDFE34000B4B30601B780434A1
:103F2000002B01D0FEF78AF90022BB5E019A0099AE
:103F3000A21A92100A61029A1D121340034A9B00B2
:103F40009B580237FEF778F908030020FC3A01007D
:103F5000F40600200903002000000020FCFFFF3FC2
:103F6000AD00661B300000F0E7FE3400E84B306027
:103F70001B780434002B01D0FEF760F90022BB5EF1
:103F8000019A0099A21A92100A61029A1D12134016
:103F9000E04A9B009B580237FEF74EF9AD00641BC8
:103FA000200000F09DFEDA4B1B78002B01D0FEF7BD
:103FB00045F90022BB5E019A0099A21A92100A618B
:103FC000029A1D121340D34A9B009B580237FEF7FA
:103FD00033F9AD00641B200005F0E6FECC4B1B78E6
:103FE000002B01D0FEF72AF90022BB5E019A00994E
:103FF000A21A92100A61029A1D121340C54A9B0030
:104000009B580237FEF718F9AD00661B300005F02B
:10401000D5FF3400BE4B30601B780434002B01D038
:10402000FEF70CF90022BB5E019A0099A21A9210C9
:104030000A61029A1D121340B64A9B009B58023730
:10404000FEF7FAF8AD00641B200005F001FEB04B4E
:104050001B78002B01D0FEF7F1F80022BB5E019A1D
:104060000099A21A92100A61029A1D121340A94ADD
:104070009B009B580237FEF7DFF8AD00661B30004F
:1040800005F01CFE3400A24B30601B780434002B7A
:1040900001D0FEF7D3F80022BB5E019A0099A21A64
:1040A00092100A61029A1D1213409A4A9B009B5873
:1040B0000237FEF7C1F8019B261DF31A0493D82B93
:1040C00004DD1A22924B1A70FEF7B8F800F044FD96
:1040D0000023914A09F002FE904B40001840012352
:1040E00018438B4B20601B78002B01D0FEF7CEF8D5
:1040F0000022BB5E049A009992100A61029A1D1276
:104100001340844A9B009B5834000237FEF794F812
:10411000AB00E61A069333685B100493012D26DD8D
:104120007068C30723D54010049BC01A02D58023B2
:10413000DB05C018012340001843069B3060E41AD9
:10414000734B04341B78002B01D0FEF777F8002264
:10415000BB5E019A0099A21A92100A61029A1D127E
:1041600013406C4A9B009B580237FEF765F800F03D
:10417000F3FCFA220023920009F0B0FD80008008D1
:10418000D2E7AB00E61A069333685B100493012D67
:1041900026DD7068C30723D54010049BC01A02D5E2
:1041A0008023DB05C018012340001843069B3060C4
:1041B000E41A574B04341B78002B01D0FEF73EF86D
:1041C0000022BB5E019A0099A21A92100A61029A1B
:1041D0001D1213404F4A9B009B580237FEF72CF8E4
:1041E00000F08CFC80008008D7E7019B221DD11ACB
:1041F000D82904DD1A22464B1A70FEF71FF87B8877
:104200003D881B042B432360414B381D1B78002B3A
:1042100001D0FEF73DF804203B5E00988910016153
:1042200002991D120B403B499B005B581400063756
:10423000FEF702F83E88BB1CB005400D3818049309
:1042400001F092FBEDB2AB00E41A01002300B00ACA
:104250002A0004F07BFD2E4B1B78002B01D0FEF7CB
:104260001AF80222BB5E019A0099A21A92100A6102
:10427000029A1D121340274A9B009B580437FDF7F2
:10428000DBFF3E88BB1CB005400D07933818EBB22E
:10429000049301F069FB049B01009B00E51A06935F
:1042A000B00A2B00049A04F051FD069B2860E41A22
:1042B000174B04341B78002B01D0FDF7EEFF0222D0
:1042C000BB5E019A0099A21A92100A61029A1D120D
:1042D0001340104A9B009B580437FDF7ADFF2200A6
:1042E000002D00DC8FE001204042FDF7F7FE231F88
:1042F0001E68012D14D12E4207D1042E05D90F239B
:10430000326830001340042B18D001235B421AE0BE
:1043100008030020FC3A010040420F00FEFFFF7F2F
:10432000022DF2D12300083B1868C307EDD40428FE
:10433000EBD90F2302681340042BE6D101F014FBE4
:10434000FDF73EFF0300AA00A21A591C5BD0022D04
:1043500037D1012131402CD1042E2AD90F203468C5
:104360002040092825D17068019D4010C0B284000A
:10437000A4461419651BD82D09DD2F4B1A3119706D
:104380001400FDF75BFF7518AD68555004318C457E
:10439000F9D1019A0099A21A92100A61FF2219001C
:1043A0009143264A91420FD11B061B0C1843FEF77E
:1043B00099FA0B21204B141D197000231360FDF78F
:1043C0003DFF14000020E4E78500651B29009847A5
:1043D00000221B4B2C1D1A60174B28601B78934240
:1043E00001D0FDF72BFF0022BB5E019A0099A21AB3
:1043F00092100A61029A1D121340124A9B009B58A8
:104400000237FDF719FF002313600B4B141D1B78B7
:10441000002B01D0FDF712FF0022BB5E019A00992C
:10442000A21A92100A61029A1D121340054A9B00BB
:104430009B580237FDF700FF0803002000FFFFFF35
:10444000D00B0020FC3A01000023F7B51D005C1ED4
:10445000002B12DA04F060FF04F044FD02F0D4FEF9
:1044600000F064FB00F078FB002904D1224B984255
:1044700001D804F089FE5F2404E00F231C4201D11F
:1044800004F038FF0023180001931C4B019A1B68AD
:1044900093420FDD0135AB4200DC0025F0266E4370
:1044A000174FF35D002B22D0F619022B0ED13000EE
:1044B000FDF79EFE134B1A68002A05D000221A60F1
:1044C000114B9C4200DD1C002300C0E7012B0ED1E4
:1044D000002801D100F012FBF0226A43BB185B6890
:1044E0000A49C31A8B4202D80223BB54DFE7019B5F
:1044F00001330193C9E7C046BFE1E400F80600209C
:10450000B01B0020FC060020881300007F96980056
:1045100080220B4B52001A600121A822A920094BCE
:10452000D20019649A58C00005321A5006481A5031
:10453000C122C020920000039850044B19707047AC
:1045400000E100E0008000404C0500004C07002026
:104550000020704704207047F8B550C9012322009D
:104560001A40101E2DD03340181E2AD0641000208F
:104570001A2C26D81D4B761035009E4200DD1D00FA
:104580001B4F3B5D012B05D00121200007F070FB84
:1045900001233B55174B1B78002B01D1FFF7B8FFC8
:1045A0000023154A9E420DDCFF2514491448D65CB1
:1045B000B44202D15E007052D5540133082BF6D1BB
:1045C0000420F8BDD15C8C4203D10C4A5B009D52A3
:1045D000F6E70133082BF5D10023D15CFF2901D187
:1045E000D454F2E70133082BF7D1E9E78813000030
:1045F000240700204C070020200000200A00002093
:10460000DC05000070B530C9012322001A40101EDD
:104610001FD02B40181E1CD064101A2C00D919244E
:10462000174E335D012B05D00121200007F020FB40
:104630000123335569100800124A1038124B90427A
:1046400008D901220021524220001A6007F02EFBF7
:10465000042070BD1C600D4809F0E4F90C4B040007
:1046600018800C4B1B78002B01D1FFF751FF012262
:10467000094B9A64A922D200995864189C50E7E724
:1046800024070020908601001C00002020A10700C4
:10469000080000204C07002000800040012370B576
:1046A0000D681C00984200DD4C682A001A40101E5C
:1046B0000BD022001A40101E07D06D10002D05DC13
:1046C000A12200201E49D2008B5070BD6410002032
:1046D0001A2CFAD81B4E335D012B05D00121200086
:1046E00007F0C6FA012333552900174809F09AF953
:1046F0000A21053009F096F9144BA400E258144B36
:1047000012021343A2221349D2008B50124C0C4BBD
:104710009C50124C1951012411495C50114B1969DC
:1047200000219950104A904200DD1000A8228021FB
:10473000D2009850012289005A5004201A60C4E720
:1047400000F001402407002000B4C404F05A010026
:10475000030003000060004040A100401405000079
:104760000405000000A00040FFFF0000030010B59A
:104770000120002B02DC1B30FDF7A2FC10BD000065
:1047800010B5C3071BD4002819D0042802D1022376
:10479000180010BD0F2302681340042B0FD101F045
:1047A000E3F80400010007480CF07AFF0028EED07F
:1047B000210005480CF074FF03230028E8D00023F3
:1047C000E6E7C046D45001004C3D010070B501251C
:1047D0000C682C4204D10D20FDF772FC280070BD3E
:1047E00064101A2C16D80026012803DD4868FFF74C
:1047F000C7FF0600084D2B5DB34204D031002000F6
:1048000007F036FA2E55200007F066FA0300042060
:10481000012BE4D00020E2E72407002070B501243A
:104820000D68254204D10D20FDF74AFC200070BD23
:104830006D100026012803DD4868FFF7A1FF060080
:104840000124002D04D105F04BFAA0402043EEE7EF
:104850002000072DEBD8094BAD00EC58084D2B5D1F
:10486000B34204D03100200007F002FA2E55200098
:1048700007F0ACF8430001201843D8E7CC3D010015
:104880002407002010B50124044002D04410200069
:1048900010BD042810D90F2302681340042B07D140
:1048A00001F062F821000A220CF0CCFF0400EEE7D0
:1048B000032B01D10430F5E70D20FDF701FCE6E7FD
:1048C000F8B50C00022803DC1C20FDF7F9FBF8BD4D
:1048D0000868FFF7D7FF06006068FFF7D3FF050001
:1048E000A068FFF7CFFF0100794809F09BF8841E0C
:1048F0001A2D01D90020EAE7764F7B5D012B05D008
:104900000121280007F0B4F901237B55002128007C
:1049100007F0CCF9002C0ED020000138C046C0466C
:10492000C046C046C046C046C046C046C046C04657
:10493000C046C046F1D1012731002800394007F0B8
:10494000B5F9002C0ED020000138C046C046C04644
:10495000C046C046C046C046C046C046C046C04627
:10496000C046F1D171103940280007F09FF9002CA2
:104970000ED020000138C046C046C046C046C046E2
:10498000C046C046C046C046C046C046C046F1D13B
:104990000127B1103940280007F088F9002C0ED00B
:1049A00020000138C046C046C046C046C046C0468A
:1049B000C046C046C046C046C046C046F1D1F11010
:1049C0003940280007F072F9002C0ED02000013881
:1049D000C046C046C046C046C046C046C046C046A7
:1049E000C046C046C046C046F1D10127311139400A
:1049F000280007F05BF9002C0ED020000138C046DB
:104A0000C046C046C046C046C046C046C046C04676
:104A1000C046C046C046F1D171113940280007F0A8
:104A200045F9002C0ED020000138C046C046C046D3
:104A3000C046C046C046C046C046C046C046C04646
:104A4000C046F1D10127B1113940280007F02EF9F5
:104A50003900002C0ED020000138C046C046C046A8
:104A6000C046C046C046C046C046C046C046C04616
:104A7000C046F1D1F6113140280007F017F9002C9B
:104A80000ED020000138C046C046C046C046C046D1
:104A9000C046C046C046C046C046C046C046F1D12A
:104AA0000121280007F002F9002C00D122E72000A4
:104AB0000138C046C046C046C046C046C046C04693
:104AC000C046C046C046C046C046F1D112E7C04607
:104AD00040420F0024070020042070470020704748
:104AE00010B5002803DC1C20FDF7EAFA10BD0B68A6
:104AF0000020DB07FAD40D30F6E700000122034B5B
:104B00001A64A822D20098587047C046008000401E
:104B10000122054B10B51A64A822FA21D200985838
:104B2000890008F0F5FE10BD008000400122074B0F
:104B30001A64A822D2009958054A13688B4203D9F7
:104B4000044803680133036011607047008000402F
:104B5000440700204807002010B5FFF7E7FF0122B7
:104B6000034B1968034B1A64A822D200985810BD51
:104B7000480700200080004000487047EC3D0100DD
:104B80001B20704770B504000D001A2806D8044E8B
:104B9000335C8B4202D007F06BF8355570BDC046D0
:104BA0002407002070B50024074D635D013B022BF4
:104BB00005D80021200007F05BF80023635501347D
:104BC0001B2CF1D170BDC046240700201A2801D942
:104BD0000120404270471120704737207047000085
:104BE000F8B5012704683C4202D045683D4203D134
:104BF0000D20FDF765FAF8BD64101A2CFBD8124E93
:104C0000335D012B04D03900200007F031F837550F
:104C10000E496D108D4202DCE943C917294020007E
:104C200006F05AFF0A4B1A68002A06D1A222032076
:104C30000849D200885001221A60335D012BDAD175
:104C4000054A1355D7E7C04624070020FF0300009C
:104C500050070020009000400407002010B5080015
:104C6000FFF7BEFF002010BD70B505000C001A282C
:104C700014D80E4E335C012B04D0012106F0F8FF4E
:104C8000012373550A4B5B5D002B08D0611E8C41DC
:104C900061428905890D280006F01EFF70BD2100C4
:104CA00028004C1EA14107F001F8F7E72407002077
:104CB00004070020036810B5DA0703D40D20FDF7C0
:104CC000FFF910BD4168581004394A425141FFF7BD
:104CD000CBFFF6E710B50800FFF7ECFF002010BD92
:104CE00037B569460A00064B30CB30C20368022054
:104CF000042B02D102F024F937BD02F049F9FBE799
:104D0000443D010010B50800FFF7EAFF002010BD88
:104D100010B5084C237D002B05D00021142006F08F
:104D2000A7FF00232375142006F0D6FF4342584105
:104D3000800010BD2407002010B5084CA37D002B77
:104D400005D00021162006F093FF0023A37516203E
:104D500006F0C2FF43425841800010BD24070020E6
:104D6000A1230121034ADB00D1500021024A08336C
:104D7000D150704700F0014000600040F7B52F4D62
:104D80002F4EEB6C002B14D0A9240023E4003759DC
:104D9000EB642C4B186800280BDB2B4B19784A422C
:104DA0005141C9B2197006F081FF284B1B88DF19E9
:104DB00037512B6D002B38D00021254B254FF4584F
:104DC00029653A780193244D8A4206D02B68072B37
:104DD00003D8224AD05C06F069FF2B68204A0133D1
:104DE000134004D50822013B5242134301331B49AF
:104DF00000228C462B60082B18D06046C05C591CE2
:104E0000FF2802D10B000122F5E7002A00D02B6019
:104E1000012106F04BFF01233B702B68114A5B0018
:104E20009B5A0C34E418019BF450F7BD01235B42FC
:104E30002B6000233B700C4BF4E7C046FC80004025
:104E4000008000401C0000204007002008000020D7
:104E50004C0500003F070020200700202000002014
:104E6000070000800A0000205C46000030B50023E7
:104E7000FF25074C074A084859001D550133885241
:104E8000082BF9D10023054A1370054A136030BD81
:104E9000200000200A000020DC0500003F07002061
:104EA000200700200122024B52421A607047C04680
:104EB0001C00002070B50D000100214808F0B2FD73
:104EC0000400FA2080006843610008F0ABFD012176
:104ED0000600192006F0CCFE0025B5422BDA012190
:104EE000192006F0E3FE002C0ED020000138C04649
:104EF000C046C046C046C046C046C046C046C04682
:104F0000C046C046C046F1D10021192006F0CEFEB1
:104F1000002C0ED020000138C046C046C046C04616
:104F2000C046C046C046C046C046C046C046C04651
:104F3000F1D10135D1E70021192006F099FE70BDAD
:104F400020A107007047704710B5034B0F2203499B
:104F5000032003F053FB10BD543D010044500100F9
:104F6000E12170B549021D4806F0C9F9002401226B
:104F700003201B4B1B491A615C50043158508018A8
:104F8000083158501A60063006F01AFDFF21164A03
:104F9000A15401341B2CFBD101220020134B010032
:104FA0001A600423124A134D1468002CFCD02C689C
:104FB0000002013B20431160002BF5D101220E4B72
:104FC0001A6006F01BFC02F065FA05F00AFC05F019
:104FD00009FC9622094B12041A6070BD601A002069
:104FE00000800040040500002407002000D000409D
:104FF00000D1004008D5004004D00040300000201F
:1050000000B57F2800DC61E39F4B984200D176E336
:1050100000DD67E1EA2800D189E300DD8FE0BD28EB
:1050200001D100F0B4FB46DCAC2801D100F0ADFBAF
:105030001DDCA32800D194E30ADCA12800D1A8E359
:1050400000DD8CE3A02801D100F011FCDB203DE362
:10505000A72800D14FE303DCA528F7D19D2035E335
:10506000AA2800D18DE3AB28F0D1AE202EE3B628DC
:1050700000D13EE310DCB12801D100F0E8FB03DCF5
:10508000B028E3D1F82021E3B22801D100F0EBFBF6
:10509000B528DBD1E62019E3BA2800D173E303DC9D
:1050A000B728D3D1FA2011E3BB2800D173E3BC2881
:1050B000CCD1AC200AE3DF2801D100F0B4FB21DC25
:1050C000C72800D127E30EDCC42800D139E303DC74
:1050D000BF28BBD1A820F9E2C52800D133E3C628F8
:1050E000B4D19220F2E2D12800D148E303DCC928F0
:1050F000ACD19020EAE2D62800D12EE3DC28A5D15D
:105100009A20E3E2E52800D10DE30BDCE12800D191
:105110002DE300DA05E3E22800D100E3E42895D18D
:105120008420D3E2E72800D1FFE200DA0DE3E8288B
:1051300000D100E3E92800D088E78220C6E2534B83
:10514000984200D173E34FDCF62800D1FFE221DC66
:10515000EF2800D1F1E20CDCEC2800D1EFE200DA1C
:10516000E7E2ED2800D104E3EE2800D06EE78C20C2
:10517000ACE2F22800D1ECE204DCF12800D065E7D3
:10518000A420A3E2F32800D1F5E2F42800D05DE7E3
:1051900093209BE2FC2800D1BFE210DCF92800D16B
:1051A000D9E204DCF72800D050E7F6208EE2FA2896
:1051B00000D1E2E2FB2800D048E7962086E2C9232E
:1051C0005B00984200D1D0E204DCFF2800D03DE72C
:1051D00098207BE22E4B984200D126E3053398427B
:1051E00000D033E7E92071E22A4B984200D174E203
:1051F0002FDC294B984200D123E314DC274B984243
:1052000000D11AE305DC264B984200D01EE7E820C7
:105210005CE2244B984200D103E30333984200D070
:1052200014E7EB2052E2204B984200D101E305DC69
:10523000033B984200D009E7E32047E2F1239B00BB
:10524000984200D1F7E2194B984200D0FEE6ED20DB
:105250003CE2174B984200D153E233DC154B9842A5
:1052600000D1FEE205DC144B984200D0EEE613209C
:105270002CE2124B984200D175E2114B984200D0BB
:10528000E4E61B2022E2C046A8210000A3030000A0
:105290009303000022200000B5030000A9030000D2
:1052A000A6030000B1030000C3030000C603000012
:1052B000912100007F2000003C200000A72000007A
:1052C00090210000AB4B984200D11CE200DA1CE2B6
:1052D000A94B984200D11AE2A84B984200D0B5E6FB
:1052E0001220F3E1A64B984200D176E200DDBCE04B
:1052F000A44B984200D16EE263DCA34B984200D1EC
:1053000007E22EDCA14B984200D19CE214DCA04BBA
:10531000984200D1A3E205DC9E4B984200D095E66E
:10532000F920D3E19C4B984200D188E29B4B9842F4
:1053300000D08BE61C20C9E1994B984200D184E251
:1053400005DC984B984200D080E6F720BEE1964BF2
:10535000984200D17DE2954B984200D076E6F2204B
:10536000B4E1934B984200D119E215DC914B98427D
:1053700000D170E205DC904B984200D066E6A9208F
:10538000A4E18E4B984200D167E2E033FF339842AC
:1053900000D05BE6C42099E1894B984200D112E22B
:1053A00005DC884B984200D050E6DA208EE1864B2F
:1053B000984200D109E2854B984200D046E6D920B8
:1053C00084E1834B984200D1F1E129DC814B984282
:1053D00000D10CE214DC804B984200D1F9E105DCED
:1053E0007E4B984200D031E6B4206FE17C4B98426E
:1053F00000D1ECE17B4B984200D027E6C52065E167
:10540000794B984200D1FEE100DAD2E1774B984225
:1054100000D1FAE1764B984200D017E6C92055E159
:10542000744B984200D1DAE10FDC734B984200D103
:10543000C1E100DAB9E1714B984200D1E1E1704B72
:10544000984200D002E6D32040E16E4B984200D152
:10545000B5E100DAB5E16C4B984200D1ADE16B4BA0
:10546000984200D0F2E5C62030E1694B984200D165
:1054700093E153DC674B984200D1B2E124DC664BE8
:10548000984200D1B9E10FDC644B984200D188E129
:1054900000DAAAE1624B984200D184E1614B984264
:1054A00000D0D3E5B92011E15F4B984200D19AE1D9
:1054B00000DAA4E15D4B984200D19CE15C4B98423C
:1054C00000D0C3E5D02001E15A4B984200D1A2E1BF
:1054D0000FDC594B984200D199E100DA99E1574B22
:1054E000984200D185E11433984200D0AEE5DF2028
:1054F000ECE0534B984200D18FE105DC514B9842D0
:1055000000D0A3E5DB20E1E04F4B984200D186E1DB
:105510004E4B984200D099E5B020D7E04C4B9842D2
:1055200000D1A6E100DDACE04A4B984200D1DCE0BE
:1055300014DC494B984200D197E105DC474B984277
:1055400000D083E5B220C1E0454B984200D1D4E0C1
:10555000444B984200D079E51E20B7E0424B984278
:1055600000D1C4E000DD83E0404B984200D06DE5FF
:105570001F20ABE093210000942100009521000042
:105580005F2500001C2500000223000029220000E6
:105590001A220000192200001E2200001F22000013
:1055A0006122000048220000642200006522000001
:1055B000022500002023000010230000212300000A
:1055C000102500000C2500001425000018250000FF
:1055D00055250000502500002C2500002425000042
:1055E000342500003C250000522500005325000012
:1055F000542500005A2500005725000058250000BA
:10560000592500005C2500005D2500005E25000096
:105610009225000069250000642500006125000036
:105620006225000063250000662500006725000054
:1056300068250000842500006B2500006C25000013
:105640008C25000088250000902500009125000091
:105650003A260000BA250000A0250000932500008E
:10566000AC250000B2250000C4250000BC250000C8
:10567000814B984233D0814B984200D0E6E4082019
:1056800024E07F4B984226D00CDC7E4B98422AD0F7
:105690001BDB0433984224D07B4B984200D0D5E4E6
:1056A0000B2013E0794B984211D005DC784B9842DF
:1056B00000D0CBE4052009E0764B984209D0764B28
:1056C000984200D0C2E40E2000E0022000BD03207A
:1056D000FCE70420FAE70620F8E70720F6E70920B0
:1056E000F4E70C20F2E70F20F0E71020EEE711209E
:1056F000ECE71420EAE71520E8E71620E6E7172094
:10570000E4E71820E2E71920E0E71A20DEE71D2091
:10571000DCE77F20DAE78020D8E78120D6E7832006
:10572000D4E78520D2E78620D0E78720CEE78820FF
:10573000CCE78920CAE78A20C8E78B20C6E78D20FE
:10574000C4E78E20C2E78F20C0E79120BEE79420F7
:10575000BCE79520BAE79720B8E79920B6E79B20E9
:10576000B4E79C20B2E79E20B0E79F20AEE7A020E0
:10577000ACE7A120AAE7A220A8E7A320A6E7A520DE
:10578000A4E7A620A2E7A720A0E7AA209EE7AB20D7
:105790009CE7AD209AE7AF2098E7B12096E7B320C9
:1057A00094E7B52092E7B62090E7B7208EE7B820BF
:1057B0008CE7BA208AE7BB2088E7BC2086E7BD20BB
:1057C00084E7BE2082E7BF2080E7C0207EE7C120BB
:1057D0007CE7C2207AE7C32078E7C72076E7C820B5
:1057E00074E7CA2072E7CB2070E7CC206EE7CD20AB
:1057F0006CE7CE206AE7CF2068E7D12066E7D220A9
:1058000064E7D42062E7D52060E7D6205EE7D720A2
:105810005CE7D8205AE7DC2058E7DD2056E7DE2099
:1058200054E7E02052E7E12050E7E2204EE7E42091
:105830004CE7E5204AE7E72048E7EA2046E7EC2086
:1058400044E7EE2042E7EF2040E7F0203EE7F1207A
:105850003CE7F3203AE7F42038E7F52036E7FB2071
:1058600034E7FC2032E7FD2030E7FE202EE7FF2062
:105870002CE701202AE7C046CB250000D8250000F0
:10588000602600003C26000042260000652600003D
:1058900063260000662600006B260000C3070CD4B8
:1058A000064B1B68834208D8054B1B68984204D8F6
:1058B000031F1B68002B00D0180070475C070020F6
:1058C000580700200023012210B50B48990001332E
:1058D0004250802BFAD1094B094C1A608E220021CC
:1058E000D20020000AF0BAFF8D235B016360054AF5
:1058F000054B1A6010BDC046082D00200400002092
:1059000060070020640700205407002010B5044BF6
:10591000044A1A60044B054A1A60FFF7D3FF10BD12
:105920005C0700206007002058070020D00B0020F3
:10593000044B1B681868000980B20238C343DB17A8
:10594000184070475407002000B59BB0020005497D
:1059500001A80BF069FE01A803F0C0F903F0DCFC1C
:10596000FCE7C046DB4301000D4BC2070DD40D4BD5
:1059700000280AD00C4B042807D00C4B05D90F2265
:1059800001680A40042A02D1031D18007047092A41
:1059900003D0032AF9D1064BF7E7064BF5E7C046DB
:1059A000AE430100FC3C0100023D0100BF43010089
:1059B000C8430100B843010000B59BB002000B00D2
:1059C00001A804490BF030FE01A803F087F91BB0D1
:1059D00000BDC046D44301000020064A0649131FFB
:1059E000186013681B099BB202339B00D2188A42CD
:1059F000F5D3704764070020D00B0020F7B50F24C3
:105A00000126314B314A1968314B324D1868136801
:105A10001F002740072F26D813681B099BB20233AB
:105A20009B00D218AA42F2D300242B4EA500AD1938
:105A30002868FFF733FF01342860802CF6D1274C0B
:105A40002068FFF72BFF2060254C2068002802D03B
:105A5000FFF724FF20600025224B1B680093009B6A
:105A60009D4214DBF7BD1B099BB29B00D3189A42E1
:105A7000D2D01F68374208D1B94206D2B84204D307
:105A8000043F3F68002F00D01F60043BEFE7F02386
:105A90006B43154A9B181A78002A01D10135DEE7BD
:105AA0001F693C2300266B43DB199B0001930136E1
:105AB000BB1BF3D4019BB4001C1B0B4B1C19A0692E
:105AC000FFF7ECFEA061F2E75C070020640700200E
:105AD00058070020D00B0020082D002004000020D3
:105AE000D00B0020F8060020B01B0020F7B50124E1
:105AF000204246D1234B1B689C46984241D3224BFF
:105B00001B68019398423CD8031F1B68002B38D1B7
:105B10000200036800941B099BB2002B0FD100996F
:105B2000131F196090422CD015682B1F1B68990019
:105B300069180C68013B14600A602A00EDE79D00BB
:105B400055192968009C214219D18C4517D8019C10
:105B50008C4214D30E1F3468002C10D10F680F3400
:105B60003C40072C08D92F60151F2B600B680A607A
:105B70001B099BB20A00D0E700993160CDE7013BD9
:105B8000CBE7F7BD5C070020580700200D4970B532
:105B90000A000D4D1368141F1B0926689BB2981C40
:105BA000002E0BD000238A4200D00B00236083001C
:105BB000C91880001218AA42ECD370BD1B011360F3
:105BC000F7E7C04664070020D00B0020F8B5124C60
:105BD00027000F223B681D09ADB213420DD06E1C89
:105BE000B600A74204D03200390020000AF023FE9C
:105BF0000022A3190436A4191A600235AD00074B20
:105C00007F199F42E5D31B1B9B10013B1B012360A7
:105C1000034B1C60F8BDC04664070020D00B002079
:105C200054070020F0B59BB003F064FB01F0ECFAE0
:105C3000FEF764FF00240700234AA300D058013474
:105C4000FFF754FF802CF7D1204B1868FFF74EFF69
:105C50001F4B1868002801D0FFF748FF00261D4B96
:105C60001B689E421BDBFFF791FFFFF7C7FEFFF7A4
:105C7000ADFFFEF743FF184BC21B1B6817491B689B
:105C800001A81B099BB2023B0BF0CEFC01A803F05C
:105C900025F803F02FFB01F0B7FA1BB0F0BDF0259B
:105CA00075430F4BED182B78002B01D10136D6E749
:105CB0002B695C1E002CF9DBA300EB189869FFF739
:105CC00015FF013CF6E7C046082D00200400002027
:105CD000D00B0020F8060020540700208E4301005E
:105CE000B01B0020F7B5174D4F1C2B6806001B6832
:105CF0000C001B099BB201929F420BDBFFF792FF46
:105D00002B681B681B099BB29F4203DB0A20FCF730
:105D1000D7F9FEBD2868A71CBA00DB1B81181B0140
:105D20000B6029600021031F19600F231E40030030
:105D30002401264340C3083A9A189A42E9D90199A6
:105D400002C3FAE754070020F7B50300012213400D
:105D500004000D000193002B2BD1174B1B688342CD
:105D600027D8164B1B68834223D90F23144F386062
:105D700000681840FFF7B6FF019B3C68061E3B60B9
:105D800017D0236804301B099BB29D4200DD1D0023
:105D9000AA00211D251F0AF045FDFFF71DFE2E60FC
:105DA000FFF72CFE00232B602268064B1340236074
:105DB00034002000FEBDC0465C07002058070020CC
:105DC000D00B0020F0FF0F000323043010B5C117E3
:105DD00019400918891000220420FFF783FF10BD25
:105DE00070B5050008000C00FFF7EEFF0023002847
:105DF00004D170BDE95CC21811710133A342F9DB13
:105E0000E343DB171C40002304192371F1E7000072
:105E100010B503480AF090FC43000120184310BD60
:105E20006C4501000300002010B5834202DC1C30E9
:105E3000FCF746F910BD10B53620FCF741F910BD4E
:105E400010B500280ADD01240B681C4006D1042B84
:105E500004D90F221B681340042B03D00E20FCF73B
:105E60002FF910BD1B20FCF72BF92000F9E708687B
:105E700010B5C30706D4042804D90F2302681340C1
:105E8000042B03D00E20FCF71BF910BDFFF76CFDAF
:105E90000378233B5A425341C0180378302B05D175
:105EA000202243789343582B00D102301022002146
:105EB0000BF0C8FC430001201843E6E7086870B502
:105EC00001240500254006D1042804D90F230268C7
:105ED0001340042B03D00E20FCF7F2F870BDFFF73F
:105EE00043FD022229000BF0ADFC40002043F5E702
:105EF000F0B5FF2485B00714061227402640029112
:105F0000019203930440B74204DA3D00A74204DD46
:105F1000250002E03500A642FADCB74204DD009716
:105F2000A74204DA009402E00096A642FADB009B46
:105F30009D420FD10023029A28001360019A13603A
:105F40000AF098F92B4B002208F07EFF0AF050FA75
:105F5000039B1860BD4235D10327341B009B581B9F
:105F600008F00CFC051C380008F008FC061C20009A
:105F700008F004FC291C07F0D9FF011C301C08F0B4
:105F800019FA0AF0E3F900221B4B09F067FB1B4BDF
:105F9000002205F09FFF0AF02BFA029B1860009B7D
:105FA000002B1CD10023019A136000980AF062F9BB
:105FB0000022104B08F048FF0AF01AFA039B186001
:105FC00005B0F0BDB54202D1E41B0527C6E7A542E6
:105FD00002D1BC1B0127C1E700273C00BEE70098A7
:105FE00008F0CCFB011C281C07F0A0FF019B1860E7
:105FF000DBE7C04600E06F4000004E400080764086
:1060000010B5002802DD0868C30703D40D20FCF793
:1060100057F810BD4010FEF795FF0020F9E710B5C6
:10602000002802DD0868C30703D40D20FCF748F8F8
:1060300010BD4010FEF787FF0020F9E710B5030000
:10604000C2070BD40A48042B07D90F2219680A404B
:10605000042A02D11800FFF787FC10BD054C43103D
:10606000054A0F2120000BF0ADFA2000F5E7C046ED
:10607000EB430100D40B0020D843010070B50C00A5
:106080009AB0022804DC1C20FCF71AF81AB070BD84
:1060900001230868184206D1042804D90F21026898
:1060A0000A40042A01D00E20EEE762681A4205D1A8
:1060B000042AF8D913680B40042BF4D1A368DB073A
:1060C00001D40D20E0E7FFF74FFC06006068FFF702
:1060D000B5FF0023A568010001AC6D1030002370EE
:1060E00004F0D4FC29006423220004F038FD2000D1
:1060F0000BF0E0FA01002000FFF772FEC6E7000097
:1061000010B51C4CA544041E02D1FFF75DFE0BE048
:1061100004F0C8FB0138062828D807F0DBFB090982
:1061200011182904240000208023DB009D4410BDA9
:10613000200004F03FFC011B2000FFF751FEF3E7B5
:10614000200004F0D9FB430001201843ECE7802233
:106150006946D200200004F0EFFB68460BF0AAFA73
:1061600001006846E9E704210348E6E70020CCE7A0
:106170000420D9E700FCFFFF5445010070B50C0076
:10618000022803DC1C20FBF79BFF70BD012308687D
:10619000184206D1042804D90F2102680A40042AB3
:1061A00001D00E20EFE762681A4205D1042AF8D91F
:1061B00013680B40042BF4D1A368DB0701D40D2036
:1061C000E1E7FFF7D1FB05006068FFF737FFA46840
:1061D00001006410280004F059FC210004F09AFC2E
:1061E000FFF78EFFD1E770B50C00012803DC1C20FF
:1061F000FBF766FF70BD01230868184206D104282A
:1062000004D90F2102680A40042A01D00E20EFE7CA
:1062100062681A4205D1042AF8D913680B40042B8E
:10622000F4D1FFF7A1FB05006068FFF707FF01004D
:10623000280004F02BFC04F0B1FC430001201843BB
:10624000D8E770B505000C001C20012D0BDD0123E3
:106250000868184206D1042804D90F2102680A40B0
:10626000042A03D00E20FBF72BFF70BD62681A4290
:1062700005D1042AF6D913680B40042BF2D1FFF79D
:1062800073FB06006068FFF7D9FE0100022D14D0F1
:10629000A468E30711D56410300004F0F7FB050093
:1062A00004F000FB012811D1002C02DD0135012C86
:1062B00006D12800FFF724FFD7E701246442EBE76B
:1062C000280004F084FB013C0500F0E70228F0D12F
:1062D000002CEEDD0135012CEBD00022280011004E
:1062E00004F0A7FB04F073FB013C0500F3E710B5D5
:1062F000002809DD0868C30706D4042804D90F2341
:1063000002681340042B03D00E20FBF7D9FE10BD0A
:10631000FFF72AFBFBF722FFC043C00F8000F6E720
:1063200010B502F0C5FC431E9841800010BD00006E
:1063300010B50E4C86B020000BF0BCF90100200017
:10634000032909D00A49122201A80AF06BFA01A810
:106350000BF0B0F9010001A8FFF742FD002802D1BF
:106360000A30FBF7ADFE06B010BDC046D8020020D3
:106370005945010010B50124044002D0441020000A
:1063800010BD042810D90F2302681340042B07D135
:10639000FFF7EAFA21000A220BF054FA0400EEE7B4
:1063A000032B01D10430F5E70D20FBF789FEE6E76A
:1063B00070B50868FFF7DEFF1C4907F019FC0C1EDA
:1063C00001DA1A4BCC181A4B01269C4204DD194BFA
:1063D0009C421FDC184B1C1B6421200007F022FB91
:1063E00064210500200007F003FC144A0B0069003B
:1063F000885E002B09D001356D00AA5E64215A43E6
:10640000CB1A5843101807F00DFB012370434000CE
:10641000184370BD0A4B9C4204DC0A4BE418012669
:106420007642D9E7014B1C1BF9E7C046A08C00005F
:10643000272300004F460000504600007045010031
:1064400077690000B0B9FFFF70B50868FFF792FFE9
:10645000C317C4185C40012C03DC012064002043F6
:1064600070BD65102900200007F0DCFA461976108F
:10647000B5420DDC6B1C1A0028005A436843121BFE
:10648000241AA24200DA1D0001206D002843E7E72C
:106490003100200007F0C6FA8019C30F1818350024
:1064A0004610E5E7F7B50C00042803DC1C20FBF7D9
:1064B00007FEFEBD0868FFF75DFF01906068FFF70B
:1064C00059FF0600A068FFF755FF0500E068FFF7D9
:1064D00051FF07002069FFF74DFFAE4201D11F2099
:1064E000E5E7019BC01B9B1B5843A91B07F09AFAC9
:1064F000C71901207F003843DBE70000F0B50D002D
:10650000A1B0022804DC1C20FBF7DAFD21B0F0BDAD
:106510000868FFF72FFF04006868FFF72BFF0600ED
:10652000A868FFF727FF0F2507000F2E02DCF543B1
:10653000ED173540224E4022310068460AF072F9CC
:1065400031004022403110A80AF06CF9F9170522F9
:106550000023380007F0E2FB00231A4AAE0080183F
:1065600059416B46F258002307F0D8FBE7170D049A
:10657000020C2A430B14650CF9032943E00301259F
:10658000FF246D42240624184D4140206946091815
:1065900088590021A4185D4107F0C0FBCE05420ACE
:1065A00032436008EE074B1230436910801859419E
:1065B0002B00220007F06EFB430001201843A5E7E3
:1065C000EC4301003C0500001FB5002804DC1C2042
:1065D000FBF776FD05B000BD0868FFF7CBFE03AB07
:1065E00002AA01A9FFF784FC039809F0AFFE054B4E
:1065F000002209F033F809F007FE43000120184398
:10660000E8E7C04600005940F8B5012803DC1C202B
:10661000FBF756FDF8BD01240868204202D04D6802
:10662000254201D10D20F3E7401009F023FE0600BA
:106630000F00681009F01EFE32003B0005F046FC1A
:106640000022074B09F00AF8064A074B08F0FCFB4A
:1066500005F0E4FB09F0D8FD40002043DAE7C0462E
:106660000094D140182D4454FB21094010B502F08C
:106670001FFB002805D0002318201A00190002F083
:1066800061FA002010BD0000086870B5C30707D587
:10669000FFF770FE05001F2814D80124200070BDEC
:1066A00004280DD90F2203681A40042A08D11B09B7
:1066B0009BB2002B04D0FFF757F9FAF7D5FDE9E7B5
:1066C00001256D42002202210320FFF70BFB041E6F
:1066D00004D10A20FBF7F4FC0400DFE7C3070AD467
:1066E000042808D00F2203681A40032A03D1C022CD
:1066F000D205134303602800FEF782FCFF28CCD8A4
:10670000052250430349231D411818000AF08AF856
:10671000C4E7C0468E3E01001FB5002804DC1C20E3
:10672000FBF7CEFC05B000BD0868FFF723FE03AB06
:1067300002AA01A9FFF7DCFB019807F0FFFF430065
:1067400001201843EEE700001FB5002804DC1C20E0
:10675000FBF7B6FC05B000BD0868FFF70BFE03AB06
:1067600002AA01A9FFF7C4FB029809F0EFFD054B4F
:10677000002208F073FF09F047FD43000120184391
:10678000E8E7C0460000594070B50E00012803DC60
:106790001C20FBF795FC70BD4B68581009F06AFD92
:1067A000040030680D00401009F064FD02000B0089
:1067B0002000290008F048FB0B4A0C4B05F0F6FBC3
:1067C00002000B0000200A4909F0BAF90022094B27
:1067D00008F044FF084B002208F040FF09F014FDC8
:1067E000430001201843D6E76C45D9CC955BC83FE0
:1067F0000000F03F40A5E54000408F40F0B50C00A0
:1068000087B0022804DC1C20FBF75AFC07B0F0BD5F
:106810000868FFF7AFFDB421490007F0E9F90E1E43
:1068200001DA6936FF366068FFF7A4FD642879DD78
:10683000642007F0A3FF564907F078FB051CA06809
:10684000FFF798FD642871DD642007F097FF504939
:1068500007F06CFB3C21041C300007F0E3F80590C6
:10686000300009F007FD00224A4B08F0EDFA06005F
:1068700005980F0009F0FEFC02000B003000390003
:1068800009F05EF909F0B4FD071C201C09F05EFD5B
:1068900000900191281C09F059FD0290039102001B
:1068A0000B0000203C4909F04BF9009A019B08F0CD
:1068B000D5FE09F09DFD291C061C381C07F048FC7C
:1068C00009F044FD02000B000020334909F038F9BB
:1068D000009A019B08F0C2FE09F08AFD051C381CD5
:1068E00009F034FD02000B0000202B4909F028F9C3
:1068F000029A039B08F0B2FE02000B00002026491A
:1069000009F01EF9009A019B08F0A8FE09F070FD3D
:10691000071C0598013804280ED806F0DBFF0B276A
:106920002C313500C343DB17184082E7C343DB1724
:1069300018408AE7271C2C1C1849201C07F008FC6B
:1069400007F0FCFE15490404381C07F001FC07F0B1
:10695000F5FE000204431149301C07F0F9FB07F073
:10696000EDFE20430124400020434FE7231C341C4C
:106970003E1C1F1CE0E7231C2F1C341C1E1CDBE7E5
:10698000231C3C1C371CF9E7371C2E1CD4E7C046DF
:106990000000C84200004E400000F03F00007F436E
:1069A00010B5034B1C220349022001F027FE10BD45
:1069B000744401006C4401000020704710B51E2093
:1069C000FBF77EFB10BD10B51E20FBF779FB10BD59
:1069D0000020704710B51E20FBF772FB10BD10B5EC
:1069E0001E20FBF76DFB10BD10B51E20FBF768FBEA
:1069F00010BD10B51E20FBF763FB10BD10B51E20A7
:106A0000FBF75EFB10BD10B51E20FBF759FB10BD58
:106A100010B51E20FBF754FB10BD10B51E20FBF770
:106A20004FFB10BD10B51E20FBF74AFB10BD10B583
:106A30001E20FBF745FB10BD10B51E20FBF740FBE9
:106A400010BD10B51E20FBF73BFB10BD10B51E207E
:106A5000FBF736FB10BD10B51E20FBF731FB10BD58
:106A600010B51E20FBF72CFB10BD10B51E20FBF748
:106A700027FB10BD10B51E20FBF722FB10BD10B583
:106A80001E20FBF71DFB10BD10B51E20FBF718FBE9
:106A900010BD10B51E20FBF713FB10BD10B51E2056
:106AA000FBF70EFB10BD10B51E20FBF709FB10BD58
:106AB00010B51E20FBF704FB10BD10B51E20FBF720
:106AC000FFFA10BD10B51E20FBF7FAFA10BD10B585
:106AD0001E20FBF7F5FA10BD10B51E20FBF7F0FAEB
:106AE00010BD10B51E20FBF7EBFA10BD10B51E202F
:106AF000FBF7E6FA10BD10B51E20FBF7E1FA10BD5A
:106B000010B5034B22220349082001F077FD10BD88
:106B10005847010068480100002070470120704775
:106B20000120704700207047012070470020704707
:106B300000207047002070470020704710B5034BBD
:106B4000092203490E2001F059FD10BD344A01000D
:106B50007C4A01000020014B18607047000C0020A7
:106B60000120034B1860034B1B6883401843704798
:106B7000040C0020E40B0020F0B5EFF3108101239A
:106B8000194083F31088134AA1261268124D013A66
:106B90009340A022114FD205F600002B17D02C688D
:106BA000945103420BD0C046C046C046C046C046C2
:106BB000C046C046C0462C68D4515B08EDE7D451AE
:106BC000C046C046C046C046C046C046F5E781F351
:106BD0001088F0BD2C000020F40B00200C050000F4
:106BE000074B10B51968FF2909D040430400054838
:106BF00006F018FF0100200006F014FFC0B210BD1F
:106C00002800002001FE000030B585B001AD0C2247
:106C10000849280009F006FE0024285D01210134FE
:106C2000FDF7B0FF0C2CF8D10022034B1A6005B021
:106C300030BDC046C94A0100E80B002030B585B020
:106C400001AD0C220849280009F0ECFD0024285D64
:106C500000210134FDF796FF0C2CF8D10022034BE4
:106C60001A6005B030BDC046C94A0100E80B0020DB
:106C7000F7B56A463B4B01AE1380062393703A4B3F
:106C800033800F23B370FDF739FF384B384DC018F0
:106C90002B68984201D200232B602C68002C41D134
:106CA000375D01213800FDF76DFF01340021380008
:106CB00004F0FCFF032CF3D1002401276B461E5D7A
:106CC00039003000FDF75EFF01343900300004F078
:106CD000EDFF032CF2D1C8200138C046C046C046A3
:106CE000C046C046C046C046C046C046C046C04674
:106CF000C046F1D16B4600211878FDF743FF6B4683
:106D000000215878FDF73EFF6B4600219878FDF78B
:106D100039FFFDF7F3FEFA2300241B01C018286099
:106D20002000FEBDFDF7EAFE2B6800249842F7D351
:106D3000042004F04BFE0600052004F047FE361840
:106D4000062004F043FE0B4B9B1B181A0A4BA04273
:106D500006DB18600023094A2B6013600124DFE77B
:106D60001C60F7E7040500000D0E0000102700006E
:106D7000FC0B002043030000E40B0020040C002067
:106D800010B5002802DD0B68DA0703D40D20FBF7ED
:106D900097F910BD5B10FF2B00DDFF230A2B00DAF3
:106DA0000A23024A00201360F3E7C04628000020AF
:106DB00010B5002804DD0B68002B05D0042B03D090
:106DC0000C20FBF77DF910BD043B5A425341024AA7
:106DD00000201360F7E7C046EC0B002010B5041E3E
:106DE0000CDA1A24084BA400E2581F231A401E3B59
:106DF0009340064A1360064A136010BDFDF7C0FEBB
:106E0000A042EEDDEEE7C046F05A0100F40B002090
:106E1000180500500200086810B5C3070FD54010D0
:106E20001823012A03DD4A68042A00D10833054AE1
:106E30001360FDF7CBFEFFF7D1FF002010BD01204E
:106E40004042EDE72C00002010B500280CDD0A6858
:106E5000131F591E8B4107490B60042A06D0FFF708
:106E6000EDFE0022044B1A60002010BDFFF7CCFE9F
:106E7000FAE7C046F80B0020E40B002010B501240F
:106E8000044002D04410200010BD042810D90F2364
:106E900002681340042B07D1FEF766FD21000A2289
:106EA0000AF0D0FC0400EEE7032B01D10430F5E733
:106EB0000D20FBF705F9E6E710B50868FFF7DEFFE0
:106EC000034B1860034B186803F08EFC002010BDC4
:106ED00030000020000C00200868F8B5C3071AD560
:106EE000FFF7CCFF0300203B5E2B25D80520434352
:106EF00001221D180020114EAB4219D0052110248B
:106F0000F75C3C4200D0801801395200641000291F
:106F1000F7D10133F0E704280ED90F2203681A4095
:106F2000042A09D11B099BB2002B05D00379DAE7AB
:106F3000012340001843F8BD0120FCE7D54A0100B9
:106F400070B508680D00FFF799FF04006868FFF747
:106F500095FF621E0100042A14D8451E042D11D885
:106F600005236B439B18012215009D402B0006480A
:106F700005682B430360054B1B68002B02D02000E3
:106F800003F031FC002070BD000C00200018002030
:106F900070B508680D00FFF771FF04006868FFF71F
:106FA0006DFF621E0100042A13D8451E042D10D85F
:106FB00005236B439B1801229A40074803689343BB
:106FC0000360064B1B68002B03D00022200003F057
:106FD0000AFC002070BDC046000C002000180020F4
:106FE000F0B5050089B008680C00FFF747FF069070
:106FF000022D3ADD6068FFF741FF0190A068FFF7BE
:107000003DFF040000210127080003F0B9FB231D08
:10701000661E0793731C0293079B9E4235D005237F
:1070200073430593019B019D05330493049BAB427D
:107030001ED0042E16D86B1E042B13D80122059BDC
:107040002549013B5B199A409446244A0B68106815
:10705000069A3A4003920DD062461A430A60012212
:1070600000280DD17F000135E0E701240194C9E734
:10707000029ECFE7624693430B600028F2D0039A4A
:107080000299280003F0AFFBECE7019B1E1D042EC4
:107090001AD8012C18D1002505273B0021006B438D
:1070A0009B1999400B000C4A0135116899430B4B11
:1070B00011601B68002B05D0019B0022581D290080
:1070C00003F091FB052DE8D10021080003F07BFBC4
:1070D000002009B0F0BDC046000C002000180020C0
:1070E0003A4BF7B51B680C00002B03D1012040423E
:1070F000FFF774FE012627683E403ED1042F3CD99D
:107100000F233A681340092B37D17B685B1001933A
:10711000019B9E4255DAB300FB189868FFF7AEFE5C
:10712000FF25040000142840FFF75AFD00902012AC
:107130002840FFF755FD0500FF202040FFF750FDD8
:10714000234B1B68002B14D0009B2D021B041D43F6
:10715000204B28431B68202B07D11F3324161C40CB
:107160001D4BA400E55800022843FFF705FD01363A
:10717000CEE7009B2D041B02E9E73800FFF77EFEF7
:10718000FF27050000143840FFF72AFD06002812EB
:107190003840FFF725FD040038002840FFF720FDA8
:1071A0000C4B240436021B6834432043202B06D1A9
:1071B000AD00AD0E084BAD00EB5800021843FFF7D1
:1071C000DBFC0120FAF78AFF0020FEBDF40B002053
:1071D000EC0B00202C000020B04C0100086810B51A
:1071E000C30703D5FFF74AFE054B1860054B1B6824
:1071F000002B03D0024B186803F0F6FA002010BDF4
:10720000000C0020001800209D4B70B51B68002B5F
:107210000DD19C4C2368002B0AD19B4A1268002A8E
:1072200006D19A4B1B68002B01D0FFF721FD70BDE2
:10723000974D2A68002A1BD1944A1268002A10D060
:10724000FFF716FD0028F2D0FFF7DEFC8E4B226818
:1072500019681A6000290BD0002A09D1FFF7EEFC4B
:10726000E5E7894A1268002AF0D1002BEED0EBE75F
:1072700000210D2004F01AFD00210E2004F016FD5F
:1072800000210F2004F012FD2E68012E5DD0022E89
:1072900000D1A2E0002E51D1013631007A4C0420F9
:1072A0002368994304F002FD042123680520194056
:1072B0004B42594104F0FAFC102123680620194082
:1072C0004B42594104F0F2FC802123680901194026
:1072D0004B4259410C2004F0E9FC8021236809024B
:1072E00019404B4259410B2004F0E0FC80212368F7
:1072F000490219404B4259410A2004F0D7FC802131
:107300002368890219404B425941092004F0CEFC00
:1073100080212368C90219404B425941082004F0DA
:10732000C5FC802321681B0319404B4259410720AB
:1073300004F0BCFC31000D2004F0B8FC2B680321E4
:10734000581C06F055FC296071E702214E4C0720BD
:10735000236819404B42594104F0A8FC08202168D9
:1073600001404B42594104F0A1FC80212368C9002F
:1073700019404B425941052004F098FC80212368B4
:10738000490119404B425941062004F08FFC8021ED
:107390002368C90119404B425941042004F086FC7E
:1073A00080212368890319404B4259410A2004F087
:1073B0007DFC802321681B0419404B425941092060
:1073C00004F074FC31000C2004F070FC31000B2040
:1073D00004F06CFC31000E20AEE720212A4C07207F
:1073E000236819404B42594104F060FC4021236856
:1073F000082019404B42594104F058FC8021236871
:10740000092019404B42594104F050FC8021236867
:10741000490019404B4259410A2004F047FC8021A1
:107420002368890019404B4259410B2004F03EFC6F
:1074300080212368890119404B4259410C2004F0F6
:1074400035FC80212368490319404B4259410620ED
:1074500004F02CFC80212368C90319404B42594198
:10746000042004F023FC802321685B0419404B4274
:107470005941052004F01AFC01210F205CE7C046A9
:10748000F80B0020000C0020F00B0020040C002062
:10749000E80B0020012010B54042FFF79FFC0020C0
:1074A000FFF76AFB012004F0E1F910BD10B5034BB2
:1074B0000D220349062001F0A1F810BDB04D0100D6
:1074C000184E010030B501248025054B054AED001A
:1074D0009C505C59002CFCD001600021995030BDBB
:1074E00000E0014004050000F0B5012480260D4BAA
:1074F0000D4DF6005C51002902DC00225A51F0BD0E
:10750000577814783F022743947824042743D4788B
:10751000043224063C439F59002FFCD010C001398F
:10752000E9E7C04600E0014004050000434258413D
:10753000064B40421840B0239B02C018036800204D
:107540001A0E532A01D11B02180A704700C0FEFF11
:1075500043425841074B40421840B0239B02C01899
:10756000A62310B50902DB05090A1943FFF7AAFF94
:1075700010BDC04600C0FEFF8023F0B50222802669
:10758000A12705005B051B6985B001930C4C0D4BD1
:107590000291F600E250FF000393029B9D4204D348
:1075A0000023039AA35005B0F0BDA359002BFCD0D3
:1075B0000323019AE5519A43AD1801F09BFEECE7D5
:1075C00000E001400405000010B5002806D1C020ED
:1075D000B02140028902FFF7CFFF10BDB02080210B
:1075E0008002C902F7E70000134B1B68002B0CD088
:1075F0008022B023D2029B0200280BD11A1D5B68A7
:107600001B0E522B00D110007047B022C0239202F3
:107610005B02F1E782420DD903681B0E522B09D1A0
:10762000436802339B00C018824203D903681B0ED3
:10763000522BE9D00020E7E7080D0020F0B500202C
:10764000B7B00024FFF7D0FF270005002600002D6B
:107650002ED1284D2868FFF769FF32003B000190CA
:107660000094254904A809F0DFFF04A801F036FBC7
:10767000224B64201C682B68A0215A425341204AA7
:107680005B421340B02292029B18E41A6043490205
:1076900006F0C8F9A0225202030000921949220004
:1076A00004A809F0C1FF04A801F018FB37B0F0BD31
:1076B000FF226B6829689C460233FF180B120136C3
:1076C00013409C4200DA1C00FF200A14024003927F
:1076D0006246014001920091039A0B4904A809F007
:1076E000A3FF04A801F0FAFA2800FFF77DFF0500C8
:1076F000ADE7C046080D00204B4F01000C0D0020E7
:1077000000C0FEFFF54E0100374F010070B50020AC
:10771000FFF70CFF04000120FFF708FF844200DAA6
:1077200004000A4D2868434258412860FFF74CFF87
:107730002868611C43424341054A5B421340054AA5
:107740009B18054A1360FFF703FF70BD080D00206A
:1077500000C0FEFF04C002000C0D0020F8B50020A0
:10776000FFF7E4FE07000120FFF7E0FE3E00204D9A
:107770000643204C0DD18021C020C9024002FFF7F2
:10778000FBFE01213000FFF7E3FE1B4B2E60236060
:107790001DE0874209DD0023B0212B60164B8902D2
:1077A000236023680020012517E0012380212B603E
:1077B000124BC9022360F4E7120E522A08D00028A7
:1077C00000D023600E4801F089FAFFF79FFFF8BD53
:1077D00028005A68023292009B188B4205D21A6820
:1077E000561CE9D10028F2D0D1E72160EFE7C0466E
:1077F000080D00200C0D00200480010004C00200D0
:10780000104F010070B50020FFF7EEFEFF260500C7
:10781000002801D1280070BD03681C143440FFF714
:10782000E3FEDA2CF4D10500F2E70000FF2270B588
:107830001F4CD2000021200009F010F8FF25FFF7AF
:10784000E1FF0026002818D1F0210A2219484942F8
:107850000B00962553432D011B185D192D78002D23
:1078600007D0154D154E5D199B191B78DB00E358A9
:107870002B60013A002AEBD170BD03681A142A402C
:107880000C2A0AD11A122A40FF2A03D0D200A118CA
:107890000B71A050FFF7A8FED4E7132AFAD11B12F0
:1078A0002B40FF2BF6D0DB00E2181671E650F1E713
:1078B00010250020B01B00206809000061090000AD
:1078C00010B59AB0FFF74AFFFFF7B0FF00231A0088
:1078D0000A48D900415801334C1EA1415218FF2BD0
:1078E000F7D1074901A809F09FFE01A801F0F6F9B8
:1078F000044801F0F3F91AB010BDC046102500206D
:10790000804F0100944F0100F0B5A1B0FDF700F9E0
:1079100080220590520000215F4808F09FFF8022DE
:10792000002152005D4808F099FF5D4E30684342E7
:107930005841FFF749FE33685A1E9341594A5B424A
:107940001340594A944663440393FFF75BFF051EB7
:1079500033D134683068FFF7E9FD63425C41411C74
:107960002000FFF7F5FD039B3460504C2360FFF7C8
:107970005DFFFAF779FA336824685A425341494A5D
:107980005B421340B02292029B18E41AFDF7C0F844
:10799000059BA021C51A642049026043019106F0AD
:1079A00041F8230000902A00414907A809F03CFE55
:1079B00007A801F093F921B0F0BD01F09BFCFF2175
:1079C0002A6813140B40121211401A000C3A049149
:1079D000072A2FD8304B5C5C002C23D12800FF21D4
:1079E00003681A120A400499914206D1FF221B141F
:1079F00013400C2B1AD0132B1AD0FFF7F5FD0028DB
:107A0000EDD1002C0AD0636822009F1C3900039836
:107A1000FFF76AFD039BBF00DB1903931E4B012197
:107A2000049A99542800FFF7DFFD90E70400E4E78B
:107A30000024E2E71A00153A082AF3D8174A0499F5
:107A4000525C002AEED12F00152B00D01700280021
:107A5000FF2103681A140A40152A15D01D2A00D1E7
:107A60000027FFF7C1FD0028F2D1002F0AD07B6864
:107A70003A009C1C21000398FFF736FD039BA400ED
:107A80001B190393054BCAE7FF221B121340049AEC
:107A90009A42E6D10700E4E7080C0020100D002010
:107AA000080D002000C0FEFF04C002000C0D0020E5
:107AB000CE4E010070B505000C00FFF725FF002D2C
:107AC00012D0002C10D0094B1A68094B1B68594280
:107AD0004B4108495B420B40B02189025B18D31A25
:107AE0002B60A0235B02236070BDC0460C0D0020FC
:107AF000080D002000C0FEFFF0B585B00392032200
:107B00000333DC17294D1440E4182B6802915942C5
:107B10004B418021A410A21D9200254E0092254FBA
:107B200001905B42326800983B40C9025B18121812
:107B3000934214D2FFF7E8FE2B6880215A4253414A
:107B40005B421F40009A3368C9027F189B189F420E
:107B500005D201F04CF80025280005B0F0BD029BCD
:107B6000356819066B461A7BA423DB051343FF22F5
:107B70002F00090C1943019B12041B0413401943E5
:107B80002800FFF79FFC0837281D21003760FFF70A
:107B900099FC002C04D00A9A21003800FFF7A4FCBD
:107BA000009B183BFF183760D6E7C046080D002041
:107BB0000C0D002000C0FEFF70477047002070478A
:107BC000704700000021094B094A5960013151609A
:107BD00059680029FCD00021196101239360022219
:107BE000044B8131FF315A501A607047FC1000403D
:107BF0000010004000E100E00222064B0121DA679C
:107C00000022054B5A61054A11615A69002AFCD0CD
:107C10007047C04604E100E0FC1000400010004046
:107C200070B5084D2B78181E06D0074B1C68002C29
:107C300003D03220FAF744FA70BDFFF7DDFF2C7055
:107C40002000F9E7AC0E0020E00200201FB58023E1
:107C50005B051A6E044901A809F0E6FC082101A899
:107C6000FEF7BEF805B000BD9C4F010070B50400E2
:107C70000D001600FCF74CFF8023012200215B055C
:107C80001B6E6270E270020AA271020CE2711A0AA3
:107C900060716372000EA2721A0C1B0E26702571A1
:107CA000A1702072E272237370BD000070B5224C87
:107CB0002578002D3FD1FAF7AEF8802201211F4B25
:107CC000D2055D6011605A68002AFCD000220720AE
:107CD0001B4B1C4901255A500439585008315A5041
:107CE00019481A4958501A491A485A501A495A50AC
:107CF000A622D2009D50082218495A5004315850EB
:107D00000220174958501749174858501748043946
:107D10005850182016495850C12189005A50053929
:107D2000FF395858921802435A501249124A995032
:107D3000FFF748FF257070BDAC0E0020FC0000402E
:107D4000001000400C050000746962751C050000FD
:107D500024050000200004022C050000140500008A
:107D6000340500003C050000FFFF00002110010069
:107D700054050000110E00200405000013B5094B46
:107D800004000093084B019307280AD8074B1B787F
:107D9000002B01D1FFF78AFF6B46054A1957054BA7
:107DA000D15013BDE2ECF0F4F8FC0004AC0E00205E
:107DB000001000400C05000070B50E4B06001B784B
:107DC000002B01D1FFF772FF00200B4D2C7884426D
:107DD0000ED00A4B202219780323091B1940084BA7
:107DE0004901C918300008F01DFD0120013C2C702C
:107DF00070BDC046AC0E0020AD0E0020100E00205D
:107E0000110E002010B5134B04001B78002B01D17C
:107E1000FFF74CFFFFF7F0FE00200F4A0F49104B11
:107E2000545058600130106058680028FCD0002081
:107E300018610130906018690028FCD0094B0A488D
:107E40001B785B011B185350FFF7D6FEFFF7BAFEF5
:107E500010BDC046AC0E002000100040040500001C
:107E6000FC100040100E0020110E002010B5322032
:107E7000FAF726F910BD0000064B10B51B68002B61
:107E800002D0FFF7F3FF10BD0120034B1B685B001E
:107E90001843F8E7E002002034000020094B10B539
:107EA0001B68002B04D0FFF7E1FF0400200010BD89
:107EB0001C000028FADD0868C307F7D54010FFF75B
:107EC0005DFFF3E7E00200200E4B10B51B680200D7
:107ED000002B02D0FFF7CAFF10BD1800002AFBDDFF
:107EE0000C68E207F8D56410FF2CF5D8064B1B7818
:107EF000002B01D1FFF7DAFE044A054B0020D450D5
:107F0000EAE7C046E0020020AC0E0020001000406E
:107F100024050000104B10B51B680200002B02D096
:107F2000FFF7A4FF10BD1800002AFBDD0C68E20774
:107F3000F8D56410532CF5D8084B1B78002B01D1D1
:107F4000FFF7B4FEFFF758FEA123054ADB00D4502B
:107F5000FFF738FE0020E5E7E0020020AC0E00202D
:107F600000100040064B10B51B68002B02D0FFF735
:107F70007DFF10BD0120034B1B685B001843F8E731
:107F8000E0020020A80E002010B5174A88B014683F
:107F90000300002C03D0FFF769FF08B010BD2000DC
:107FA000002BFADD0A68012113000B40F5D11800FF
:107FB000042AF2D90F24106804401800092CECD1CF
:107FC00054683F2CE9DD98001018806800240842AE
:107FD00001D04010C4B26846C4540133202BF2D102
:107FE000FFF710FF0020D8E7E00200201FB50A4B82
:107FF0001B68002B04D03220FAF762F805B000BDF0
:10800000064B07491A6801A809F00EFB082101A8D0
:10801000FDF7E6FEF2E7C046E0020020B00E0020C9
:108020009C4F0100084B10B51B68002B02D0FFF7D6
:108030001DFF10BD054C200009F03CFB0100200095
:10804000FDF7CEFEF5E7C046E0020020910E0020CD
:10805000124B10B51B68002B02D0FFF707FF10BDB5
:108060000F4B104C1B685A1C0FD00F4C002B0CD020
:108070000E4C012B09D00E4C022B06D00A4C042BBF
:1080800003D00C4C052B00D1084C200009F012FB4A
:1080900001002000FDF7A4FEE1E7C046E002002059
:1080A00038000020A14F0100FF370100AC4F010054
:1080B00006380100A64F010070B51D4B88B01A6844
:1080C000002A06D03220F9F7FBFF0300180008B0A1
:1080D00070BD13000028F9DD012408680440F5D1C3
:1080E00023000428F2D90F2203681A402300042A2F
:1080F000ECD1FDF739FC060009F0DCFA0500122886
:1081000000D912252A0002210D326846FFF7AEFD84
:108110006B465D73A54205DD2300325D6B449A73A7
:108120000134F7E76846FFF76DFE0023CEE7C0464F
:10813000E0020020F0B5264B8BB01A680D00002A33
:1081400006D03220F9F7BCFF030018000BB0F0BDD9
:1081500013000128F9DD0868012104000C40F4D166
:1081600023000428F1D90F2203681A402300042AAF
:10817000EBD16A680A42E8D0FDF7F6FB6E680700AB
:108180007310019309F096FA05000E2800D90E2508
:108190002A000121113202A8FFF768FD6A46127910
:1081A00002AB5A7302AA73129373019B76141B0ECF
:1081B000D67313745574A54205DD3A5D02A96318A0
:1081C0009A740134F7E702A8FFF71CFE0023BCE70E
:1081D000E002002070B5124B88B01B68002B05D060
:1081E000FFF744FE0500280008B070BD1D00002800
:1081F000F9DD0C68E307F6D5684610222900FFF781
:1082000035FD6B466A4666105E7368466312360E2D
:1082100064149373D4731674FFF7F4FDE3E7C04658
:10822000E002002070B5224B88B01A68002A06D000
:108230003220F9F745FF0300180008B070BD1300A5
:108240000028F9DD0D6801262C003440F4D123000C
:10825000042DF1D90F222B681A402300092AEBD1F3
:108260006A683F2AE8DD6846FFF7A6FD230000287C
:10827000E2D06B4619783300A14203DB6B461B5DED
:108280005B003343A200AA1801349360202CF2D182
:10829000092169444A780B7812021A438B781B042F
:1082A0001A43CB781B061343024A13600423C3E727
:1082B000E0020020B00E0020F0B5474B8BB01C68E8
:1082C000002C03D0FFF7D2FD0BB0F0BD434B1B7861
:1082D000002B01D1FFF7EAFC02AE3000FFF76CFD86
:1082E000002801D10020EFE733780B2BFAD97378FF
:1082F000012BF7D1F378012BF4D100231120384F53
:10830000384D3B602B7068443379374A41781360AD
:10831000027809021143827812041143C2781206CE
:108320000A4332490A60002B11D1152169444A7869
:108330000B7812021A438B781B041A43CB781B0666
:1083400013433B60002300220420EA54BCE7012BC6
:1083500019D1152169444A780B7812021A438B7897
:108360001B041A43CB781A211B0613433B600E23D0
:10837000727C6944934200DD13009C42E3D00A5DA5
:108380002A550134F9E7022B03D1727B10331621F1
:10839000EFE7042B0DD1152108226944684608F047
:1083A00041FA0098019903F0A9FC07F02DFF38600D
:1083B000C8E7052BC6D1152108226944684608F094
:1083C00031FA0098019903F099FC07F01DFF38601D
:1083D000727D0A231E21CCE7E0020020AC0E0020B3
:1083E000A80E0020910E002038000020B00E0020C2
:1083F000174B184A5968002903D0002159600131F0
:108400009160196900291FD0002018618023DB00CA
:10841000D3581149012B18D1A923DB00D3585B4253
:108420000B600E490B78032B01D801330B7003202E
:108430000B490B78013303400B700A495B015B1851
:10844000094953500123936070470860FAE7C0461A
:10845000FC1000400010004034000020AD0E002051
:10846000100E0020110E00200405000010B50A4B6C
:108470001B78002B0ED0FFF7BFFBA1230722074C70
:10848000DB00E250FFF79EFB0022054B0620E25086
:10849000FFF774FC10BDC046AC0E00200010004079
:1084A0002405000010B5034B102203490A2000F0F8
:1084B000A5F810BDB44F010034500100044A05492D
:1084C0001368C85401339B059B0D13607047C04669
:1084D000CC120020CC0E002070B5124C124A23683A
:1084E000834202DC0023236018E0115C451C0E006F
:1084F000FA3E012E07D8AB4211DD515D002902D0B2
:1085000028399F2901D82800EAE70100151A565C8E
:108510006E5401318B42FADC181A206070BD117064
:10852000FAE7C046D4160020D412002010B5FCF79C
:10853000E5FA064B1A68824201D900221A601B68CC
:10854000C31A034898428041404210BDC80E002023
:10855000204E000070B50E4C0E4D21682B689942DC
:1085600009DD80220C48D200F9F774FC2368C0189A
:108570008005800D206021682A68914207DA06484C
:10858000F9F768FC2368C0188005800D206070BD75
:10859000D0120020CC120020CC0E002010B5040018
:1085A000064B074A1B6812689B1ADB439B059B0D11
:1085B000A34200DB10BDFFF7CDFFF1E7CC12002096
:1085C000D012002070B5FFF71DF9FF250400002828
:1085D00001D1200070BD03681B142B401D2B00D15E
:1085E0000400FFF701F8F2E707B500211D20009114
:1085F0000B000A00FFF780FA07BD000030B50C251C
:108600006843034C015120184260836030BDC0466E
:10861000082F0020F0B5B5B0050009F04BF801288F
:1086200043D92B785B2B40D101382C1823785D2B54
:108630003BD101353A21280009F024F8061E34D038
:10864000471B002F31DD290000253A0002A809F060
:1086500049F802AB711CDD55641AAC4225DD2200DD
:108660001BA809F03FF8642202AB9B181D55133577
:108670000C277F426F43144BFF183B00E43318680C
:1086800000280FD002A909F00BF8061E0AD13B0002
:10869000EC331C68002C05D0E8373B680193019B44
:1086A0009E4204DB013D002DE2D1002008E020685D
:1086B0001BA908F0F5FF27000834002802D17868CC
:1086C00035B0F0BD0136EAE7082F002010B5E422EE
:1086D0000021134808F0C2F8F9F78EF9FEF7E6FE1C
:1086E000F9F76EFBFCF730FCFEF75AF9FEF708FAD3
:1086F000F7F750FDFFF7D6FE01F01EFB02F032F84F
:1087000002F074F802F0CEFAF9F778FBFEF716FAE9
:10871000F7F754FDF9F718FB01F05AF810BDC04601
:10872000082F0020962210B512010021034808F0FE
:1087300095F80022024B1A6010BDC046B01B002005
:10874000F8060020174BC000C3587F2070B50D00FD
:10875000598914000140052901D0002070BDDA8933
:108760000240292AF9D11A000C20185E0A32013081
:1087700040001018FDF7F8F8037806000120002BE0
:10878000ECD0300008F096FF0023A042E5D1A342D0
:1087900001DB0120E2E7F15CEA5C9142DDD10133CB
:1087A000F5E7C04610250020064B074A1B681268F3
:1087B0009B1ADB439B059B0D0122834200DC0022B8
:1087C00010007047CC120020D0120020F8B5050030
:1087D0000C0016001F1E0ED10320FFF7E5FF002836
:1087E00008D0FA20FFF76AFEE8B2FFF767FEE0B2B2
:1087F000FFF764FEF8BD501DFFF7D6FF0028F9D043
:10880000FB20FFF75BFEE8B2FFF758FEE0B2FFF790
:1088100055FEF0B2FFF752FE3012C0B2FFF74EFE27
:108820003C00E31B9E42E5DD2078FFF747FE013464
:10883000F7E7000070B50024F0250C4B1B68A3423D
:1088400005DCFFF76FFF0020F9F73AFC70BD2B0045
:108850006343074A9B181A78002A05D059780023E9
:1088600011201A00FFF7B2FF0134E6E7F8060020F6
:10887000B01B002013B50024FFF7DCFF230022000B
:1088800021000094DA20FFF737F9FF222100D200FF
:10889000014807F0E3FF13BD10250020F8B50700DD
:1088A0000024F0252B0063430C4A01349E18B74284
:1088B00011D0317800290BD00133D15C0023112075
:1088C0001A00FFF783FF2A000021300007F0C6FFDF
:1088D0000A2CE7D1F8BD024B1C60F9E7B01B002061
:1088E000F8060020F0B5150001222F007B4C174040
:1088F000A54401900291002F11D005AB1A706A10A7
:108900005A70120E1A710522691299706D1402992B
:10891000DD70FFF75BFFCF239B009D44F0BD042D6E
:108920002AD90F2428680440042C32D1022304AA37
:1089300028001371FDF718F8050008F0BBFEC823E6
:1089400002009B00984200DD1A007C1C97420DD16A
:10895000984206D9624804AB03226249C01807F066
:1089600061FF220005AB02990198D2E72700611E42
:10897000695C05ACE155E8E7042D00D0AAE00323CB
:1089800004AA043D13716B425D4105AB557102228F
:10899000E9E7092C00D080E0042205AB1A706A6870
:1089A000511000916946521209789A70009A5970D4
:1089B0001F2A01DD202200926A46127806ACDA7086
:1089C000009BBB4202DC05ABE21ACCE70126BB00F0
:1089D000EB189868064008D1002839D0042837D011
:1089E0000F210368194002290CD101232370431081
:1089F000637042121B0E4014A270E07023710534A4
:108A00000137DDE7042921D102232370FCF7ACFFF5
:108A1000039008F04FFEA31C142809D8607086420A
:108A200001D19C19ECE7039A925D9A550136F6E75D
:108A300014226270039A925D9A550136112EF9D173
:108A40002E23E374237563751634D9E7012907D102
:108A50000323043823704342584160700234CFE747
:108A6000092909D10423237043685A1062705B12EC
:108A7000A370E6700434C3E703290BD105232370E8
:108A80000068020992B2430F92000B40D31A637040
:108A90001B12EDE726700134B2E7032C00D03AE751
:108AA000052205AB01091A7089B2420F89002240E4
:108AB0008A1A11125A709970642A00DD6422042106
:108AC000DA70081F824201DC04324CE7685C5854BB
:108AD0000131F6E7002D00D01DE750E7C4FCFFFF91
:108AE000220300002D38010070B502000024F0219F
:108AF0000D4E0800604380194578954203D001343B
:108B00000A2CF6D170BDF022002107F0A7FE074A1B
:108B10001368013BA34200D11460002329001A000E
:108B20001120FFF753FEEDE7B01B0020F8060020F0
:108B3000002310B501001A001A20FFF747FEFFF7C7
:108B400009FD10BDF8B505000E001F001400501DF2
:108B5000FFF724FD3B00310028002200FFF736FE1E
:108B6000F8BD10B5B2B002236A460400137008F0D5
:108B7000A1FDC72800D9C7200023984207DC421C6A
:108B80006B46FE211420FFF721FE32B010BD69466E
:108B900001335A1EA25CCA54EFE7002310B501004E
:108BA0001A001120FFF712FE10BD07B56B461970B1
:108BB00069465A7013128B701314120ECB700A711F
:108BC0006B46010005221320FFF700FE07BD10B51C
:108BD0000A0001001220FFF785FE10BD10B50C0041
:108BE0000300110014202200FFF7F0FD10BD002348
:108BF00010B51A0019001920FFF7E8FD10BD00009C
:108C0000012370B5FF24084A41185B42884201D312
:108C1000D84370BD06781D0A234073409B009B58C3
:108C200001306B40F2E7C0460851010013B5040063
:108C3000FF2815D00B4BC200D058002810D0436835
:108C400008309900FFF7DCFF01900920FFF7A6FC30
:108C500001AB042221001720FFF7B8FDFFF77AFCD3
:108C600013BDC04610250020F7B50190FFF7AAFC00
:108C700001250400FF276D42002C01D12800FEBD14
:108C8000266833143B40152B0DD121000198083183
:108C900008F006FD002801D135123D402000FEF706
:108CA000A3FC0400E8E71D2BF8D101256D42F5E790
:108CB000002010B5074C236883420AD0FBF71EFF43
:108CC00022680300904200D3831A0020024A9A428D
:108CD000404110BDC80E00203F4B4C0030B5B3B032
:108CE0000500FFF7E5FF002821D002236A4628008F
:108CF000137008F0DFFC0400C72800D9C724002344
:108D0000A34216DB20003230FFF748FC621C6B46A2
:108D1000FF211420FFF75AFDFFF7CAFF002806D0F5
:108D2000084B094A1B6812689B1A9B0507D133B090
:108D300030BD694601335A1EAA5CCA54E0E7FFF70A
:108D400009FCE9E7CC120020D0120020F0B5B9B040
:108D50000500029104920593122803D91B20F9F70C
:108D6000AFF924E00C2200264243134B9B185A68AB
:108D70009C680392039B9E420BDB029B0F4A00936D
:108D8000C8212B0006A808F01DFC06A8FFF7A6FFC7
:108D9000E4E7206800280CD0029908F081FC071E47
:108DA00007D16368059904989847054B1F6039B04F
:108DB000F0BD01360834DDE7082F0020085501001A
:108DC000D00B0020F7B5234B06001B68F021009361
:108DD0000023009A9A4211DC0024F0231A00624317
:108DE000019201991C4A55182F78002F12D0013496
:108DF0000A2CF3D11948FFF771FF2AE00A005A4301
:108E0000154882185078B04202D11278002A20D139
:108E10000133DEE7F0223900280007F01FFD0223AE
:108E20000D4A01996E7053540D4BF200D358AE7039
:108E3000AB600423EB60009B2F616F61A34202DCF7
:108E4000044B01341C60002331001A001020FFF78E
:108E5000BDFCF7BDF8060020B01B002056550100F0
:108E600010250020F8B505000E00FCF7B9FFFF241F
:108E70000D4B18600D4AE3005B429B180C4AD35C13
:108E8000062B01D0032B0BD1E743FFB232002900A0
:108E90003800FFF757FC002802D03800FFF792FF98
:108EA000013C002CE6D1F8BD04000020FC070000C6
:108EB0001025002070B50500FF24084AE3005B423E
:108EC0009B18074AD35CAB4203D1E043C0B2FFF723
:108ED00079FF013C002CF0D170BDC046FC070000BA
:108EE00010250020F7B5FBF709FE574B1A688242A0
:108EF00001D900221A601A685449821A8A420DD98F
:108F0000FF2253491860D3005248CB1A1B181B7814
:108F1000073B022B0CD9013A002AF4D1F7BD0720F8
:108F2000FFF7C8FF4C4B27E00820FFF7C3FF38E0EE
:108F3000FBF7EEFD071E00D101270020FBF7E8FE3E
:108F400001900020FBF7F8FE019B0090434C444D3C
:108F5000002B12D02368002B6ED12B682760002BCA
:108F60006ED0404B01261B78002BD8D10920FFF78B
:108F7000A1FF394B1E703B4B1E70009B002B12D083
:108F80002B68002B0FD123682F60002B1ED0324B93
:108F900001261B78002BC7D10920FFF78BFF2E4B32
:108FA0001E70304B1E702368002B0FD02A4E327873
:108FB000002A0BD19F4200D227602368FB1A312B75
:108FC00004D90720FFF776FF012333702B68002BAD
:108FD0000FD0244E3278002A0BD1BB4200D92F602B
:108FE0002B68FF1A312F04D90820FFF763FF0123F4
:108FF00033702368002B0CD0019B002B09D1164E37
:109000003378002B02D10720FFF754FF00232360A1
:1090100033702B68002B00D180E7009B002B00D021
:109020007CE7104C2378002B02D10820FFF742FF89
:1090300000232B60237071E7009A002AA0D1B5E7C6
:10904000009B002B9FD1AEE7C40E00200F2700002D
:1090500010250020FC070000B80E0020B40E0020F0
:10906000BC0E0020C00E002013B50400FFF7E2FB89
:10907000FEF7A3FD00230093134B1B68002B02D1C6
:109080006846FBF72DFE0021042308000193FDF73D
:1090900061FD01A90120FDF7D7FEFEF7B5F8FFF746
:1090A000E5F9FBF75DFEFBF7E1FEFBF7FBFEFEF7E4
:1090B000F1F9FBF777FD002C04D0FCF703FC034823
:1090C000FFF70CFE13BDC0460018002047550100F5
:1090D00010B5FFF7AFFB0120FFF7C6FFFF24F9F73C
:1090E0001DF8084AE3005B429B18074AD35C043B27
:1090F000012B03D8E043C0B2FFF764FE013C002C13
:10910000EFD110BDFC0700001025002070B50D0048
:109110003235060028000C00FFF746FB002806D178
:10912000FFF7C6FD00280BD02800FFF737FA1B20F9
:10913000330022000021FFF749FB0120F8F7CEFFA2
:1091400070BD000010B5FFF7B3FD002806D1FEF793
:1091500035FD002803D00A48FEF732FD10BDFFF7A9
:1091600043FAFFF787FB0120FFF77EFF054B1B68E3
:10917000002B01D001F036FBFEF7A2FBEEE7C04664
:10918000205501000018002073B501A8FBF7D4FD9D
:10919000254C264E042805D00023254A2360336041
:1091A000136073BD3368002B09D0FBF7B1FC336843
:1091B000C01A204B984202D900221D4B1A6001A808
:1091C000FBF7A6FD2368042826D1002BE9D1184D12
:1091D0002B68002B02D1FBF79BFC30602B6801331E
:1091E0002B60032B12DDC420C8218000FBF762FE38
:1091F000C8211148FBF75EFEC820400002F036FB94
:10920000FFF7A0FFFFF764FF00232B600A2002F0A6
:109210002DFB01232360C4E7002B02D00A2002F0BB
:1092200025FB0023F6E7C046D8160020E0160020F4
:10923000DC160020DC0500009302000010B5FBF7EF
:109240005DFC014B186010BDC80E0020F8B500236E
:109250001800264DDA00AA580133511E8A418018A1
:10926000FF2BF7D1052444430A20FFF797F9FB2091
:10927000FFF724F92720FFF721F90020FFF71EF957
:10928000E0B22412FFF71AF9E0B2FFF717F9184B12
:10929000FA21186804F0C6FB00260700F300E8581E
:1092A00000281CD0436808309900FFF7A9FC04008F
:1092B0000520FFF773F9F0B2FFF700F9E0B2FFF70E
:1092C000FDF82004000EFFF7F9F82002000EFFF76A
:1092D000F5F8200EFFF7F2F8380002F0C7FA013671
:1092E000FF2EDBD1FFF7AAFFF8BDC04610250020F6
:1092F00000000020802110B5054C064B2068C900F5
:10930000091AC018F8F794FD23681818206010BDDA
:10931000D4160020D4120020F0B5A1B0FFF71AF93E
:109320008021B34CB34F2068C900091AC019F8F75F
:109330007FFD2368C0182060002811D0FBF7DEFBFA
:10934000AD4B18603B78FA2B00D063E12368022B09
:1093500008DCFFF7EBF8002802D00120FFF7BCF88B
:1093600021B0F0BD7B78BC78981E242800D933E169
:1093700004F0C4FA250038003F00430048005100C3
:1093800032015C0091009800A400BA00FF000B01BC
:109390003201320132013201320132013201320135
:1093A000320132013B0032013201320132012E0121
:1093B0003201320132013201320132019C00FF2CB4
:1093C0000ED02000FFF790FB00228C4BE100CA502A
:1093D0005B181A712100009213001320FEF78CFB1A
:1093E0000320BBE72000FFF7EDFC2000FFF7A0FB08
:1093F000F6E72000FFF778FBF7E7012CF0D1FFF745
:1094000067FEEDE7FFF716FA0020FFF72DFE7C4818
:10941000FFF764FCE4E763B2002BE1DB794BA200C9
:10942000D25821001520FFF75DFAD9E7FFF7CAF8F7
:10943000FF270400002C02D1FFF700FFD0E72568CA
:109440002B143B40152B04D02000FEF7CDF8040070
:10945000F0E72000083008F02DF906000530FFF78E
:109460009DF8FB20FFF72AF82D121D20FFF726F8A4
:10947000E8B2FFF723F8F0B2FFF720F83012C0B2DD
:10948000FFF71CF825002B1B9E42DDDD287AFFF735
:1094900015F80135F7E7012CA2D1FFF7A5F8FCF785
:1094A00011FA9DE72000FFF7C1FB99E7012C97D146
:1094B0002000FFF73DFBFFF7C9FE91E7FBF75CFBE0
:1094C00007AC0090504A6421504B200008F07AF815
:1094D00002232000237008F0EDF823000200002191
:1094E0001620FFF773F97BE7012C00D078E7200006
:1094F000FFF71EFB464BFA21186804F093FA00268A
:1095000004903E4AF3009B181C68002C28D01B795D
:109510000593636808349F00B81D0393FFF73EF876
:10952000FB20FEF7CBFF20207D1CFEF7C7FFF0B22B
:10953000FEF7C4FFE8B22D12FEF7C0FFE8B2FEF757
:10954000BDFF0598FEF7BAFFE719A7420CD8FFF751
:1095500001F8049B0398584302F088F9FEF7FAFFDC
:109560000136FF2ECDD167E72078FEF7A7FF013443
:10957000EBE7012C00D033E7FFF77CF9FCF7A2F909
:1095800000210800FDF7E6FA2AE7012C02D1FEF7D8
:1095900055F825E7022C0CD108A907A8FEF78AFA8E
:1095A00007AB082200212120FFF710F9FEF7D2FFB8
:1095B00016E7032C07D100210800FDF7CBFA0120A4
:1095C000FFF752FD0CE7C72CF9D1FFF70DF8F6E7CE
:1095D0002000F8F721FC03E71A00C83A052A00D951
:1095E000FEE6002218001100F8F7F6FBDEE7C046A1
:1095F000D4160020D4120020C80E00201025002010
:109600002E550100082D0020405501006B4501003A
:1096100000000020FB2B00D09FE62268042A00DC1B
:1096200097E63E79F878644B360206439E4200DDA9
:1096300093E6331D9A4200DC8BE6FB5CFE2B00D0E8
:109640008BE67878BC78751E1D2800D187E01DD880
:10965000082855D01B287DD0072800D0A1E0632D15
:109660004CDC07AF2A005549380007F0DBF800232F
:1096700038007B55FFF7F8FA00283FDB504B80009D
:10968000C25821001520FFF72DF937E0202818D007
:10969000222833D01E2800D083E0022C7BD0032C5C
:1096A0007CD0012C2AD1002D28DD7B79002B03D022
:1096B0001C00322B00DD322464235C43414B1C60D0
:1096C0001CE02000FFF734FAFF2C14D02000FFF735
:1096D0000BFA7D793C4AB31E009221002A000C202F
:1096E000FEF70AFA394BE200D050411E8841404251
:1096F00005409B181D712000FFF798FA701D2DE69C
:1097000063B2002BFADB7A79022A13D0032A1BD02A
:10971000012AF3D1F979BB79090219433B7AA400F4
:109720001B0419437B7A1B060B435B001343244A3B
:10973000A350E3E7002DE1DDB11E2348FCF750FB09
:109740001F4BA400E050D9E7BB79A4005A1E9341F7
:109750009B00ECE729001948FFF784FBCEE7632D57
:1097600000DD6325002307A99D420FDCEB430022A7
:10977000DB172B40CB181A70152000916B1C2100B1
:10978000FEF7BAF92000FFF7D3F9B7E7FA185279D4
:10979000CA540133E8E7FEF70FFAAFE7FEF70DFA18
:1097A000ACE70300C83B052BA8D8044A2900F8F70A
:1097B00013FBFEF7CFFEA1E7F6030000D91200204D
:1097C000082D002000000020DA12002010250020C3
:1097D00010B5034B002203491020FEF70FFF10BD08
:1097E0006C5501006C550100012070470120024BAF
:1097F0001B685B0018437047F816002010B50B4C2F
:10980000200001F0C9FB200001F06EFB2000084998
:1098100001F09EFB0122074B522120001A6001F04B
:1098200036FC200001F0A2FC10BDC0462818002024
:10983000801A0600E416002070B5002801DC002024
:1098400070BD0C68E307FAD50A4D64102B68002B35
:1098500001D1FFF7D3FF2B68002BF0D0E1B2064C0B
:10986000200001F014FC200001F080FC0028E6D16B
:109870000430E5E7E41600202818002010B51B206E
:10988000F8F71EFC10BD000070B5124C0D002068EA
:10989000002801DB01F05CFF012328685B424010D7
:1098A0002360FBF793F90023984210DB1900206036
:1098B000FBF768F902220849206801F0D5FE002272
:1098C000064B1A60FBF71AF9054B186004231800C1
:1098D00070BDC0464C000020019A0000F816002020
:1098E000F4160020F8B5154C2068002801DB01F0C3
:1098F0002FFF20680021FBF745F901235B4223601D
:1099000000240F4B22001D680920691C1C60FCF715
:10991000E9F9A04210D001266B0033432200094C24
:109920004360AA4208DA5300E35E91005B004118ED
:1099300033438B600132F4E7F8BDC0464C00002091
:10994000F8160020FC16002070B5002812DD0C6807
:10995000E3070FD56410012C0CDD074D2B68002B9D
:1099600001D1FFF74BFF2B68002B03D021000348E8
:1099700001F0EEFA002070BDE41600202818002047
:1099800070B500282CDD01240B68234228D0234128
:10999000174A1360174AA04209D04B68234206D0E9
:1099A0002341022B20D0032B20D0A3421AD0022324
:1099B00013600124104D2C70032811DDC868044089
:1099C0000ED104280CD90F2302681340042B07D1B1
:1099D000FBF7CAFF094907F063FE002800D02C708E
:1099E000002070BD0023E3E70323E1E71460E0E714
:1099F00044000020400000203C0000206F55010082
:109A0000F8B50C4D2B687F2B13DCFBF777F80A4E6B
:109A100007003368C41A094B186802F05DF9012881
:109A200000D164422B6837605A1C2A60044A5B00EC
:109A30009C52F8BDF8160020F41600204C000020BF
:109A4000FC160020F7B50868C30703D40D20F8F70B
:109A500037FBFEBD4010FBF7B9F8051E23DBFBF713
:109A60008FF8A8421FDB02212800FBF78BF801F0DA
:109A7000E3FEFA2406006400280002F02DF9002815
:109A80000CD0FA277F00280002F026F9041E0CD023
:109A900001F0D2FE801BB842F5D904E001F0CCFE03
:109AA000801BA042E8D90020D3E706000023072747
:109AB0000193FA2201219200280001F009FF0028F9
:109AC000F1D0282804DD0123BB40019A1A430192FA
:109AD000013FEED26B460F4F1B79F3550136052E31
:109AE000E4D100212800FBF74DF8012206210920CE
:109AF000FCF7F8F80028D6D00B23012143603B5D2A
:109B0000A2005B0082180B4301349360052CF6D150
:109B10009FE7C046E816002010B51B20F8F7D0FAE2
:109B200010BD10B5012803DC1C20F8F7C9FA10BDE0
:109B300001230A681A4203D04A681B201A42F4D152
:109B40000D20F2E71FB500211020FBF71BF80121C3
:109B50001620FBF717F801211120FBF713F81E4C14
:109B6000200001F01FF91D4B1D491A6809681D4BA3
:109B70001D481B78C9B282420DD8802292040192FE
:109B800001AA1171013B581E83410199029A2000DC
:109B900001F024F91FBD1548824202D88022D20468
:109BA000EDE71348824202D880221205E7E7114808
:109BB000824202D880225205E1E70F48824202D851
:109BC00080229205DBE70D48824202D88022D2052E
:109BD000D5E780221206D2E70818002044000020B2
:109BE000400000203C00002048E8010090D0030025
:109BF00020A1070040420F0080841E0000093D00A4
:109C000070B5002820DD0D68EB071DD4002D1BD09A
:109C1000042D19D00F242B681C40032C14D11A09D1
:109C200092B25B0F92001C40141B2E00FFF78AFFBC
:109C3000731B06489C4205DD317901F0D5F80136E9
:109C4000F070F5E701F0CFF8002070BD0818002093
:109C500070B50468E3070FD564101720FF2C27D8D0
:109C6000FFF770FFE1B2144C200001F0BDF82000B6
:109C700001F0B9F8002070BD002C18D0042C16D0CB
:109C80000F2523681D40032D11D11A0992B25B0FD5
:109C900092001D40551B2600FFF754FF331B06485A
:109CA0009D42E5DD317901F09FF80136F6E70D20A0
:109CB000F8F706FADFE7C0460818002070B5FFF78E
:109CC00041FF064D0021280001F08EF80400280015
:109CD00001F089F801206400204370BD08180020BD
:109CE000A02101220B4BC9005A500B480B49585078
:109CF0000B491A604A68002AFCD000224A60A12160
:109D0000C900585801215960A021C9005A50054B7B
:109D1000C0187047007000406A1000000405000081
:109D2000FC700040FBFDFFFF10B5FFF7D9FF4300BB
:109D30000120184310BD000010B5034B1622034943
:109D40000420FEF75BFC10BD845501003456010071
:109D5000F8B5124F04003B680E001500002B01D12E
:109D6000FFF74CFD3B68002B17D0E1B20C4C2000F4
:109D700001F08DF9F1B2200001F082F8E9B2200083
:109D800001F07EF8200001F0F1F9011E05D0054830
:109D9000FBF712FE0520F8F7A1F9F8BDE416002044
:109DA000281800203757010010B50124036823420A
:109DB00005D04168214202D08268224203D10D20A1
:109DC000F8F77EF910BD5810802801D91520F7E763
:109DD0004910FF2901D91620F2E75210FF2A01D9B4
:109DE0001720EDE7FFF7B4FF0020EBE710B50028E0
:109DF00003DC1C20F8F764F910BD0B68DA0701D406
:109E00000D20F7E75B100322012B06DD0522022B54
:109E100003D00C22042B00DC08220F211820FFF7AE
:109E200097FF0220F8F75AF90020E5E70122F0B584
:109E3000130085B0904217DD0D682A4214D01541F9
:109E40004C680192022805D08B68043B5A4253416A
:109E5000DBB201933B4E3368002B01D1FFF7CEFC00
:109E60003368002B03D10023180005B0F0BD01209A
:109E70004042F8F733F9344EE9B2300001F007F907
:109E800027000122174013D01441FF2C02D91720BC
:109E9000F8F716F9E1B2300000F0F2FF0199300056
:109EA00001F002F90028DED00520F8F717F9DAE70B
:109EB000042CF3D90F2523681D40092D1CD163689C
:109EC00003925B100293029BBB42E7DDBB00E318E9
:109ED0009D68039B1D420BD06D10FF2D02D91720EA
:109EE000F8F7EEF8E9B2300000F0CAFF0137EAE710
:109EF0001720F8F7E5F8F9E7032D0FD127001A0925
:109F000092B25B0F92001D40551B3B1B9D42C5DD6D
:109F10003979300000F0B4FF0137F6E7042DBDD1E8
:109F20002000FBF721FD050007F0C4FB2C00070013
:109F3000631B9F42B2DD2178300000F0A1FF0134A5
:109F4000F6E7C046E41600202818002070B5194D29
:109F500006002B680C00002B01D1FFF74FFC2B688B
:109F6000002B24D0144DF6B23100280001F08FF8F8
:109F7000E1B2280000F084FF0021280001F094F8ED
:109F8000041E04D00520F8F7A9F8604270BD72B62F
:109F900001223100280001F075F862B6280000F0B7
:109FA00060FF0028F2D0280000F060FFEEE7642098
:109FB0004042EBE7E41600202818002010B50124E9
:109FC0000368234202D04168214203D10D20F8F7F3
:109FD00077F810BD5810802801D91520F7E74910EF
:109FE000FF2901D91620F2E7FFF7B0FF4000204318
:109FF000EFE7000070B5284D04002B68002B08D156
:10A0000005211820FFF7A2FF022001F02FFC0123F9
:10A010002B60012C14D105211820FFF797FF7F2812
:10A020002BDC03007F3301DA7F204042C8235B42F0
:10A0300058437F2103F0F6FC052C00D1404270BD4F
:10A04000032C11D121001820FFF780FF7F2814DC9A
:10A0500003007F3301DA7F204042C8235B4258432C
:10A060007F2103F0DFFCEAE70020052CF5D1072172
:10A070001830FFF76BFF7F2802DD0138FF38D0E78B
:10A0800003007F3301DA7F204042C8235B425843FC
:10A090007F2103F0C7FCD1E7F016002010B50120A6
:10A0A000FFF7A8FF43000120184310BD10B503209F
:10A0B000FFF7A0FF43000120184310BD10B5052095
:10A0C000FFF798FF43000120184310BD10B5082189
:10A0D0001820FFF73BFF0300C00FC01801234010FA
:10A0E00015304000184310BDF8B5524B05001B68F1
:10A0F000002B01D1FFF782FB4F4C23787F2B00D838
:10A1000094E007210E20FFF721FFC42835D101225A
:10A110000E264A4B10211A70494B30001A702670D7
:10A12000FFF716FE802211213000FFF711FE0021FB
:10A130006156002920DB434EC9B2300000F0A7FF72
:10A140003E4B3000197800F09BFE300001F00EF815
:10A1500021780622300000F095FFAC1D300000F0A1
:10A1600080FE0023984203D0300000F07FFEC3B28F
:10A170002B700135A542F1D1F8BD0F211920FFF751
:10A18000E5FE33280FD168222C4B1E261A700022C0
:10A190002B4B60211A7030000C322670FFF7D8FD6F
:10A1A00002226121C0E700211820FFF7CFFEFA2824
:10A1B0001CD14222214B10261A700022204B4B2129
:10A1C0001A70300001322670FFF7C2FD042001F042
:10A1D0004DFB38224C213000FFF7BAFD0F225121F0
:10A1E0003000FFF7B5FD1B2252219DE70F211C20F7
:10A1F000FFF7ACFE3D289AD128221C2600270F4BE2
:10A2000020211A700E4B263A30001F702670FFF77F
:10A210009FFD3A0022213000FFF79AFD3A002321EA
:10A220003000FFF795FD402224217DE70021615693
:10A2300081E7C046E4160020480000204A000020C4
:10A24000490000202818002073B5002606220021AE
:10A25000684606F003FB6846FFF746FFFFF75CF829
:10A260001A4B6A469E576C466B4691781878D5789B
:10A270005B7812796479002E1FD000020902034333
:10A2800029431BB209B2120211482243007812B2CC
:10A2900040B2102802D15210DB10C910D8171B1879
:10A2A0004340C8170918414001205918D317D21844
:10A2B0005A408A185200104376BD1B022D020343F8
:10A2C00029431BB209B22402DEE7C0464900002040
:10A2D00048000020F7B5012801DC0120FEBD012562
:10A2E0000B6801932B42F8D04E68354045D1042EBF
:10A2F00043D90F2233681A40092A33D17368009575
:10A300005C10002CE9DD224F3B68002B01D1FFF7E8
:10A3100075FA3B68002BE0D0202C00DD20240120C2
:10A320004042F7F7DBFE72B6019B1A4F5910C9B2D3
:10A330002200380000F0A6FE62B6380000F091FD61
:10A34000FF23002803D0380000F090FDC3B2009A2C
:10A35000002A16D053550135AC42EEDC01206400D2
:10A360002043BBE7032A08D11C09A4B25B0F1340AA
:10A37000A400E41A331D0093C3E72420F7F7A0FEDE
:10A38000ACE70121AA005B00B2180B439360E2E73F
:10A39000E41600202818002070B52F4B86B01B68EB
:10A3A000002B02D10120FFF725FE01AD1422002170
:10A3B000280006F053FA294E1821300000F067FEFD
:10A3C0000321300000F05CFD0021300000F06CFE45
:10A3D000041E2CD001002248FBF7EEFA0520F7F707
:10A3E0007DFE019B7F2B01DD013BFF3BAA687F2A9D
:10A3F00001DD013AFF3A29697F2901DD0139FF3981
:10A40000C820434342434843DB11D2115243C01199
:10A410005B4340439B18181805F02CFF01F080FFA8
:10A4200005F0F2FE43000120184306B070BD72B67D
:10A4300005221821300000F025FE62B6300000F041
:10A4400010FD002802D0300000F010FDA300013400
:10A45000E850052CF2D1C4E7F0160020281800209F
:10A46000735501000020704710B5054C2368002B80
:10A4700002D01B20F7F724FE0020206010BDC0464C
:10A48000FC1700202E4BF7B51B68002B03D12520AD
:10A49000F7F716FE40E0012801DC1C20F8E74B68C6
:10A4A0005D102A00013A019201D51220F0E70C68F4
:10A4B000E2070BD4002C09D0042C07D00F26226809
:10A4C0001640F21E012A03D9092E01D02420DFE70D
:10A4D00001273B4201D11120DAE7FEF70BFF092EDD
:10A4E0001BD129006368019A5B1080319A42DCDA43
:10A4F000AB420BDB0135AA00A2583A42EBD0521016
:10A50000FF2A01D92820C3E78D42F1D11B20F7F79C
:10A51000D7FDFEF7EFFE0120FEBD042E08D120007E
:10A52000FBF722FA07F0C6F8019B8342EEDBBCE79B
:10A530002268100980B252008000920F801AF3E75F
:10A54000FC17002010B50400002C0CDDFEF7D2FE35
:10A550001B20F7F7B5FDFEF7C5FCFEF7DDFE012079
:10A5600001F084F9F0E710BD10B5002803DC1C20D1
:10A57000F7F7A6FD10BD0B68DA0706D4042B04D943
:10A580000F221B681340032B01D02420F0E7054B5A
:10A5900025201B68002BEBD001204042F7F79EFDE1
:10A5A0001B20E5E7FC1700200020704700207047C3
:10A5B000064B10B51B682520002B04D0012040421B
:10A5C000F7F78CFD1B20F7F77BFD10BDFC17002073
:10A5D000084B70B51B6804000D00002B05D11B2033
:10A5E000F7F76EFD052001F041F929002000FFF783
:10A5F00049FF70BDFC17002010B50C00002803DCDB
:10A600001C20F7F75DFD10BD01230A681A4201D135
:10A610000D20F6E702280CDD4868184209D08A6848
:10A620001A4206D04010FAF7D1FAA0684010FAF7A3
:10A63000CDFA1B20F7F744FDFA200138C046C0468A
:10A64000C046C046C046C046C046C046C046C046DA
:10A65000C046C046F1D11B20F7F732FD0020D2E7FB
:10A66000074B10B51B68002B05D11B20F7F728FD01
:10A67000052001F0FBF800210800FFF799FF10BD4D
:10A68000FC17002070B50D00012803DC1C20F7F733
:10A6900017FD70BD01230868184202D04A681A42AB
:10A6A00001D11120F3E74010FAF790FA040068682E
:10A6B0004010FAF78BFA030000208442E9DB834262
:10A6C000E7DB1B30E3E70000F8B5002803DC1C20C3
:10A6D000F7F7F6FCF8BD224B25201B68002BF7D0BE
:10A6E0000D6801202C00044004D00541FF2D1EDD23
:10A6F0002730EDE7042D0ED90F212A6811400429D7
:10A700000BD12800FBF730F906F0D4FF80280ED9D2
:10A710002620F7F7D5FC0020DCE703290AD1100931
:10A7200080B2520F80000A40801A8028F0DCFFF7C8
:10A7300009FFF0E70929EED1040007006B685E10FD
:10A74000A642E8DB0134A300EB583B42F8D05B1093
:10A75000FF2B01DD2820BBE73800FFF7F3FEEFE712
:10A76000FC17002010B5034B0C2203490520FDF710
:10A7700045FF10BD48570100A85701000120704750
:10A78000002070470120404270470120404270473E
:10A790000020704701204042704700207047012090
:10A7A000704700207047002070470020704700204D
:10A7B000704700207047002070470020704700203D
:10A7C000704700207047002070470020704700202D
:10A7D000704700207047002070470020704700201D
:10A7E00070477047704770477047000010B5034BC3
:10A7F000182203490B20FDF701FF10BDFC57010093
:10A80000BC5801000378013B1F2B00D97047013071
:10A81000F8E710B5FFF7F6FF0378002B0BD00130F7
:10A82000222B11D10378002B03D0421C222B03D101
:10A830001000FFF7E7FF10BD5C2B03D14378002B1E
:10A8400000D0821C1000EDE73A2BF2D02C2BF0D078
:10A850007B2B0BD1FFF7D6FF0378002BE9D07D2BA4
:10A8600001D10130E5E7FFF7D4FFF5E720225B2BAC
:10A8700014D1FFF7C7FF0378002BDAD05D2BF0D09F
:10A88000FFF7C7FFF7E7202BD3DD2C2BD3D0190020
:10A8900091435D29CFD0222BCDD001300378002BFE
:10A8A000F1D1C6E7002210B5904216D0FFF7AAFFFB
:10A8B00003780422222B10D0023A7B2B0DD0013AD0
:10A8C0005B2B0AD0190030390232092905D92D2B0A
:10A8D00005D14178303909290AD8100010BD052268
:10A8E000742BFAD00132662BF7D001326E2BF4D0E4
:10A8F000581E83415A42F0E770B5FFF783FF037893
:10A9000001222D2B01D18018023A0023084D0A267E
:10A9100004E0AB420ADC73430130CB1801783039D4
:10A92000CCB2092CF5D95A43100070BD014BFAE79F
:10A9300065666606FFFFFF3FF8B50C001500FFF7E0
:10A9400061FF0378222B02D000232370F8BD0D2372
:10A950006A1E210008250C260A279C460130037830
:10A96000222B01D1002308E0002BFBD0441C5C2BE0
:10A970000FD14378841C002B01D10B70E6E7622BCA
:10A980000ED0662B0ED06E2B0ED0722B0ED0742BE9
:10A990000ED0002AE6DD0B70013A01312000DEE71F
:10A9A0002B00F6E73300F4E73B00F2E76346F0E7FD
:10A9B0000923EEE710B50400FFF72BFFA04203D9EF
:10A9C0000378013B1F2B00D910BD0138F6E710B505
:10A9D000002815D00378002B13D0FFF713FF202198
:10A9E000037802008B4300205D2B09D01000FFF795
:10A9F00010FF03782C3B5A425341C018FFF702FF67
:10AA000010BD1800FCE70300002070B50C00814267
:10AA10000EDD1A785B2A0BD1581CFFF7F3FE0125D7
:10AA2000AC4205D0FFF7D3FF002801D00135F7E78E
:10AA300070BD70B50C001500002901D000230B700B
:10AA4000002820D00378002B1ED0FFF7DBFE037810
:10AA500006002C2B03D10130FFF7D4FE060033781B
:10AA600000207D2B0FD0844204D02A00210030002A
:10AA7000FFF762FF3000FFF7CCFE03783A2B02D1DC
:10AA80000130FFF7BFFE70BD1800FCE7F0B50D0008
:10AA900004009DB02F78002F39D02E21280006F019
:10AAA000F1FD0190461B002803D1280006F002FEAC
:10AAB0000600303F092F0FD82800FFF71DFF0100C7
:10AAC0002000FFF7A0FF0400002C20D0019B002BEA
:10AAD0001DD00136AD19DDE723787B2B16D1601C24
:10AAE000642203A9FFF7A5FF041E10D003A806F0F7
:10AAF000E1FD864206D13200290003A806F0E1FDFF
:10AB00000028E1D02000FFF784FEE9E700242000C0
:10AB10001DB0F0BD70B5050000200C0081421DDDA8
:10AB20002800FFF7BFFE0300681C012B14D0002093
:10AB3000022B13D10022681C1100FFF77AFF012CB1
:10AB40000CD0FFF744FF00221100FFF772FF013C19
:10AB5000F5E7FFF73CFF013C012CFAD170BDF8B5D9
:10AB6000050000200C0016001F0081420DDD2800AA
:10AB7000FFF798FE03000020022B06D1681C3A0064
:10AB80003100FFF756FF012C00D1F8BDFFF71FFF82
:10AB90003A003100FFF74DFF013CF4E710B5002407
:10ABA000A04218D0FFF72EFE03787B2B0AD101308C
:10ABB00000221100FFF73DFF00280CD0FFF729FE0F
:10ABC0000134F5E75B2B06D10130FFF700FF0028C9
:10ABD00001D00134F9E7200010BDF8B5002816DDDA
:10ABE0000D68EB0713D56D10013D0124FCF70AFE3B
:10ABF0000026FF27644200280CD1002E21D030000F
:10AC000006F058FD01003000FBF7EAF8F8BD012519
:10AC10006D42EAE703681A143A40152A0BD11B1259
:10AC20003B409C4200DA1C009D4201D106000836E0
:10AC3000FCF7DAFCDFE71D2AFAD101240026644282
:10AC4000F6E70120013464002043DFE710B508680F
:10AC50000C00FAF789FEFEF707F8002803DB6268AC
:10AC6000024B8000C250002010BDC046082D0020BD
:10AC700010B50868FAF778FEFDF7F6FF0123002803
:10AC800002DB024B8000C358180010BD082D0020C5
:10AC900010B50868FAF768FEFDF7E6FFC043C00F7D
:10ACA000800010BD10B5034B042203490020FDF7BE
:10ACB000A5FC10BDB4590100AD59010010B5FAF75B
:10ACC00025FEFDF703FDFAF74BF90A48FEF706F8F3
:10ACD000FCF7F6FDF7F7A6F8002801D0F7F79AF889
:10ACE000054B1B68002B01D0FEF72CFAFEF7F0F99C
:10ACF00010BDC046035A01000418002010B5F9F732
:10AD0000A3FB10BD70B5002504AC24780573A942DF
:10AD100005D10A4B0A4A25210A4805F0EFFC0160DB
:10AD20000949920052589B0002715B58A40083713C
:10AD30006358856043710223C37170BD1B5A0100C3
:10AD4000905A0100295A0100F05A0100037B002BA0
:10AD500004D14373837303610133037370470000AD
:10AD60001FB50191A02100240068C900D2B244504F
:10AD7000012A10D0A24209D0032A0AD0074A8350E0
:10AD8000074B019AC250012343501FBD02221343B7
:10AD9000F4E70422FBE70622F9E7C0465405000069
:10ADA0002405000010B50400FFF7D0FFA12223689E
:10ADB000A179D20099506179064A200099502179F1
:10ADC00004329950044B19685A689B68FFF7C8FF12
:10ADD00010BDC0460C0500001C1800201FB5FFF771
:10ADE000BFFF05B000BD70470368074A99501A00BD
:10ADF000FC32D1680029FCD0A321C9005858002397
:10AE0000C0B2D3607047C0461C05000007B5802261
:10AE1000074BD2051A6000229A6002321A71112380
:10AE20000E320093034905330348FFF76BFF07BD5C
:10AE30001C1800200030004008180020F8B505005C
:10AE40000E0017000024BC4208D02B68315D1B683F
:10AE500028009847002801D00134F4E72000F8BD0D
:10AE6000704710B51C3000F0D4F910BD10B51C307F
:10AE700000F0C1F910BD10B51C3000F0D3F910BDC1
:10AE800070B5437E0D00002B01D1002070BD253030
:10AE9000FF30040000F0D1F90028F6D1200029008D
:10AEA00000F098F90120F1E7F7B50193FA230025A6
:10AEB00004009B0083600B4B4560083303601C302B
:10AEC0000F00160000F078F920002530FF3000F068
:10AED00073F96B461B79276166756576A576200048
:10AEE000A375FEBDD05A0100012330B5A024C3755F
:10AEF000837D13499B005A58437DC132114DFF3267
:10AF0000E40592009B005B581551CC22C133FF33FE
:10AF10009B001D5104690C4B5204E2500522046948
:10AF2000243BE250837D04699B005A58A123DB0037
:10AF3000E250437D02699B005958044BD15030BD0B
:10AF4000F05A01000C060000240500000C0500006A
:10AF5000A022002310B50469D200A3500A4CA142DC
:10AF60000FD90A4C8C425B4109495B420B40CD2111
:10AF7000C9045B18046907496350052103699950A6
:10AF800010BDCC235B04F5E7A086010090D0030040
:10AF9000000098FD24050000A02300210269DB00C9
:10AFA000D1507047F7B5040000200D000193824294
:10AFB00067D0802316005B009A4200D91E0027004C
:10AFC0001C37380000F012F9B1232269DB00D5509C
:10AFD00080220123216992008B50A27E002A03D196
:10AFE00022691362226913600025731EAB4207D1E8
:10AFF000019B002B04D080220221236992009950EA
:10B00000012223691A622369FC33DA68002A02D11B
:10B010009A6A002AF9D09A6A002A0BD1DA60A3232F
:10B020002269DB00D1583800C9B2013500F0D2F8EE
:10B03000B542DAD3019B2269002B0FD11300FC33F8
:10B040009B6A002B0AD10133A376D3612369FC33B9
:10B05000DA6C002AFCD00022DA640AE00023012125
:10B06000A37651611A002369FC3399680029FCD04A
:10B070009A602369FC339A6A002A01D000229A62FE
:10B08000E8B2FEBD10B50123FFF78CFF10BD8B2386
:10B090009B0010B5C15404002530FF3000F0A6F825
:10B0A0000123637610BD000000238B2270B592004F
:10B0B00043760D00815CB12204000069D20081500A
:10B0C0008022216992008B50226901331362226928
:10B0D000936026002536FF36300000F09AF80028ED
:10B0E00012D0300000F087F81E4B2269D05023693F
:10B0F000FC331A6A002A02D19A6A002AF9D09A6AA5
:10B10000002A01D11A62E4E723690122002D0DD142
:10B110001900FC31896A002908D1DA612369FC33FE
:10B12000DA6C002AFCD00022DA6407E05A61236955
:10B13000FC339A68002AFCD000229A600020236920
:10B14000FC339A6A82420BD098622169064A8B5876
:10B150008B501800022B03D0181F431E9841033058
:10B1600070BDC0461C050000C404000010B50121DC
:10B17000FFF79AFF10BD000010B5132312220249F9
:10B180000248FFF791FE10BD004000402818002043
:10B19000F7B506000D000C008B180193019B671B8F
:10B1A0009C4207D0336821781B68300098470134EF
:10B1B0000028F3D13800FEBD802210B504005200F3
:10B1C000002105F04BFB23000022FC3320005A60D5
:10B1D0009A6010BD020030B5FC3254689568631C5B
:10B1E000DBB29D4201D00155536030BD0023FC30DD
:10B1F0004360836070470200FC32936851688B4261
:10B2000004D0C05C0133DBB2936070470120404240
:10B21000FBE70300FC3358689B68C01A01D5013076
:10B22000FF3070470200FC3293685268934201D0AD
:10B23000C05C704701204042FBE70300FC335A68C2
:10B240009B68501CC0B2C01A43425841C0B27047FC
:10B2500003210A4802680A430260094802680A4357
:10B2600002600849084A094B9B1A03DD043BC85891
:10B27000D050FBDC00F012F8F4F746FF2405004044
:10B280005405004058600100000000208C0200209E
:10B29000FEE7FEE7FEE7FEE7FEE7FEE7014B024AB8
:10B2A0001A607047500000200024F40010B504001C
:10B2B00000F0AAFAE06023682000DB6898470028C5
:10B2C00008DA00F0A1FAE368C01AA3689842F2D342
:10B2D0000120404210BDF7B50E000C0001908D1802
:10B2E000A71BAC4207D00198FFF7E0FF002802DB64
:10B2F00020700134F4E73800FEBD0120704710B51E
:10B3000003681322DB69984710BD7047054B02693B
:10B31000D1500369FC331A6A002AFCD000220120B4
:10B320001A6270471C050000030010B5FF335A7FF6
:10B330001F231A401E3B19009140114AD167C222B7
:10B34000042104699200A150026953600269D3602C
:10B35000A02300220169DB00CA5001230169094AC8
:10B360005B428B500169084A8B5001690C3A8B5043
:10B37000016908328B501430FFF738FF10BDC0460A
:10B3800004E100E00C0500001405000010B51430C5
:10B39000FFF73FFF10BD10B51430FFF743FF10BD9E
:10B3A00010B51430FFF727FF10BD00000200F0B504
:10B3B000FF32D47F0569704BEC50947F6F4B056969
:10B3C000EC502223FF33C55C04696D4B012D00D086
:10B3D0009CE02026FF36875DA226F600A751902428
:10B3E0006400065DA1240769E4003E510469E5504C
:10B3F0009623DB00994200D88AE096231B019942EC
:10B4000000D888E096235B01994200D886E0962315
:10B410009B01994200D883E0E1239B01994200D827
:10B4200080E09623DB01994200D87EE0E123DB0136
:10B43000994200D87BE096231B02994200D878E01D
:10B44000E1231B02994200D875E096235B029942E2
:10B4500000D872E0E1235B02994200D86FE0E1235B
:10B460009B02994200D86CE0464B994200D86AE0B2
:10B47000E123DB02994269D9E124002324038C42B1
:10B480005B4141495B420B40802149055B180469DF
:10B490003E496350A02304210469DB00E1500024ED
:10B4A0000369FC33DC600369FC331C62012304691B
:10B4B00023600469A3600469C120800021501F201B
:10B4C000517F01408B4062303149FF300B501D20CD
:10B4D000105600283CDA0F230340083B2D4C9B08F4
:10B4E0009B001B1903242040A040FC348440DD69EC
:10B4F000A5432C00C025854028002043D8611F2388
:10B50000527F1A401E3B93400B60F0BD00256EE752
:10B510009E23DB02BBE79D231B03B8E71E4BB6E768
:10B520001E4BB4E7EC239B03B1E71D4BAFE71D4B6C
:10B53000ADE71D4BABE71D4BA9E71D4BA7E71D4B27
:10B54000A5E71D4BA3E78023DB04A0E71B4B9EE789
:10B5500084080F4BA400E41803230340FF20C025F8
:10B56000DB009840AD00665986433000C0269E40FF
:10B57000330003436351C2E70C05000014050000CB
:10B580006C05000090D0030000D0BEFE2405000032
:10B5900000E100E000ED00E000B0130000502700E3
:10B5A00000A04E0000F0750000509D0000F0EB0080
:10B5B00000903A0100E0D70100B0AF0300705F07D0
:10B5C000F7B5009308AB1B7800250193FA2304001C
:10B5D0009B0083600D4B45600833036014300F00FF
:10B5E0001600FFF7E9FD2300009AFF3308492761A1
:10B5F00092005E77525820009A77019A9200525832
:10B60000DA772223FF33E554FEBDC0466C5B0100B0
:10B61000F05A0100036910B51A00FC32D268040028
:10B62000002A0AD0A322D20099581430C9B2FFF7D9
:10B63000D1FD00222369FC33DA6010BD10B5024849
:10B64000FFF7E8FF10BDC046601A00201D2307B5B4
:10B6500002220093024901330248FFF7B1FF07BD00
:10B6600000200040601A0020F8B5304F0D00396806
:10B670000600140000291ED110222D4805F0EEF816
:10B680000121042249422B4805F0E8F840222A49CA
:10B69000C120CA67C021294B49005A50800019585F
:10B6A00027480840802109040143C1208000195027
:10B6B0001A6001233B601E2E2ED8032C05D0042CCB
:10B6C0002BD0022C28D1032400E0022400211D4BA2
:10B6D000B600F358174A8856461C20D114485354D4
:10B6E0008A0015501848194E1218A220C00015588B
:10B6F0001B023540F82615507601155824043340B6
:10B7000023432B431350012314581C431450C122CC
:10B710008B400D4992008B50F8BD0124D6E798422A
:10B72000DCD001310429D6D1F6E7C046981B0020B1
:10B73000841B0020941B002004E100E000E100E0F5
:10B74000FFFF00FFF05A010000600040FFE0FCFF37
:10B7500010B51E281AD8104B8000C15800230F4A7C
:10B760009856884213D1FF210020D1540C499A00E9
:10B77000A22450500B49E40052180121105988436B
:10B780009940C2231051074A9B00D15010BD01338C
:10B79000042BE5D1FAE7C046F05A0100941B0020C3
:10B7A000841B00200060004070B5C1260024B60054
:10B7B0000D4BE518AD002B68012B11D1A3400B4AAE
:10B7C00092591A420CD00A4BE356013306D0094B6A
:10B7D000EA18094BD358002B00D0984700232B6060
:10B7E0000134042CE4D170BD40180010006000400A
:10B7F000941B0020009FFFBF841B002010B5002871
:10B8000001D005F077FE10BD0849094A094B10B573
:10B810001B688858FA22190A1B0618439200002355
:10B8200002F07CFA4904C00B084310BD001001402F
:10B83000040500009C1B0020084B0949094A1B68AD
:10B840008858190A1B0610B51843074A002302F04E
:10B8500065FA4904C00B084310BDC0469C1B00207C
:10B86000001001400405000040420F0070B5041EA6
:10B8700009D0FFF7C9FF050000F014F8FFF7C4FF77
:10B88000401BA042F8D370BD0022044B9A60044ACA
:10B8900013680133DBB213607047C046FC100140EF
:10B8A0009C1B00207047704710B500F05FF8FFF751
:10B8B000FAFF0120FFF7DAFFFFF700FAFFF71EFAA1
:10B8C000024B002BFAD000E000BFF7E700000000B9
:10B8D000F8B54C1EA1410125104B114F8000C358F3
:10B8E0004C4238680F499D40160002F011F80A21B9
:10B8F000704302F00DF82C400300220029000A4892
:10B9000000F016F8FA21094C89004443386801F028
:10B91000FFFF0100200001F0FBFFF8BDF05A01001D
:10B920005000002040420F0010050050102700007A
:10B9300030B504680C40944206D1013B002BF8D18D
:10B9400012E0013B002B0FD004680C409442F8D168
:10B95000002405680D40954204D101349C42F8D181
:10B96000002002E0201C00E0181C30BDC420114B58
:10B9700080001A5810491140C02212020A431A507E
:10B98000C0218022490092025A501A608023A322CB
:10B990000021DB05D20099500122F9309A60074B53
:10B9A000FF301950C1200231800019504030195029
:10B9B0001A60704700E100E0FF00FFFF0010014047
:10B9C000014B18607047C0469C000020F7B500236B
:10B9D0001E285AD8384B8000C258042A5BD007D89A
:10B9E000022A54D055D80423012A09D000234CE060
:10B9F000062A54D051D31A2A53D002231B2AF5D138
:10BA00002E4A116808294ED909294FD00A24022646
:10BA1000A02001252A4AC00015502A482A4D07684F
:10BA20001C20BF0007402948019700685759009023
:10BA300027481B0207401F43C02300989B02034076
:10BA4000FF2057515759000207401F43019B1F43D6
:10BA5000009B58016023184007433E43565101257F
:10BA60001C4B156058680028FCD000205860A123AA
:10BA70000125DB00D3585560A025ED0050511BB2C5
:10BA8000A14202D015D2611ACB401800FEBD082396
:10BA9000B6E71023B4E72023B2E74023B0E78023C2
:10BAA000AEE70123ACE708240026B1E70C0001262D
:10BAB000AEE7091B8B40E8E7F05A01009800002030
:10BAC00000700040540000200405000058000020D1
:10BAD000FF00FFFFFC700040F0B51E285BD8364B1E
:10BAE0008000C258354B1E68002E30D1C227344B1F
:10BAF000BF00D859334C03250440C0200002204326
:10BB0000D851C02480206400800018512E4F186046
:10BB10002E4B803CD859FF3CA043D8510437D8590C
:10BB2000A8432043D8510837D8590C35A843844638
:10BB3000072065462843D851A820C0001E50C120C8
:10BB40008026800076021E501C601C4B1C60142551
:10BB500000202B001E4C2E0046433659771C1BD16B
:10BB60004343E250A0230325C132FF329200DB059C
:10BB7000D550184B1A68082A14D114234343E318EC
:10BB80009A6812485132FF32920059601150DA68B7
:10BB9000C1239B00C250F0BD9642E1D00130032882
:10BBA000D9D1F8E7082A02D9083AD140E5E70823B5
:10BBB0009A1A9140E1E7C046F05A0100A01B00200C
:10BBC00000E100E0FF00FFFF0405000000900040DE
:10BBD0005C0000209C0000202149F0B54A6C2148FF
:10BBE000002A14D0A025A12600230124ED05F6008B
:10BBF000C258571C06D0C7187F68002F02D02700F4
:10BC00009740AF5114333C2BF2D100234B64A02357
:10BC10000121DB0500260F009C4614234B43C3186B
:10BC20001A1F1268104C0E4D920014195219526CC2
:10BC3000002A10D01A00143A1268551C09D0103B83
:10BC40001B68FF2B05D03B00934065461A00074B4D
:10BC5000EA50FC34666401310429DED1F0BDC046EF
:10BC6000FC9000405C000020009000400C050000AB
:10BC700000B51E2810D80C4A8000835803290BD821
:10BC8000A0220800C133FF33D2059B0001F022FE41
:10BC9000020905070021D15000BD0C21FBE704215A
:10BCA000F9E70321F7E7C046F05A01001E280AD839
:10BCB000074B8000C25801239340A022D2050029DF
:10BCC00002D1044953507047A121C900FAE7C04688
:10BCD000F05A01000C050000030000201E2B0AD8BA
:10BCE000A021A222C905D2008858034A9B009B5874
:10BCF000D840012318407047F05A0100F0B5C646FD
:10BD000000B5CB0F9846404A4B005B0D9A1882B0A5
:10BD10000D000400132A2FDC002A49DB3B4F17419A
:10BD20003E000E40064323D07F08390029400C43D3
:10BD30000AD03749BD438C4663445C425C41802352
:10BD4000DB021341E4071D434146CE0031492B007D
:10BD50008E192200346875682000290002F058FD11
:10BD6000009001910098019922002B0003F0E8FE59
:10BD700002B004BC9046F0BD332A08DD8023DB000E
:10BD80009A42F5D102000B0002F042FDF0E7224A90
:10BD90009446012263445242DA400242E8D05208FB
:10BDA0000242D1D094438022D2051A411443CBE7FA
:10BDB0004B005B080343DBD00B031B0B1C436342AC
:10BDC000234380244D0C24031B0B23406D042B4381
:10BDD00019004346DA000F4B9B181C685D6802008F
:10BDE0000B002000290002F013FD00900191009843
:10BDF000019922002B0003F0A3FE42464B005B0892
:10BE0000D60733431900B3E701FCFFFFFFFF0F0024
:10BE1000EEFBFFFFA05B0100EDFBFFFFF8B5274A3B
:10BE20004B005B0D9A180C000700132A10DC002A47
:10BE300036DB234B13410B423AD0802424031441B8
:10BE4000002064189C430600250030002900F8BD3E
:10BE5000332A0EDD80230600DB000D009A42F4D168
:10BE600002000B003800210002F0D2FC06000D0099
:10BE7000EBE7144D0600AC46012563446D42DD40FE
:10BE8000AC4663460D000342DFD033239A1A323B9F
:10BE900093401818874200D94C1C63469843D2E758
:10BEA000C90FCC070020531CCDD1074B1C43CAE758
:10BEB00006000D000028C0D1C7E7C04601FCFFFF07
:10BEC000FFFF0F00EDFBFFFF0000F03F10B500F09B
:10BED00087FA10BDF0B54746CE4680B58DB01D003F
:10BEE00006000F00140000F037FB2E4B009001916C
:10BEF0001B785BB2984601333CD022002B00200017
:10BF0000290004F065F9002834D132003B003000EC
:10BF1000390004F05DF9814600282BD1002200236E
:10BF20002000290001F088FE002823D0012302937D
:10BF30001D4B0496059703934B460A93434606947C
:10BF40000795002B1DD0002300221900100002F0DD
:10BF50007BFF434608900991022B14D104F0F2FBB9
:10BF6000212303600A9B0093002B15D1089B099C99
:10BF700000930194009801990DB00CBC904699462D
:10BF8000F0BD0896099702A801F022FC0028E5D030
:10BF90000A9B0093002BE9D004F0D4FB0A9B00938A
:10BFA0000360E3E7A0000020B05B0100F0B5574656
:10BFB0004E46DE464546E0B58FB01D0006000F0038
:10BFC000140000F025FCCE4B009001919A461B789E
:10BFD0005BB2994601333ED022002B00200029009D
:10BFE00004F0F6F88346002835D132003B003000DB
:10BFF000390004F0EDF800220390002800D06FE033
:10C0000000233000390001F017FE00282CD0002258
:10C0100000232000290001F00FFE8346002800D1F4
:10C0200092E004AB9846012342460493B54B53601B
:10C030004346039A1C615D611A629E60DF6042465E
:10C04000002300249361D4614B46002B67D000236A
:10C05000AD4C00930194009801990FB03CBC904600
:10C060009946A246AB46F0BD0098019901F0A6FBA7
:10C070008146002800D19AE000980199002200230F
:10C0800001F0DAFD0028E6D03000390001F096FB1F
:10C090000028E0D02000290001F090FB0028DAD031
:10C0A00004AB9846042342460493964B14615561B1
:10C0B000536000230024136200239361D46153462C
:10C0C0001B789660D7605BB2022B04D0404601F02B
:10C0D0007FFB002829D104F035FB2223036024E0F4
:10C0E00000232000290001F0A7FD0028B3D004ABF5
:10C0F0009846012342460493824B4146536043468F
:10C100005A461A6200229E60DF601C615D617E4BB0
:10C110008A61CB61009201934B46022B9BD0404633
:10C1200001F056FB002800D18AE043461B6A002B31
:10C1300004D004F007FB43461B6A03604346DC69F6
:10C140009B690093019486E72000290001F036FBEB
:10C15000002800D17FE7002200232000290001F001
:10C1600071FD002800D176E704AB984601234246D2
:10C170000493644B536043465A469E60DF601A62E4
:10C180001C615D6153461B785BB2002B5DD00020C3
:10C1900042465E499061D161022B5BD104F0D2FA34
:10C1A0002123036043461B6A002BC7D0C1E7300040
:10C1B000390001F003FB002800D15DE720002900D1
:10C1C00001F0FCFA002800D156E700980199534687
:10C1D0001B7802005BB29B460B0003F0F9FF04AB37
:10C1E0009846002862D1032342460493454B1461CC
:10C1F0005561536010629660D760454B200029005E
:10C20000002203F02BFA5B4604000D00002B27D11F
:10C21000E02241463F4B12068A61CB61300000228A
:10C220000023390001F00EFD00282AD1404601F01C
:10C23000CFFA0028B6D104F085FA22230360B1E7D3
:10C2400004F080FA212303606FE7424600230024B4
:10C250009361D461404601F0BBFA0028A2D19DE76A
:10C26000002241462C4B30008A61CB610022002322
:10C27000390001F0E7FC002835D15B46022BDAD00B
:10C28000D4E720002900FFF739FD22002B0001F040
:10C29000D3FC002805D1E022204B120641468A61DA
:10C2A000CB6153461B785BB29B46E6E701234246CF
:10C2B0000493144B536043464A469E60DF601A6203
:10C2C0001C615D615B46002BBFD00023002219007A
:10C2D000100002F0B9FD43469861D9615B46022B1C
:10C2E00000D15BE7B6E720002900FFF707FD220039
:10C2F0002B0001F0A1FC0028D3D10022034BCDE795
:10C30000A0000020B85B01000000F03F0000F0FF3B
:10C310000000E03FFFFFEF470000F07FFFFFEFC7A7
:10C32000F0B54746CE4680B58DB004000D0000F054
:10C33000D5FF294B06001B780F005BB298460133EE
:10C3400010D022002B002000290003F041FF81467D
:10C35000002807D1002200232000290001F072FCF0
:10C36000002806D1300039000DB00CBC904699462B
:10C37000F0BD01230293194B0694079503934B4696
:10C380000A93434604940595002B15D00023002200
:10C390001900100002F058FD434608900991022B45
:10C3A0000ED104F0CFF9212303600A9B0193002BE7
:10C3B0000CD1089E099FD5E7002300240893099417
:10C3C00002A801F005FA0028EFD1EAE704F0BAF973
:10C3D0000A9B01930360ECE7A0000020BC5B010016
:10C3E000F8B515004746CE465A001C006B4280B592
:10C3F0002B434B4F5208DB0F1343BB421DD84B005E
:10C400005B089846464643420343DB0F8946334365
:10C41000BB4212D8434BE3182B4339D00226A31753
:10C420001E40CB0F1E434346034310D1022E47D07C
:10C43000032E08D13C483D4905E002000B002800CE
:10C44000210002F0E5F90CBC90469946F8BD1300B6
:10C450002B4320D0BA4224D0B8451CD043469A1A68
:10C4600012153C2A2FDC002C30DA3C322EDA002068
:10C470000021012E3ED0022E31D0002EE3D02C4AD6
:10C480002C4B03F05DFB284A2B4B03F059FBDAE7FA
:10C4900000F0FCFFD7E74B462348002B0EDB274973
:10C4A000D1E790452BD0022E0AD0032EC2D0002017
:10C4B0000021012EC7D180210906C4E72049C2E727
:10C4C00019481D49BFE718481C49D2E72A00230034
:10C4D00002F0BAFC01F06EF900F0D8FFC9E7144A87
:10C4E000144B03F02DFB02000B000F48124903F020
:10C4F00027FBA8E7802424060B191900A3E7022EC6
:10C5000006D0032E09D00848012E04D00D499AE721
:10C510000D480E4997E70E4995E70B480D4992E7FC
:10C520000000F07F000010C0182D4454FB2109C00A
:10C53000075C143326A6A13CFB210940FB21F93FEF
:10C54000FB21F9BFFB21E93FD221337F7CD9024097
:10C55000FB21E9BF7CD902C0F0B557464546DE460F
:10C560004E465C006408E0B5250083B092469446D0
:10C57000154322D09B4E4D006D08B5421DDC56423E
:10C580001643994FF60F2643BE4216D8CE0FF60734
:10C5900083460700B146A54220DC06008846A54236
:10C5A00013DB904211D319D14B46DA0F8F4BD200D7
:10C5B0009B181E685B68984607E003F04FF802007E
:10C5C0000B0002F041FC060088463000414603B0F3
:10C5D0003CBC90469946A246AB46F0BD844EB5425F
:10C5E00045DD2E15B346834EB0465E464644019661
:10C5F0007F4EB44200DDA5E0002C00D0BDE05646E1
:10C60000002E00DCE7E07C4EB04601267642B346C1
:10C6100056467600D844B246002EF6DC774EB24637
:10C62000019E564500DA7EE080250903090B6D0363
:10C630000D437249884568DB80241B031B0B640390
:10C640002343424601998E1A6246E91AB81A002E0F
:10C650002DD0674592415242891A19D40A000243EB
:10C660001CD04900C50F4D194700013EECE7002DD5
:10C6700076D15E46002E00DCB0E05F4E0196019E52
:10C68000013E01965E467600B346002EF7DCAFE72A
:10C69000FA0F6D00AD187F00013ED5E74B46D90F6C
:10C6A000524BC9005B181E685B6898468DE767456A
:10C6B0009B415B42C91A01D5380029000B00034396
:10C6C000ECD04B4B1A00994209DCC30F4900C91842
:10C6D00001235B429C464000E0449142F5DD474B1C
:10C6E00098455FDA42469B1A142B67DC02000C0067
:10C6F0004348DA404044194184404B4620000B43F4
:10C70000994610430600C8465FE74346C91A1F29E9
:10C710001EDC10003A4B8C404344D8408A40030052
:10C72000944623438DE75146019E8F1B1F2F32DC19
:10C73000B24606003249BD405144CE40B840354370
:10C74000070076E72615B0462A4EB246D04465E784
:10C7500041462C4B5B1A9A4013000022944670E726
:10C76000EE02B046254E0196019E013E01964646D8
:10C770007600B046002EF7DC3AE7E602B2461F4EDE
:10C78000B04601267642B34656467600D844B246B5
:10C79000002EF6DC42E7019D1A490027491B88401C
:10C7A000050046E7184B194C9C464B4644446144EF
:10C7B000240519430C430600A04606E71F2B05DCA1
:10C7C000D8400F4B4344994008439BE70D4B9B1ABD
:10C7D0001941080096E7084EB0461FE7064E01963D
:10C7E00006E7C046FFFFEF7F0000F07FC85B010057
:10C7F000FFFF0F0001FCFFFFEDFBFFFF02FCFFFF4F
:10C800001E040000E2FBFFFF0000F0FFFF0300003A
:10C81000F0B55746DE464E4645465C006408E0B536
:10C8200098461F00230093B083468A4616001343A0
:10C830000CD07D4B4D00029181466D089D4212DD6A
:10C840007A4B9C465B4665441D4361D10023784C7E
:10C85000009301940098019913B03CBC904699460E
:10C86000A246AB46F0BD9D4250D09C42E8DC6E4BE8
:10C870009C426BD0002304935346002B69DB002AB3
:10C8800010D1694B9C424CD0694B9C4200D1A3E033
:10C890008023DB05984500D1BCE0664B984501D16B
:10C8A00000F0D6FB5846514600F084FF4B460090FE
:10C8B0000191002B07D1002D67D053465C4A9B00A5
:10C8C0009B08934261D05346DB0F013B99464A4691
:10C8D000049B134300D190E0574B9C4200DCBBE02B
:10C8E000564B9C4201DC00F010FC554B9D4201DC94
:10C8F00000F004FC4346002B23DD524A524B10004B
:10C90000190002F0ABFE00900191A3E7002805D0CA
:10C910004E4800F05FFF009001919BE7AC42F7DCCE
:10C92000A5E75A46414BEB18134300D18EE7444B21
:10C930009D4200DC99E3434600960197002B00DB03
:10C9400088E7002300240093019483E7002A91D014
:10C9500076E73F4B9C423CDC394B9C428FDD3D49A6
:10C9600023158C466344142B00DCB2E33421CB1A2C
:10C970003100D94008009840904200D07FE7012361
:10C98000194001335B1A049379E74346002B07DA19
:10C99000009A019B0020264902F056FA009001916E
:10C9A000029B002B00DB55E7204B9C46049B654413
:10C9B0001D4301D100F00EFC049B012B00D049E780
:10C9C000009C019D8021220009066B1800920193B2
:10C9D00040E70223049352E75846514643460090ED
:10C9E0000191002B00DB35E75A46534600201049E1
:10C9F00002F02AFA009001912CE75A465346584615
:10CA0000514603F09DF802000B0002F01DFA009061
:10CA100001911FE75A4653465846514602F01EFE02
:10CA20000090019116E7C0460000F07F000010C0A2
:10CA30000000F03F0000E03F0000E0410000F04354
:10CA4000FFFFEF3F9C7500883CE4377EB45B01003C
:10CA5000FFFF3F4301FCFFFFE44B00229D420ADC45
:10CA6000009801990022E24B02F0F8FD35220D00FA
:10CA7000009001915242DF492B158C466344984641
:10CA80002D03DD4CDD4B2D0B90442C439D420ADDE4
:10CA9000DB4B9D4201DC00F001FC01239C46D94B9D
:10CAA000E0449C466444002200230E920F931092AF
:10CAB000119300220025D04B06920793009801990C
:10CAC000069A079B21000890099103F039F8069A0D
:10CAD000079B0A900B910898099901F099FE0200B2
:10CAE0000B000020C44902F0AFF90A000100130056
:10CAF0000C910D9202000A980B9902F0AFFD0A000A
:10CB000001001300029103920022009201938023FE
:10CB100064109B05234380242403A446002063441F
:10CB2000591904000D0002000B000098019902F051
:10CB300095FD02000B000A980B9903F001F8069A84
:10CB4000079B0A900B912000290002F0F9FF0200D8
:10CB50000B000898099902F0F3FF009A019B02F07C
:10CB60007DFD02000B000A980B9902F0E9FF0C9A78
:10CB70000D9B02F073FD029C039D08900991220019
:10CB80002B002000290002F069FD04000D009E4AE0
:10CB90009E4B02F063FD9E4A9E4B01F039FE22003F
:10CBA0002B0002F05BFD9C4A9C4B01F031FE220001
:10CBB0002B0002F053FD9A4A9A4B01F029FE220005
:10CBC0002B0002F04BFD984A984B01F021FE220009
:10CBD0002B0002F043FD964A964B01F019FE22000D
:10CBE000069007912B002000290002F037FD02007B
:10CBF0000B000698079902F031FD009A019B040092
:10CC00000D000298039901F003FE089A099B02F0B7
:10CC100025FD22002B0001F0FBFD009C019D0A90E8
:10CC20000B9122002B002000290002F017FD0022AA
:10CC3000814B04000D0001F0EBFD0A9A0B9B01F003
:10CC4000E7FD00220B0011001A00069107920A006E
:10CC50000098019902F002FD00220C900D910698B7
:10CC60000799754B02F06CFF22002B0002F068FF61
:10CC700002000B000A980B9902F062FF029A039BD4
:10CC800002F0ECFC069A079B04000D000898099935
:10CC900002F0E4FC02000B002000290001F0B8FDC6
:10CCA00004000D0002000B000C980D9901F0B0FD7E
:10CCB00000221000E022614B12060090019102F068
:10CCC000CDFC0C9A0D9B029003910098019902F003
:10CCD00037FF02000B002000290002F031FF584A04
:10CCE000564B02F0BBFC574A04000D000098019916
:10CCF000554B02F0B3FC02000B002000290001F0AC
:10CD000087FD109A119B01F083FD06900791404624
:10CD100003F0B0FA069A079B04000D0002980399ED
:10CD200001F076FD0E9A0F9B01F072FD22002B00A0
:10CD300001F06EFD002022002B000090019102F016
:10CD4000FFFE0E9A0F9B02F0FBFE029A039B02F07D
:10CD5000F7FE02000B000698079902F0F1FE06901C
:10CD600007914A46049B013B134300D188E100230D
:10CD7000214C0293039400223B0030003900140040
:10CD800002F0DEFE009A019B02F068FC32003B00DC
:10CD9000049005910698079902F060FC02000B00D0
:10CDA0000498059901F034FD3D0006000F0000983D
:10CDB000019922002B000496059702F04FFC020017
:10CDC0000B00300039000092019301F021FD1F4B50
:10CDD00004000D008B460200994200DC55E11C4B1B
:10CDE000CB18034300D0FBE134E0C046FFFF0F0047
:10CDF0000000404301FCFFFF0000F03F8E9803005D
:10CE000079B60B000000F0FFEF4E454A287ECA3F7E
:10CE100065DBC9934A86CD3F01411DA96074D13FAE
:10CE20004D268F515555D53FFFAB6FDBB66DDB3FC0
:10CE3000033333333333E33F0000084009C7EE3F89
:10CE4000FD033ADCF5015B14E02F3EBEFFFF8F408F
:10CE5000000070BF04980599E84AE94B01F0D8FC3E
:10CE6000009A019B06000F002000290002F068FED6
:10CE700002000B003000390000F0F8FEAA4600283E
:10CE800000D0ADE18024DF4A53469446640322007B
:10CE90001B1563441A411300DB495B445A001E0012
:10CEA0001B038C461B0B23431424520DD74D6244A5
:10CEB0001541A21A134199465B46AE43002031004A
:10CEC000002B02DA4B465B42994602000B000098A9
:10CED000019902F035FE4B461B05009001910200BE
:10CEE00098460B000498059901F092FC0D0000246F
:10CEF0000022C74B2000290002F0B0FB009A019BE2
:10CF0000069007912000290002F01AFE02000B0093
:10CF10000498059902F014FEBE4ABF4B02F09EFB36
:10CF2000BE4A06000F00BE4B2000290002F096FB0F
:10CF300002000B003000390001F06AFC04000D0013
:10CF400002000B000698079901F062FC069A079B05
:10CF500006000F0002F0F4FD02000B002000290083
:10CF600002F0EEFD3200009001913B0030003900EC
:10CF700002F074FB04000D00AA4AAB4B02F06EFBFA
:10CF8000AA4AAB4B02F0DCFD22002B0002F066FB4C
:10CF9000A84AA94B01F03CFC22002B0002F05EFBEA
:10CFA000A64AA74B02F0CCFD22002B0002F056FB54
:10CFB000A44AA54B01F02CFC22002B0002F04EFBF2
:10CFC00002000B003000390002F0BAFD04000D0031
:10CFD00002000B003000390002F040FB8023049077
:10CFE00005910022DB052000290002F0A9FD0200C6
:10CFF0000B000498059901F027FF009A019B04009B
:10D000000D003000390002F029FB009A019B01F06D
:10D01000FFFB02000B002000290002F091FD32000E
:10D020003B0002F08DFD02000B000020874902F05A
:10D0300087FD43465B181A15002A00DC3FE1190002
:10D04000029A039B02F00AFB00900191FFF702FC99
:10D050005346002B01DAFFF725FC5846514600F0F5
:10D060003DF900900191FFF7F5FB4346002B00DBF3
:10D0700067E480231B06FB1800960193FFF7EAFB89
:10D080000023734C0293039475E64B005B089A46A9
:10D09000704B9A4500DCF9E06F4B5B441A430AD1B0
:10D0A000009A019B02F04CFD049A059B00F0E8FDFC
:10D0B000002800D1E6E602980399684A684B02F01E
:10D0C000CDFA664A664B02F0C9FA00900191FFF76B
:10D0D000C1FB002A01D0FFF7E5FB1432D31A22006E
:10D0E0001A4111009940A14201D0FFF7CDFB012365
:10D0F0001A40DB189B1A0493FFF7C6FB4346002B2C
:10D1000001DBFFF71EFCFFF7F8FB564B9D42F5DDF8
:10D110004E4B9D4201DDFFF7EDFB00980199002287
:10D120004A4B02F00DFDC0224F4BD20504000D000A
:10D1300002F094FA4D4A029003914D4B20002900D1
:10D1400002F08CFA0022009001914A4B2000290045
:10D1500002F084FA02000B004748484902F0F0FC54
:10D1600022002B0002F07AFA02000B000020444952
:10D1700002F0E6FC2200069007912B002000290017
:10D1800002F06CFA02000B000698079902F066FAAA
:10D190001A4A354B02F062FA02000B00009801991E
:10D1A00002F0CEFC02000B0004000D00029803996F
:10D1B00001F02EFB029A039B00200090019102F0E7
:10D1C000BFFC02000B002000290002F0B9FC069011
:10D1D0000791C6E50098019902000B00FFF711FCCA
:10D1E000284A294B0298039902F038FA254A264B1F
:10D1F00002F034FA00900191FFF72CFBFE822B65C0
:10D200004715973C02FCFFFF01FCFFFFFFFF0F00EB
:10D21000432EE63FEF39FAFE422EE63F396CA80C6A
:10D22000615C20BED0A4BE726937663EF16BD2C588
:10D2300041BDBB3E2CDE25AF6A56113F93BDBE16E5
:10D240006CC1663F3E5555555555C53F0000F03FF2
:10D250000000F0BFFFCB904000346F3F59F3F8C29D
:10D260001F6EA501FEFFEF3F4715F73F44DF5DF856
:10D270000BAE543E0000D03F555555555555D53F42
:10D280000000E03F9C7500883CE4377E00220E4B96
:10D29000904691469A4500DC29E6F3E580220B4B47
:10D2A000D2050E920F930A4A0A4B802510921193D1
:10D2B0000022094BED0206920793FFF7FFFB4A4657
:10D2C00000F08EFABCE6C0460000E03F03B8E23F43
:10D2D00006D0CF43EBFD4C3E0000F83FF8B5474683
:10D2E000CE46674B80B50A000F0019000500394093
:10D2F000994200D19BE004000100002F69DD3F1539
:10D3000000D1B4E05F4B12039C468023120B5B03F9
:10D3100013435B00CA0F67449B184A00F80703D504
:10D32000D20F5B009B188A0079108C460021802068
:10D330001624894680030D189D4202DC29185B1BC8
:10D340008144D50F5B00013C5B1952004008002C62
:10D35000F1D100208046802020250027000609E02A
:10D360008B425CD0D40F5B00013DE31852004008B3
:10D37000002D16D0C4198B42F2DD27180E00002CA8
:10D3800049DB5B1AA242894149425B1A121BD40F46
:10D390005B00013D80443100E31852004008002D3D
:10D3A000E8D113434ED143465B0837494A46884685
:10D3B000494652104244C90702D5802109060B4351
:10D3C00061460F05BD18180029000CBC904699460F
:10D3D000F8BD7B005B0803433900002BF5D0002F1C
:10D3E0003CD1E30A153A6405002BFAD080204003B3
:10D3F00003423FD1002700E00F005B00791C03428D
:10D40000FAD0250020208D40401A2900D71B220089
:10D41000C2401A4376E7FE43F60F8E19B1E79442F5
:10D42000A0D82718002CF6DB1E000023AEE7020070
:10D430003B002800390002F011F92A003B0001F0FE
:10D44000E7F9C2E74346013303D0434601335B08A3
:10D45000ABE7012398460023C144A6E73B00020046
:10D4600002F06EFB02000B0001F0EEFCADE71300D2
:10D470000022BBE70127210020207F42C6E7C046EB
:10D480000000F07F01FCFFFF0000E03FF8B54E46D2
:10D4900057464546DE46A04BE0B54E0080468A46DC
:10D4A000894676089E420CDD9C4B9E4200DDA2E040
:10D4B00000D19DE04B46002B00DCE0E0984B994A00
:10D4C000A1E0994B9E4200DDB3E0984B9E4200DC08
:10D4D000A1E001235B429B464246534640465146EB
:10D4E00002F0BCF802000B0006000F0002F0B6F8D4
:10D4F00004000D008E4A8F4B02F0B0F88E4A8F4B1D
:10D5000001F086F922002B0002F0A8F88C4A8D4B1E
:10D5100001F07EF922002B0002F0A0F88A4A8B4B22
:10D5200001F076F922002B0002F098F8884A894B26
:10D5300001F06EF922002B0002F090F8864A874B2A
:10D5400001F066F932003B0002F088F8844A0600D8
:10D550000F00844B2000290002F080F8824A834BA0
:10D5600002F0EEFA22002B0002F078F8804A814B9C
:10D5700002F0E6FA22002B0002F070F87E4A7F4BA0
:10D5800002F0DEFA22002B0002F068F87C4A7D4BA4
:10D5900002F0D6FA22002B0002F060F802000B0025
:10D5A0003000390001F034F95346424602F056F893
:10D5B0005B46013366D05B46734A744CDB00E4186B
:10D5C000D3181A685B6802F0BBFA4246534602F071
:10D5D000B7FA02000B002068616802F0B1FA03009C
:10D5E00048460A0000280EDA802212068A180AE04D
:10D5F000002800D15EE7424653464046514601F0BE
:10D6000007F903000A00180011003CBC9046994637
:10D61000A246AB46F8BD5E4A5E4B01F0F9F8002227
:10D620005D4B00F023FB002800D152E743465246F1
:10D63000E9E700F0BFF8594B04000D009E422ADCD8
:10D64000574B9E4250DC02000B0001F0E1F8002233
:10D65000514B02F075FA802306000F000022DB0513
:10D660002000290001F0D4F80B000200390030003E
:10D6700001F0EAFB002380468A469B462CE7284BB4
:10D68000484AC0E702000B004046514602F058FAF3
:10D6900003000A00B7E7444B9E421ADC0022434BCA
:10D6A00002F04EFA002206000F00404B2000290035
:10D6B00001F0D4FF0022384B01F0AAF80B00020061
:10D6C0003900300001F0C0FB022380468A469B46A9
:10D6D00002E70B0002003649002001F0B5FB0323EE
:10D6E00080468A469B46F7E600222B4B02F028FA3A
:10D6F000002206000F00284B2000290001F088F8C6
:10D700000B0002003900300001F09EFB012380462F
:10D710008A469B46E0E6C046FFFF0F440000F07FCC
:10D72000182D4454FB21F93FFFFFDB3FFFFF1F3E55
:10D7300011DA22E33AAD903FEB0D76244B7BA93F03
:10D74000513DD0A0660DB13F6E204CC5CD45B73FD1
:10D75000FF8300922449C23F0D5555555555D53F7D
:10D760002F6C6A2C44B4A2BF9AFDDE522DDEAD3F71
:10D770006D9A74AFF2B0B33F711623FEC671BC3F11
:10D78000C4EB98999999C93FF85B0100D85B0100F7
:10D790009C7500883CE4377E0000F03FFFFFF23FBD
:10D7A000FFFFE53FFB21F9BFFF7F03400000F83F8B
:10D7B0000000F0BF49004B0819007047034B4800B8
:10D7C0009C4640086044C00F7047C046000010806F
:10D7D00000207047002001497047C0460000F87FD4
:10D7E0004B0070B55B0D14000A00002B1AD14B00E2
:10D7F0005B08034315D0234B002201F02FFF224B7F
:10D800009C422DDB0A004B005B0D363B1F4DE3189D
:10D81000AB422ADC002B0DDD1D4C1B0522401A43B8
:10D82000110070BD1B4DAB42F0D102000B0000F0A7
:10D83000EFFFF6E71D00353519DA174B02009C4261
:10D8400009DD0B001548164900F032F8134A144B55
:10D8500001F004FFE5E70B001248134900F028F837
:10D86000104A114B01F0FAFEDBE70200E9E7084C31
:10D87000363322401B051343190000220B4B01F0E5
:10D88000EDFECEE700005043B03CFFFFFE07000076
:10D89000FFFF0F80FF07000050C300009C75008849
:10D8A0003CE4377E59F3F8C21F6EA5010000903C9E
:10D8B00030B54A00DB0FDB0752081A43110030BDB8
:10D8C00002B4714649084900095649008E4402BC19
:10D8D0007047C04602B4714649084900095C4900D6
:10D8E0008E4402BC7047C04603B4714649084000EC
:10D8F0004900095E49008E4403BC704703B4714679
:10D90000490840004900095A49008E4403BC704749
:10D91000002243088B4274D303098B425FD3030A6E
:10D920008B4244D3030B8B4228D3030C8B420DD381
:10D93000FF22090212BA030C8B4202D3121209020F
:10D9400065D0030B8B4219D300E0090AC30B8B424D
:10D9500001D3CB03C01A5241830B8B4201D38B03FB
:10D96000C01A5241430B8B4201D34B03C01A5241A0
:10D97000030B8B4201D30B03C01A5241C30A8B42E3
:10D9800001D3CB02C01A5241830A8B4201D38B02CE
:10D99000C01A5241430A8B4201D34B02C01A524172
:10D9A000030A8B4201D30B02C01A5241CDD2C309E4
:10D9B0008B4201D3CB01C01A524183098B4201D360
:10D9C0008B01C01A524143098B4201D34B01C01A4B
:10D9D000524103098B4201D30B01C01A5241C308C3
:10D9E0008B4201D3CB00C01A524183088B4201D332
:10D9F0008B00C01A524143088B4201D34B00C01A1E
:10DA00005241411A00D20146524110467047FFE789
:10DA100001B5002000F0F0F802BDC0460029F7D0A3
:10DA200076E7704703460B437FD4002243088B42BE
:10DA300074D303098B425FD3030A8B4244D3030B95
:10DA40008B4228D3030C8B420DD3FF22090212BA5A
:10DA5000030C8B4202D31212090265D0030B8B42D6
:10DA600019D300E0090AC30B8B4201D3CB03C01AC0
:10DA70005241830B8B4201D38B03C01A5241430B9B
:10DA80008B4201D34B03C01A5241030B8B4201D38B
:10DA90000B03C01A5241C30A8B4201D3CB02C01AF6
:10DAA0005241830A8B4201D38B02C01A5241430A6E
:10DAB0008B4201D34B02C01A5241030A8B4201D35D
:10DAC0000B02C01A5241CDD2C3098B4201D3CB0104
:10DAD000C01A524183098B4201D38B01C01A5241B3
:10DAE00043098B4201D34B01C01A524103098B42B7
:10DAF00001D30B01C01A5241C3088B4201D3CB00A2
:10DB0000C01A524183088B4201D38B00C01A524184
:10DB100043088B4201D34B00C01A5241411A00D234
:10DB200001465241104670475DE0CA0F00D049429D
:10DB3000031000D34042534000229C4603098B420D
:10DB40002DD3030A8B4212D3FC22890112BA030A95
:10DB50008B420CD3890192118B4208D38901921117
:10DB60008B4204D389013AD0921100E08909C3099C
:10DB70008B4201D3CB01C01A524183098B4201D39E
:10DB80008B01C01A524143098B4201D34B01C01A89
:10DB9000524103098B4201D30B01C01A5241C30801
:10DBA0008B4201D3CB00C01A524183088B4201D370
:10DBB0008B00C01A5241D9D243088B4201D34B008B
:10DBC000C01A5241411A00D20146634652415B10CD
:10DBD000104601D34042002B00D5494270476346AE
:10DBE0005B1000D3404201B5002000F005F802BDF3
:10DBF0000029F8D016E770477047C046D0400B1C8C
:10DC00001141203A03D49C461341184363465242C3
:10DC1000934018437047C0468446101C62468C46A9
:10DC2000191C634600E0C0461FB501F0AFFC002898
:10DC300001D40021C8421FBD10B501F007FC4042CD
:10DC4000013010BD10B501F0A1FC002801DB00205F
:10DC500010BD012010BDC04610B501F097FC002892
:10DC600001DD002010BD012010BDC04610B501F03F
:10DC700029FC002801DC002010BD012010BDC04699
:10DC800010B501F01FFC002801DA002010BD0120B2
:10DC900010BDC046002B15D1002A13D1002906DB88
:10DCA00001DC002806D00020C043410802E08021AA
:10DCB0000906002007B4024801A14018029003BDE4
:10DCC00039FFFFFF03B4684601B5029800F012F96E
:10DCD000019B9E4602B00CBC7047C046002B11D180
:10DCE000002A0FD1002900D1002802D00021C94309
:10DCF000081C07B4024802A14018029003BDC046A8
:10DD0000F9FEFFFF03B4684601B5029800F030F851
:10DD1000019B9E4602B00CBC7047C046F0B5CE4693
:10DD2000474615042D0C2E0080B50704140C3F0C3B
:10DD30009946030C7E435D43674363437F19340C6C
:10DD4000E4199C46A54203D980235B029846C4444B
:10DD50004B4643435143250C36046544360C24049A
:10DD6000A4195B19591820000CBC90469946F0BDC7
:10DD7000F0B54F464646D646C0B5040082B00D0009
:10DD8000914698468B422FD82CD04146484602F007
:10DD9000D1FB29000600200002F0CCFB331A9C4680
:10DDA000203B9A4600D576E04B46524693401F00F2
:10DDB0004B46624693401E00AF4228D825D05346BA
:10DDC000A41BBD41002B00DA7BE00022002300925F
:10DDD00001930123524693400193012362469340ED
:10DDE000009318E08242D0D90022002300920193D0
:10DDF0000A9B002B01D01C605D600098019902B065
:10DE00001CBC90469946A246F0BDA342D7D9002239
:10DE10000023009201936346002BE9D0FB0798464C
:10DE2000414672080A437B0866460EE0AB4201D1C8
:10DE3000A2420CD8A41A9D41012024196D41002151
:10DE4000013E24184D41002E06D0AB42EED9013ED2
:10DE500024196D41002EF8D10098019953460019FC
:10DE60006941002B23DB2B005246D3402A00644635
:10DE7000E2401C0053461500002B2DDB26005746C0
:10DE8000BE40330026006746BE403200801A9941EA
:10DE900000900191ACE7624620239B1A4A46DA4083
:10DEA0006146130042468A4017001F4380E76246DE
:10DEB00020239B1A2A0066469A402300F34013430E
:10DEC000D4E76246202300219B1A00220091019290
:10DED0000122DA40019280E72023624626009B1A45
:10DEE000DE402F00B0466646B74046463B0033430F
:10DEF000C8E7C046F0B583B016001F00009001913E
:10DF000002F024FB04000D0002000B003000390079
:10DF1000FFF704FF009A019B121A8B410899200019
:10DF20000A604B60290003B0F0BDC046F8B5574603
:10DF30004E464546DE464402E0B546008846640A41
:10DF4000360EC70F002E63D0FF2E24D08023E400AE
:10DF5000DB041C43002399469B467F3E43464246D2
:10DF60005D02D20F5B006D0A1B0E9046924665D093
:10DF7000FF2B55D080220021ED00D2047F3B1543BA
:10DF8000F61A43464A467B400F2A00D98DE06D4879
:10DF9000920082589746002C54D108239946063B9C
:10DFA000FF269B46DAE70025534602291BD00329AA
:10DFB00000D1BFE0012928D030007F30002820DDCB
:10DFC0006A0704D00F222A40042A00D004352A010F
:10DFD00003D530005C4A80301540FE2803DCAC01DC
:10DFE000640AC2B201E0FF2200246402D205600A82
:10DFF000DB07104318433CBC90469946A246AB460B
:10E00000F8BD0122101A1B287CDD00220024ECE759
:10E01000002C1DD104239946033B00269B469DE717
:10E02000FF3E002D20D1022143464A467B400A4351
:10E030000F2AD8D84548920082589746002D19D10A
:10E040000121F1E70C239946093BFF269B4685E712
:10E05000200002F051FA7626431F9C4000237642AE
:10E06000361A99469B4679E74A4603231A43914656
:10E07000032186E7280002F03FFA431F36189D402F
:10E08000763600217DE780240023E403FF22ACE7FD
:10E0900000258023DB031C4228D01D4226D12B43C0
:10E0A0005C02640A4346FF229FE762016C01A242C0
:10E0B00024D21B210025013E012710006D005200D3
:10E0C000002801DB944201D8121B3D43013900298D
:10E0D000F3D11400621E944125436DE7BA465946B8
:10E0E00025005346022900D061E77CE78023DB034B
:10E0F0001C436402640A3B00FF2276E7121B1A21CC
:10E100000125D9E79E362A00B5402C00C240651E85
:10E11000AC411443620704D00F222240042A00D0ED
:10E120000434620103D4A401640A00225DE70122E1
:10E1300000245AE78024E4032C436402640AFF228B
:10E1400053E7C046185C0100FFFFFFF7585C010071
:10E15000F0B54E4657464546DE46E0B543025B0AFB
:10E16000450083B00F1C99462D0EC60F002D57D0C9
:10E17000FF2D24D08020DB00C004184300238146FB
:10E180009A469B467F3D7C027A00FB0F640A120E82
:10E19000984623D0FF2A4BD0E30080240020E404DB
:10E1A0007F3A1C43AD186B1C47460193534677409A
:10E1B0003A000F2B48D87D499B00CB589F46002B37
:10E1C00000D085E008339A46063B9B467C027A00E5
:10E1D000FB0FFF25640A120E9846DBD1002C00D0FD
:10E1E00090E0524601231A4392460120DBE74C4659
:10E1F00058461700022824D0032800D1CFE000227F
:10E20000002301284DD15802D205400AFF071043D0
:10E21000384303B03CBC90469946A246AB46F0BD9D
:10E22000002B5BD104239A46033B00259B46AAE7BB
:10E23000FF35002C60D1524602231A439246022039
:10E24000B1E7FF220023DEE74B461B0C9C464B4602
:10E250002604360C180461463300220C6446000C78
:10E2600043434E435043544380191A0C12189642AC
:10E2700003D9802149028C4664441B041B0C100402
:10E28000C01883015E1EB341800E1843130C1B1986
:10E290009B0103431C00230179D5012362081C4024
:10E2A0001443019A7F32002A4DDD630704D00F2307
:10E2B0002340042B00D00434230103D53C4B019AA6
:10E2C0001C408032FE2ABCDCA3015B0AD2B29AE772
:10E2D0000C239A46093BFF259B4654E7180002F0A1
:10E2E0000BF94A46431F76259A4000236D4291461A
:10E2F0002D1A9A469B4646E7524603231A439246F6
:10E30000032050E7200002F0F7F8431F2D1A9C402D
:10E31000763D002047E780230027DB03FF2272E7DA
:10E32000424666E74C463200584662E780234A463A
:10E33000DB031A4222D01C4220D123435B025B0A3A
:10E340004746FF225FE701239A1A1B2A21DC23009C
:10E350000199D3409E318C401A0023005C1EA341DA
:10E3600013435A0704D00F221A40042A00D0043362
:10E370005A0111D49B015B0A002244E780234A46DC
:10E38000DB0313435B025B0A3700FF223BE7019587
:10E3900087E70022002336E70122002333E78023AA
:10E3A000DB0323435B025B0AFF222CE7985C01003E
:10E3B000FFFFFFF7F8B54746CE464400C20F80B5D1
:10E3C00047024802400A8446664648007F0A240EF7
:10E3D000F60025009046FB00000EC90FB146FF284D
:10E3E00000D185E001267140261A914257D0002EB7
:10E3F00043DD002800D07FE04946002900D1AAE093
:10E40000013E002E00D0F7E05B1A5A0100D48BE0E9
:10E410009B019C09200002F06FF80538844085427A
:10E4200000DDD3E0451B230020200135EB40451BD8
:10E43000AC40621E94412343072400251C40012266
:10E4400041460A40002C04D00F211940042900D075
:10E450000433590100D480E00135ECB2FF2D00D027
:10E46000A3E0FF2400235B02E405580AD2072043FF
:10E4700010430CBC90469946F8BD002E74D1601C28
:10E48000C0B2012800DCA7E04A469C1A620100D510
:10E49000B6E0002CBED1002200240023E3E7002ECA
:10E4A00000DC85E0002846D0FF2C49D08022484679
:10E4B000D2041043814601221B2E09DC20204C4649
:10E4C000801B84404A462000F240441EA041024383
:10E4D0009B185A0128D50135FF2D00D1A8E0012253
:10E4E000072494491A405B080B4013431C40A6E7DD
:10E4F000002E00D078E775E7FF2C54D080224946E3
:10E50000D2041143894601221B2E09DC20214846F2
:10E51000891B88404A460100F240481E81410A4357
:10E520009B1A5A0100D573E7012241460A40590758
:10E5300000D089E711E04846002858D1FF2C0CD1C3
:10E54000DB08002B00D18CE78020C00303435B0273
:10E550005B0AFF2487E7FF2C25D0DB08FF2DF0D0D6
:10E560005B025B0AECB27EE7002C4DD0FF2818D08E
:10E570008024E404724223431B2A00DDC4E01C0013
:10E580002025D440AA1A93405A1E934123434A4659
:10E590000500D31A884638E7721CF8D0F243FF28EA
:10E5A000EAD10A004B46FF25D7E79B015B0A5AE7F1
:10E5B000002E41D1651CE9B2012945DDFF2D00D1B6
:10E5C0004FE707244B445B081C4038E707225A4BAF
:10E5D0002D1A2340144032E7002C1DD1002B7AD194
:10E5E0004B46002B00D191E00A000025B5E7013E23
:10E5F000002E19D14B446CE7FF2C84D1FF25ACE7EA
:10E600004A468846D41A05E7002BC5D10A00FF28E0
:10E61000C8D005004B46A0E7002B49D14B46002B44
:10E6200077D00A00FF2598E7FF2C00D043E787E763
:10E630000A00FF24002316E7002C15D1002B57D128
:10E64000FF28E6D14B467BE7002C20D1002B57D08A
:10E650004946002953D04B445A0168D50724364A0D
:10E660001C4001251340EAE6FF28EBD08022D204AB
:10E67000764213431B2E53DC2025AD1B1A00AB4002
:10E68000F2405C1EA34113434B44050021E7002BDD
:10E69000D8D04946002900D152E78021C9030F4252
:10E6A00000D14DE76046084200D049E74B4647E7B6
:10E6B0004846FF25002800D14FE78022D2031742A9
:10E6C00004D06046104201D14B46884601224146A3
:10E6D000FF250A4041E7484600281FD01A1A50017A
:10E6E00020D54A460724D31A1C4088460025A6E6B2
:10E6F000741CC9D0F643FF28BCD14B4620E799468D
:10E700004B460025DB082BE7012340E700220023CE
:10E71000A9E680230022DB03FF24A4E600251CE7F2
:10E720000123B1E7002AF1D013000025FCE6002503
:10E73000FAE6C046FFFFFF7DFFFFFFFB41024200FC
:10E74000C30F490A120E00207E2A0DD99D2A0CD82B
:10E75000802000040143952A0ADC9620821AD140C9
:10E760004842002B00D108007047034A9818FBE785
:10E77000963A9140F4E7C046FFFFFF7F70B500284E
:10E780003DD0C317C5185D40C40F280001F0B4FE8A
:10E790009E22121A962A07DCD2B2082833DD0838E6
:10E7A00085406802400A23E0992A0BDD05232900F1
:10E7B0001B1AD94003001B339D402B005D1EAB414B
:10E7C00019430D00052801DD431F9D402B000F4913
:10E7D0000B406E0709D00F263540042D05D00433B9
:10E7E0005D0102D59F220B40121A9B01580AD2B23A
:10E7F0004002D205400AE4071043204370BD0024C4
:10E8000000220020F4E76802400AF1E7FFFFFFFB67
:10E81000F0B54F464646D6460C000903C0B5490A36
:10E82000470F5E0039431F03DB0F9C4665007B0AE0
:10E83000570F1F436D0DE40F760DA146C000B8467B
:10E84000D200AB1B64457BD0002B5FDD002E00D0D7
:10E85000A4E03E00164300D112E15E1E002E00D05F
:10E860009EE1871A4346B84280410125C91A4042B9
:10E87000091A0B0200D431E149024E0A002E00D1E0
:10E880006EE1300001F038FE0300083B1F2B00DD75
:10E8900061E120223900D21A9E40D1409F400E43B0
:10E8A0009D4200DD51E15D1B6B1C1F2B00DD7CE1F7
:10E8B0002021C91A3D0030008F408840DD40791E7C
:10E8C0008F41310007222843D940002507433A40B1
:10E8D000002A09D00F233B40042B05D03B1DBB422F
:10E8E000BF417F42C9191F000B0200D426E26A1CF7
:10E8F000C64B55056D0D9A4200D106E1C44AFF088A
:10E900000A40530752023B43120B8EE0002B00D00B
:10E91000B8E06B1C5B055B0D012B00DC30E1871A56
:10E920004346B842B641CB1A76429E1B330200D50D
:10E930004CE13B003343A1D100220024002570E0CC
:10E94000002B00DCE5E0002E00D183E0AF4EB542A5
:10E9500060D0802636043743B846382B00DC3EE1D1
:10E96000434613431F007A1E97413F188742804158
:10E97000404209180B0200D4B0E0A44B01359D427F
:10E9800000D1C3E0A24A7B080A4001210F401F4387
:10E990005108D30707221F433A4099E79B4EB542DF
:10E9A00038D0802636043743B846382B00DDDCE00B
:10E9B0001F2B00DC30E11E004746203EF740BC46DE
:10E9C000202B04D04026F31A46469E4032431700BF
:10E9D00063467A1E97411F43CCE0002B00D104E22E
:10E9E0004346134300D159E14B07C0081843802325
:10E9F000C9081B03194208D04546ED081D4204D141
:10EA00004346D008590708432900420FC9007F4DEB
:10EA10001143C0004B07CA087C49C00803438D421C
:10EA200068D012036D05120B6D0D00211203180042
:10EA3000130B0A0D12051A43764B2D0513402B4379
:10EA40005B00E4075B08234319001CBC9046994611
:10EA5000A246F0BD3E00164312D05E1E002E00D02E
:10EA600000E187188742804141444042091801254E
:10EA70000B0233D5022585E764463300414610007A
:10EA80001D00C7E7002D00D0DAE00C000443F3D0EE
:10EA90005C1C00D19FE15D4CA64200D12FE1DB431D
:10EAA000382B00DD66E11F2B00DD83E1202405000B
:10EAB000E41A0F00DD40D940A0404346A7405B1A4E
:10EAC000441EA04198462F433843171ABA42924138
:10EAD00043465242991A64463500CAE607223A4034
:10EAE000002A00D0F6E64B07CA084849FF083B4316
:10EAF0008D4296D11900114300D19EE18021090376
:10EB00000A431203120B414D8FE715000022002328
:10EB10008BE7002B00D0C7E06B1C5F057F0D012F3A
:10EB200000DCF1E0394DAB4200D1B9E085180A00B4
:10EB3000854289414244494251180722CF076D0856
:10EB40002F4349083A401D00C2E607223049ED1A1A
:10EB500031403A40BCE63E002838864000279FE618
:10EB6000380001F0C9FC20308EE6434613431F00F5
:10EB70007A1E9741C71BB84280414042091A78E685
:10EB80000E003B0006431343002D61D1002E00D040
:10EB9000F4E0002B00D11BE164463900100039E796
:10EBA0001A4FBB427AD03300FFE630001F3DE840E9
:10EBB000202B03D04021CB1A9E4037437B1E9F4120
:10EBC000072207433A400021002589E7171A4346E8
:10EBD000BA42B641591A76428E1B64464EE61F2B46
:10EBE00000DDADE020264746F61AB740B9461700CB
:10EBF000B246DF404E463E4337005646B240561EB0
:10EC0000B24117434246DA408918AEE6FF070000DA
:10EC1000FFFF7FFFFFFF0F8020264746F61AB74011
:10EC2000B9461700B246DF404E463E4337005646CF
:10EC3000B240561EB24117434246DA40891A99E75C
:10EC40007F4CA6425BD0802424045B42214327E70B
:10EC5000002E0CD1002B00D1CBE06446390010000F
:10EC6000774DD7E6764FBB4218D0330075E6002BC0
:10EC700014D04B07C00818438023C9081B0319424E
:10EC800007D0FC081C4204D17907D0080843E146AC
:10EC900021004C46420FC9001143C000684DB9E63F
:10ECA0001D0000220023C0E6002D5BD10D000543AE
:10ECB00000D1E2E65D1C00D1B0E0614DAE421FD054
:10ECC000DB43382B71DC1F2B00DD96E020250F0085
:10ECD000ED1AAF40B9460700AA46DF404D463D4316
:10ECE0002F005546A840D940451EA84188440743F7
:10ECF000BF18974292415142414435003AE664467A
:10ED000035004146100085E60B000343002D00D07E
:10ED100063E6002BF5D04346134300D17AE687180B
:10ED20008742804107224144404209183A400B0281
:10ED300000D4D5E6434B01351940C9E5380069E6F2
:10ED40001E004746203EF740BC46202B04D04026FC
:10ED5000F31A46469E403243170063467A1E974197
:10ED60001F4302E6364DAE42CAD080252D045B42D9
:10ED70002943A6E70843411E8841A6E6002B00D19F
:10ED800048E6871A4346B842B641CB1A76429E1BE4
:10ED900033024BD5171A4346BA429241591A52428E
:10EDA000891A072264463A4092E501430F00791E12
:10EDB0008F419DE71C000F00203CE740202B03D033
:10EDC0004024E31A99400843411E884138437CE6B9
:10EDD0000022002425E6171A4346BA429241591AE6
:10EDE0005242891A6446350043E541461000144DED
:10EDF00010E680220024120380E61D000F00203D53
:10EE0000EF40BC46202B03D04025EB1A9940084325
:10EE100007006346781E87411F4369E787189742BA
:10EE20009B4141445B42C9183500A3E53B00334395
:10EE3000CED0072231003A4052E600231A00F4E512
:10EE4000FF070000FFFF7FFFF0B55746DE464E4646
:10EE50004546E0B5834607000E03480085B092465C
:10EE60001C00360B400DCD0F002800D19DE0954BC6
:10EE7000984239D08023F6001B041E43924A7B0F30
:10EE800033439946944603006344009300230026CD
:10EE9000FF00029323031B0B98466300E40F5246C6
:10EEA0005B0D019400D1B3E086498B4200D19EE016
:10EEB0004246D100802212040A435146490F1143B1
:10EEC0008B46814952468C4600996344CB1A0021F7
:10EED000D20000932B0063409A460F2E00D905E123
:10EEE0007A4BB6009B599F465B463343994600D008
:10EEF000B8E002230826002700900293CAE7CB4619
:10EF00003A0002990195019B9A46022927D00329CC
:10EF100000D180E2012944D06D49009B8C466344B6
:10EF20001C00002C38DD530700D013E2D2085B46EA
:10EF3000DB0109D55946674B19408B468021C90032
:10EF40008C46009B63441C00634B9C4207DC5B4681
:10EF500064055F075B0217431B0B620D02E0002391
:10EF60000027584A00211B031C0B0B0D1B052343D4
:10EF700014055A4A380013401C4353466400DB070B
:10EF800064081C43210005B03CBC90469946A2464B
:10EF9000AB46F0BD0122524201231B1B382B00DC83
:10EFA000ADE1002200230027DCE75B4633439946AE
:10EFB0005ED0002E00D18AE1300001F09DFA0300FE
:10EFC0000B3B1C2B00DD7BE11D22D31A5A460100AE
:10EFD000DA4008398E4013005F46334399468F402C
:10EFE0003F4B00261B1A00930023029352E7414631
:10EFF00053460B433B499B468C46009B634400931E
:10F000005B46002B3BD1022300221E43022161E715
:10F01000434613439B4637D04346002B00D162E161
:10F02000404601F069FA03000B3B1C2B00DD53E165
:10F0300002004146083A914088461D21CB1A5146AC
:10F04000D9400B0041460B439B46534693401A0060
:10F05000009B25499C46604403008C466344009312
:10F06000002137E70323B14600900C26029311E7F5
:10F070000023009301330426002702930AE70323A9
:10F08000C3461E43032125E701331E43002201210D
:10F0900020E700239A46802300271B03094A61E7E3
:10F0A000802349461B03194200D1E2E05946194228
:10F0B00000D0DEE00B431B0317001B0BA246014AE6
:10F0C00050E7C046FF07000001FCFFFFD85C0100CD
:10F0D000FF030000FFFFFFFEFE070000FFFF0F80A1
:10F0E0000DFCFFFF01F8FFFFF3030000D94500D935
:10F0F000CBE000D1C6E03C0048460027009B013B26
:10F1000000935B46160E1B021E43130298463304FF
:10F110001B0C9946310C0191FEF780FC4A46424394
:10F120000B04210C050019438A4207D98919013DB6
:10F130008E4203D88A4201D9851E8919881A0199FD
:10F14000FEF76CFC09048C464A462104644642439F
:10F15000090C030021438A4204D98919013B8E42DC
:10F1600000D8F1E02D041D43AB464346891A4246C0
:10F17000280C12041D0C5B46140C22001B041B0CF3
:10F180005A4303946B434443029568431B19150C7F
:10F19000EB189C4203D980246402A44660441C0CF2
:10F1A00015041B042D0C20185D19814277D373D0F0
:10F1B0000C1AA24A7D1BAF42BF419446009B7F427E
:10F1C0006344E01B1C00864200D1DBE00199FEF79E
:10F1D00025FC4A4642430B04290C070019438A4286
:10F1E00007D98919013F8E4203D88A4201D9871E67
:10F1F0008919881A0199FEF711FC09044A468946C3
:10F2000029044D464243090C030029438A4207D989
:10F210008919013B8E4203D88A4201D9831E89197C
:10F220003F04891A3A00039F1A43380013041B0C49
:10F23000584381460298150C6F4343434543484663
:10F24000000C8446DB1963449F4203D980204002AE
:10F250008446654448461F0C00041B04000C7D19BD
:10F260001818A94200D284E000D17FE001231A439C
:10F2700057E680234A461B0313431B031B0BAA4676
:10F280006F4A6FE6BA4200D935E74B46DC075808AB
:10F290007B081C43FF0734E70024AF4289D2474470
:10F2A0004745A4415B466442A4196418013BA64249
:10F2B0001ED2A0426DD800D1B6E0241A9B4678E752
:10F2C00003005A46283B9A400027914688E6584654
:10F2D00001F012F9203072E603005246283B9A40B2
:10F2E00093460022B4E6504601F006F920309AE633
:10F2F000A642E2D1B845DCD9341A9B4659E71F2B08
:10F3000065DC504C0099A4465C46614408008C4082
:10F3100011008240D940501E82410C4314435A468A
:10F32000DA401300620709D00F222240042A05D0D8
:10F330002200141D9442894149425B181A0262D589
:10F340000122002300270DE68A4200D80AE7831E27
:10F35000891907E70F231340042B00D1E6E5171D99
:10F360009742924153429B44FA08E0E5002800D1BD
:10F37000D7E57118531EB14227D3A94215D358D0EF
:10F380001A0073E7002B00DC04E6012300229B44F3
:10F39000CDE502234744474589415B429C464942AB
:10F3A00089190C19E344241A03E743465F004745D3
:10F3B0009B41B8465B429E19023A8919A94200D086
:10F3C00054E7404500D051E7ABE51A00F6E71F21AE
:10F3D0005F4649420C1BE740202B07D01A49009B8F
:10F3E0008C46634418005B4683401A43501E82419A
:10F3F0003A4307270023174009D00F21002311406B
:10F400001400042995D122005F075B021B0BD20870
:10F4100017430022A6E5802359461B030B431B0319
:10F4200017001B0B064A9DE5BD42B2D89B4600243F
:10F43000BFE68045B9D31A00C3E7C046FF0300000A
:10F44000FF0700001E0400003E040000F0B54F4618
:10F450004646D6468446C0B58046194E18030F036B
:10F460004D00000B5C0082463F0B6D0DC90F9146AD
:10F47000640DDB0F0120B5420AD0B44203D0A5428F
:10F4800001D157450CD01CBC90469946A246F0BD10
:10F4900066463E43F7D1AC42F5D154461443F2D10F
:10F4A0000120C845EFD1994207D0002DEBD163462A
:10F4B0001F433800471EB841E5E70020E3E7C04698
:10F4C000FF070000F0B54F464646D6464D00C0B592
:10F4D0000E03C90F8A462C491F035C008046360B79
:10F4E0006D0D91463F0B640DDB0F8D421ED08C429B
:10F4F00016D0002D1ED130438446002C01D13A4352
:10F5000023D06246002A1AD09A4529D051460220BB
:10F510000139084001381CBC90469946A246F0BD0E
:10F5200039001143E5D002204042F4E73043FAD1DC
:10F53000AC420FD0002C0FD13A43E7D00CE00122AF
:10F54000013B934318000130E5E763460020002BA0
:10F55000E1D0DBE73A43E6D19A45D7D1A542D5DCE5
:10F56000A54205DBBE42D1D808D00020BE42D2D28F
:10F5700050460123013898430130CCE7C845C5D82F
:10F580000020C845F4D3C6E7FF070000F0B54F469A
:10F590004646D6464D00C0B50E03C90F8A462E49D1
:10F5A0001F035C008046360B6D0D91463F0B640DCA
:10F5B000DB0F8D4218D08C4211D0002D18D1304372
:10F5C0008446002C1ED13A431CD163460020002BF8
:10F5D00030D0514602200139084001382AE0390074
:10F5E0001143EAD0022025E03043FBD1AC4226D0C3
:10F5F000002C26D13A4324D151460220013908403B
:10F60000013817E06246002A0FD09A45E1D1A542A1
:10F6100005DBBE42DDD819D00020BE420AD25046DA
:10F62000012301389843013004E00122013B934358
:10F63000180001301CBC90469946A246F0BD3A43E2
:10F64000D0D19A45C5D1A542C3DCE0E7C845C0D8B2
:10F650000020C845E3D3EDE7FF070000F0B55746AB
:10F66000DE464E464546E0B5834606000F03480099
:10F6700087B092461D003F0B400DCC0F002800D1F3
:10F680006FE0DE4B984238D08023FF001B041F43FD
:10F69000730F3B430193DA4B0027994600239B46A7
:10F6A000F60081442B0369001B0B52469846490D16
:10F6B000ED0F002900D185E0D04B994200D173E0D5
:10F6C0004346DA0080231B0413435246CC48520FB2
:10F6D00084461343524600206144D20089442100ED
:10F6E000694000918C46012149448A460F2F00D978
:10F6F00090E0C449BF00CF59BF465B463B430193EE
:10F7000000D06AE102230827002681469B46C9E70C
:10F7100032005846019B61460091022800D175E0F5
:10F72000032800D1FEE1012800D02CE100230027AE
:10F73000002600253F032A0D3F0BB34812053A432C
:10F7400002401B051343009A5B00D1075B080B4383
:10F750003000190007B03CBC90469946A246AB4623
:10F76000F0BD5B463B43019300D12FE1002F00D158
:10F77000A5E1380000F0C0FE03000B3B1C2B00DDB0
:10F7800096E11D22D31A5A460100DA405E46083936
:10F790008F4013008E403B4301939C4B00271B1A64
:10F7A000994600239B467DE7414653460B439349C8
:10F7B0008C46E144002B00D01AE1022202201743BC
:10F7C00000228CE7134300D10DE14346002B00D10A
:10F7D00081E1404600F090FE02000B3A1C2A00DD59
:10F7E00072E10100434608398B4098461D239A1A5E
:10F7F0005346D3401A004346134352468A40494673
:10F80000081A824989468144002068E77B4B00271B
:10F8100000268EE7140C1204120C1100370C36046B
:10F82000350C794328008C462E00604360448346A3
:10F8300056432100300C804658467943404402919B
:10F84000844506D98846802149028C46E0444146D9
:10F8500002913604010C360C00048B4681191E0CF3
:10F860001B041B0C0391190079438C462800754337
:10F870006544A8465843050C45447743A94203D93B
:10F88000802149028C466744290C8C4639000004CB
:10F89000000C2D042D186144AB4405915946049188
:10F8A00001990F043F0C080C390051434243904624
:10F8B00002008C46090C8B4662437C4344445C4402
:10F8C000A04503D98021490288464244210C88463C
:10F8D00061460904090C8C4639005943434370437F
:10F8E0007E430F0CF6182404BE19644442448C462F
:10F8F000B34203D980235B0298464044029B614691
:10F900009846049B370443449B46AB45AD416B424C
:10F910000D0405992D0C8C467F196744FD18A846E7
:10F920005D462D19A542A44193466442A446C344B2
:10F93000DC448F42BF4198459B4193459241A44589
:10F94000A4415B427F421F43360C52426442BF19BE
:10F950002243BF18624638184302D20D039913435D
:10F960006A020A43501E82416146ED0D2A434E024F
:10F970003243D90100D4B3E001265008324002439B
:10F98000DE0732435B08224C5444002C62DD5107F1
:10F9900009D00F201040042805D0101D904292413C
:10F9A00052429B180200D90104D580241948E40072
:10F9B000034054441848844200DD27E75E075B0299
:10F9C000D2081F0B630516435B0DB2E60023994670
:10F9D0000133042700269B4664E6032301978146F2
:10F9E0000C279B465EE6012201201743002276E6A3
:10F9F000032303201F43434671E6C046FF07000070
:10FA000001FCFFFF185D0100FFFF0F800DFCFFFFF1
:10FA1000FF030000FFFFFFFEFE070000002380271A
:10FA200000933F030026434B83E6019B3200A4462C
:10FA3000584670E6AC466EE6802701993F0339428E
:10FA40002DD03B422BD11F433F033F0B00951600A7
:10FA5000384B6EE601252D1B382D00DD66E61F2D87
:10FA600040DC35481C005044160082408440EE4083
:10FA7000501E824134431443EB40620709D00F22E9
:10FA80002240042A05D02200141D944280414042A5
:10FA90001B181A023ED501230027002649E68027BD
:10FAA000019B3F031F433F033F0B0094214B40E664
:10FAB00003005A46283B9A40002601926DE65846BC
:10FAC00000F01AFD203057E603005246283B9A40CA
:10FAD0001300002293E6504600F00EFD20307BE636
:10FAE000CA4650E71F201E004042041BE640202D5E
:10FAF00003D0124C5444A3401A43501E8241324357
:10FB000007260027164009D00F20002310401400BC
:10FB10000428B9D122005E075B021F0BD2081643EE
:10FB2000002306E680273F031F433F033F0B1600D9
:10FB3000004BFEE5FF0700001E0400003E0400002D
:10FB4000F8B557464E464546DE460C000903E0B57B
:10FB5000490A460F5F0031431E03DB0F760A9B46BE
:10FB6000530F3343C84E6500C000E40FD2006D0D43
:10FB7000A24681467F0D9C469046B74200D1B9E02F
:10FB80005B46012673409B46EE1BA34500D183E0F4
:10FB9000002E63DD002F00D0B1E06346134300D197
:10FBA00023E1731E002B00D0BAE1861A6346B042EF
:10FBB00080410125C91A4042091A0B0200D447E1CD
:10FBC00049024B0A98464346002B00D189E1404642
:10FBD00000F092FC0300083B1F2B00DD7CE120229B
:10FBE0003000D21A4146D040994002009E400A435C
:10FBF0009D4200DD6AE15D1B6B1C1F2B00DD94E163
:10FC0000202110003500C91A8E40DA408840DD40BE
:10FC1000711E8E4111000722284300250643324001
:10FC2000002A09D00F233340042B05D0331DB342E3
:10FC3000B641764289191E000B0200D43DE26A1CCF
:10FC4000914B55056D0D9A4200D119E18F4AF60886
:10FC50000A40570752023743120B9BE0002E00D098
:10FC6000C5E06E1C7605760D012E00DC48E1674686
:10FC7000861ACB1BB042BF417F42B8461F004346A5
:10FC8000FF1A3B00B8461B0200D55FE137439AD10B
:10FC900000220024002579E0002E00DCFAE0002F8D
:10FCA00000D18DE0784B9D4267D0802367461B04CE
:10FCB0001F43BC46382E00DC52E1634613435A1EF4
:10FCC00093411E1886428041404209180B0200D41D
:10FCD000BEE06D4B01359D4200D1D2E06B4A730806
:10FCE0000A4001210E401E435108D30707221E433C
:10FCF000324095E71E00164300D045E740E7624BCF
:10FD00009D423AD0802367461B041F43BC46382ED1
:10FD100000DDEBE01F2E00DC3AE133006746203BBC
:10FD2000DF403B00202E05D04027BF1B6646BE406B
:10FD3000324390464646721E96413343DAE0002B2A
:10FD400000D114E26346134300D168E180234E07DB
:10FD5000C008C9081B030643194208D06046C00802
:10FD6000184204D163460100D2085E071643F3002F
:10FD70009946C900720F444D11434B46DE08424B71
:10FD80004F073743CA089D4200D16EE012036D054C
:10FD9000120B6D0D00211203130B0A0D12051A43ED
:10FDA0003B4B2D0513402B435B00E4075B082343CB
:10FDB000380019003CBC90469946A246AB46F8BDB7
:10FDC0006346134311D0731E002B00D007E1861841
:10FDD0008642804161444042091801250B0237D513
:10FDE00002257BE73E00614691463500C5E75C464B
:10FDF000002D00D0E1E00B000343F3D0731C00D1D1
:10FE0000ACE1214B9F4200D13AE1F343382B00DDB6
:10FE10006FE11F2B00DD8CE120250E00ED1AAE40B6
:10FE2000B0460600AA46DE40454635432E005546FC
:10FE3000D940A8406346451EA8415B1A9C46304302
:10FE4000161AB242924163465242991A3D00B4E6F4
:10FE500007223240002A00D0E4E60B4BF6084F0799
:10FE60003743CA089D4200D090E73B00134300D1BE
:10FE7000A6E180231B031A431203120B024D89E7EC
:10FE800015000022002785E7FF070000FFFF7FFF26
:10FE9000FFFF0F80002E00D0C7E06B1C5E05760DC3
:10FEA000012E00DCF0E0C84DAB4200D1B9E085186E
:10FEB0000A00854289416244494251180722CE070F
:10FEC0006D082E43490832401D00A9E6BF49ED1ACE
:10FED000114007223240A3E6320028388240002633
:10FEE00086E6300000F008FB203073E663461343DB
:10FEF0005A1E9341C61AB04280414042091A5CE63C
:10FF00000E00674606431743002D5ED1002E00D039
:10FF1000F3E0002F00D11EE15C46614691462CE7DC
:10FF2000A94FBE427BD01E00F1E610001F3DE84005
:10FF3000202B03D04021CB1A9A401643731E9E41BA
:10FF40000722064332400021002583E7161A634644
:10FF5000B2428041591A40420B1A98465C4632E63A
:10FF60001F2E00DDABE02027BB1B9A466346574699
:10FF7000BB40994613004F46F3401F433B00574692
:10FF8000BA40571EBA4113436246F240891898E6B8
:10FF90002027BB1B9A4663465746BB409946130031
:10FFA0004F46F3401F433B005746BA40571EBA41E5
:10FFB00013436246F240891A9CE7834B9F425FD00D
:10FFC00080252D047342294320E7002E0CD1002FF9
:10FFD00000D1D0E05C46614691467B4DCDE67A4F3C
:10FFE000BE421CD01E0065E6002F18D0C0084E0788
:10FFF00006438020C9080003014208D06346DC089C
:020000021000EC
:10000000044204D12100DA46D2085E071643F30009
:10001000994601245346C900720F11431C406A4D92
:10002000ABE61D0000220027B4E6002D59D10B00DD
:10003000034300D1D6E6731C00D1B2E0624B9F426D
:100040001ED0F343382B6FDC1F2B00DD97E02025FB
:100050000E00ED1AAE40B0460600AA46DE40454608
:1000600035432E005546A840D940451EA8418C4432
:100070000643B61896429241514261443D0025E63E
:100080003D006146914678E60B000343002D00D009
:1000900055E6002BF5D06346134300D16DE6861874
:1000A0008642804161444042091800220B0200D47C
:1000B000D0E6464B01351940B2E5B1465DE6330066
:1000C0006746203BDF403B00202E05D04027BF1B6A
:1000D0006646BE40324390464646721E96413343C2
:1000E000EFE5394B9F42CBD080252D047342294345
:1000F000A8E70843411E8841A2E6002F00D13CE654
:100100006346861ACF1AB0429B415B42FB1A98465F
:100110001B024ED5161A6346B2429241591A5242F8
:10012000891A5C4600227BE501430E00711E8E4158
:100130009FE71D000E00203DEE40B046202B04D06E
:100140004025EB1A99400843814648464346411EE4
:100150008841184374E60022002417E6161A634605
:10016000B2429241591A5242891A3D0025E5614630
:100170009146154D01E680220024120379E61D0008
:100180000E00203DEE40B046202B04D04025EB1A57
:100190009940084381464E464346711E8E411E4398
:1001A00067E7861896429B4161445B42C9183D004F
:1001B0008CE547463743CED007224146324049E6D8
:1001C00000273A00E6E5C046FF070000FFFF7FFF7B
:1001D00070B50C4E0D031C0349005B002D0B490D3F
:1001E000240B5B0DB14208D0064900208B4203D19D
:1001F00014432000441EA04170BD05430120002D82
:10020000FAD1F1E7FF07000030B5144D0A034B00A7
:10021000120B5B0DC90F0024AB4211DD104CA34241
:1002200010DC8024640322430E4CE41A1F2C0CDDE6
:100230000D48C31ADA4013005C42002900D11C00AB
:10024000200030BD094BCC18FAE7094DE040AC4620
:1002500063449A4013000343EEE7C046FE030000E8
:100260001D0400003304000013040000FFFFFF7FA3
:10027000EDFBFFFF70B500282DD0C317C5185D40FA
:10028000C40F280000F038F9154B1B1A5B055B0DF5
:100290000A2815DD0B38854000222D032D0B002187
:1002A00010002D030A0D2D0B12052A430D4D1B05C1
:1002B0002A4013435B00E4075B082343190070BD29
:1002C00002002900153291400A000B21081AC5408E
:1002D0002D032D0BE3E70024002300250022DEE799
:1002E0001E040000FFFF0F8010B5041E25D000F093
:1002F00003F9144B1B1A5B055B0D0A2812DD0B3842
:10030000844000222403240B0021100024030A0D42
:10031000240B120522430C4C1B05224013435B00A7
:10032000590810BD02002100153291400A000B212E
:10033000081AC4402403240BE6E70023002400220B
:10034000E2E7C0461E040000FFFF0F804100090ED7
:100350004B1C70B5DBB24602750AC40F012B14DDCD
:10036000E0239B006D07360BCB1800210A0D2800F7
:1003700012051C4D32435B052A405B0813435B00AA
:10038000E4075B082343190070BD002914D1002D38
:100390001ED0280000F0B0F80A281CDC0B232A002D
:1003A0001B1ADA40030015339D400F4B12031B1A32
:1003B0005B05160B5B0DD8E7002D06D0320B8026AF
:1003C00036036D071643094BCFE7084B0026CCE7F1
:1003D00000230026C9E703002A000B3B9A400025B2
:1003E000E3E7C046FFFF0F8089030000FF0700001E
:1003F000F0B54C00640D0B03621C5B0A460F5205FE
:10040000C90F1E43C500520D012A29DD374BE718DD
:10041000FE2F1CDC002F3BDD8001431E984107228C
:10042000F3006D0F03432B431A40002A04D00F2220
:100430001A40042A00D004338022D2041A4024D067
:100440000137FAB2FF2F02D09B01580A01E0FF22C8
:1004500000204002D205400AC90710430843F0BDFE
:100460003543002C04D1002D0AD100220020F0E7F2
:10047000002DECD08020C0033043FF22E9E70024A8
:1004800000235B02580AE2B2E3E7DB083C00F8E72E
:100490003B001733F3DB80231B0433431E26F61B7C
:1004A0001F2E14DD02225242D71B1A00FA401700F9
:1004B000202E04D00E4A94466444A3401D432B00D2
:1004C0005D1EAB4107223B431A400027ADE7094AB6
:1004D0002800A218954093406C1EA541F0400722C9
:1004E0002B4303431A4000279FE7C04680FCFFFFD1
:1004F000A2FCFFFF82FCFFFF1C2101231B0498428A
:1005000001D3000C10391B0A984201D3000A0839A4
:100510001B09984201D30009043902A2105C40185B
:100520007047C046040302020101010100000000FF
:100530000000000010B5002903D1FFF7DDFF2030D7
:1005400002E0081CFFF7D8FF10BDC046F0B54E46CC
:100550005746DE464546E0B50F00002183B0060051
:100560008946002F06DA3900002746428F410121D3
:1005700049428946002B07DA4946C943100089469B
:100580001900002342428B4134003D0092469846B8
:10059000BB4269D866D041465046FFF7CBFF834641
:1005A00039003000FFF7C6FF5B461B1A9C46203B14
:1005B0009B4600D575E05146584681400B00514698
:1005C000604681400A00BB4261D85ED034003D00E5
:1005D0005946A41A9D41002900DA7AE00021002042
:1005E00001260090019159468E40019661460126F0
:1005F0008E4061460096002950D0D90756085F0802
:100600000E4363460EE0AF4201D1A6420CD8A41BB4
:10061000BD41012124196D410022013B641855415F
:10062000002B06D0AF42EED9013B24196D41002BBF
:10063000F8D1009801995B4600196941002B3DDB18
:100640002E00DE4063462C00DC405B46002B4BDB7B
:1006500034005D46AC4023006446A6403200801A58
:10066000994103E0B24296D9002000214B46002B6D
:1006700004D003000C0000215842A14103B03CBC4F
:1006800090469946A246AB46F0BDB1429ED90021A4
:1006900000200090019161460029AED10098019997
:1006A000E4E72023624651469B1AD9404046009118
:1006B00061468840030000990B4380E7624620238F
:1006C0009B1A2A009A40260013006246D6401E4319
:1006D000B8E7614620260127761A00200021F7405E
:1006E00000900191019781E767462023624635001B
:1006F000BC409B1ADD4023002B43ADE730B51C0006
:10070000094B05001B6885B0D868084B002A01D149
:10071000074B1A000292019300912B002200054919
:1007200000F02CF801F07AF9A4000020585D0100D7
:10073000EB430100655D010010B50A22002101F0C4
:1007400081F810BD014B18687047C046A400002016
:10075000084B10B50400002B02D0002100E000BFC0
:10076000054B1868836A002B00D09847200002F0E0
:10077000ADFFC04600000000945D01000EB403B55B
:10078000010003AB044804CB0068019300F03EF97C
:1007900002B008BC03B01847A400002070B50026C2
:1007A0000C4D0D4C641BA410A64209D1002602F08A
:1007B0008FFF0A4D0A4C641BA410A64205D170BDE0
:1007C000B300EB5898470136EEE7B300EB58984773
:1007D0000136F2E774020020740200207402002047
:1007E00088020020EC3000687047000010B5034B11
:1007F0000100186800F084F810BDC046A400002075
:1008000082B0002900D101A9101E06D0002B06D00D
:1008100013780B601078431E984102B07047022095
:100820004042FAE7002310B59A4200D110BDCC5CDB
:10083000C4540133F8E710B5884202D98B189842A6
:1008400003D3002307E08B5C8354013AFBD210BD35
:10085000CC5CC45401339A42FAD1F8E70300121871
:10086000934200D1704719700133F9E770B5050064
:10087000002910D00C1F2368002B00DAE418280090
:1008800002F049F91D4A1368002B05D1636014601A
:10089000280002F041F970BDA34209D9216860180F
:1008A0008342F3D118685B6841182160EEE71300BA
:1008B0005A68002A01D0A242F9D919685818A042F2
:1008C0000BD120680918581819608242E0D11068CD
:1008D0005268411819605A60DAE7A04202D90C2325
:1008E0002B60D5E721686018824203D110685268F6
:1008F0004118216062605C60CAE7C046A41B00200A
:10090000032370B5CD1C9D43083506000C2D1ED267
:100910000C25A9421DD8300002F0FDF8254A1468C4
:100920002100002919D1244C2368002B03D1300069
:1009300000F036FE20602900300000F031FE431C3C
:100940002BD10C233000336002F0E6F803E0002DD9
:10095000DFDA0C233360002070BD0B685B1B19D4F9
:100960000B2B03D90B60CC18256003E04B688C423D
:100970000DD11360300002F0CFF8200007220B30B9
:10098000231D9043C31AE7D05A42E250E4E7636064
:100990000C00EFE70C004968C3E70323C41C9C4329
:1009A000A042E1D0211A300000F0FAFD431CDBD157
:1009B000C7E7C046A41B0020A81B0020936810B501
:1009C000013B9360002B04DA9469A34207DB0A29F8
:1009D00005D01368581C10601970080010BD00F095
:1009E00045FF0100F9E7F8B506000F001400D5181F
:1009F000AC4201D1002007E021783A003000FFF737
:100A0000DDFF0134431CF3D1F8BD0000F0B59FB009
:100A100002900F0016000593002805D08369049307
:100A2000002B01D101F060FF7B4B9F425BD1029B09
:100A30005F68BB891B0762D53B69002B5FD0002331
:100A400006AC6361203363761033A37635002B78D0
:100A5000002B01D0252B5CD1AB1B04930CD03200B2
:100A600039000298FFF7BFFF431C00D1C4E0626960
:100A7000049B9446634463612B78002B00D1BBE058
:100A8000012200235242626002A9543252186E1CA5
:100A90002360E360A3601370A365317805225F488B
:100AA00002F02EF8751C002835D12268D30604D533
:100AB000532302A95B1820211970130704D553236F
:100AC00002A95B182B21197033782A2B2CD0350002
:100AD00000210A20E3682A786E1C303A092A64D97A
:100AE00000292ED026E04E4B9F4202D1029B9F68E8
:100AF0009FE74C4B9F429CD1029BDF6899E73900EE
:100B0000029800F015FF002899D0012040421FB044
:100B1000F0BD01359BE7414B2268C01A0123834099
:100B2000134323602E00B8E7059B191D1B68059130
:100B3000002B01DB099304E05B42E36002231343D3
:100B400023602B782E2B0AD16B782A2B35D1059B6D
:100B500002351A1D1B680592002B2BDB0793324EC2
:100B600029780322300001F0CBFF002806D0402373
:100B7000801B8340226801351343236029780622B5
:100B80002A486E1C217601F0BBFF00283AD0284B82
:100B9000002B25D10722059B073393430833059388
:100BA0006369039A9B18636150E7434301219B18D3
:100BB000350090E701235B42D0E700230A201A00AA
:100BC0000135636029786E1C3039092903D9002B5F
:100BD000C5D00792C3E74243012352183500F1E71D
:100BE00005AB00933A00134B2100029800F0C0F8C7
:100BF0000390039B0133D3D1BB895B0600D584E707
:100C00000B9884E705AB00933A000A4B2100029849
:100C100000F068FBECE7C046105F01009E5D01003C
:100C2000305F0100F05E0100A45D0100A85D0100DD
:100C3000710D0100E7090100F0B58BB014001D1E15
:100C4000129953DA802424061B191D0014002D2349
:100C50000B702023149E03229E43462E07D03300A0
:100C6000453B59424B411099013ACB18109309ABBF
:100C7000049308AB0393139B00920293109B2200F2
:100C800001932B0000F058FF0700472E02D1119B63
:100C9000DB0724D5109BFB180793462E14D13B7815
:100CA000302B0CD10022002320002900FCF7C4FFC8
:100CB000002804D10123109A9B1A139A1360139BE6
:100CC000079A1B68D31807930022002320002900ED
:100CD000FCF7B2FF302200280DD0079B09933800A3
:100CE000099B159ADB1B13600BB0F0BD0023AFE727
:100CF000591C09911A70099B07998B42F8D3EEE7AA
:100D0000F0B5831C85B0019306000C0002702B2304
:100D1000002901DA2D234C427370092C22DD02AB2D
:100D2000DD1D20000A21FCF763FF6F1E3031397092
:100D300020000A21FCF776FE040009280BDC023DA6
:100D40003034019B2C7002AA07321800AA4204D842
:100D5000801B05B0F0BD3D00E3E72A7801351A702D
:100D60000133F0E73023E418B370301DF470EFE77F
:100D7000F0B595B00C000A920B931A9D099001F002
:100D800047FE036818000C9300F094FC00231293B4
:100D900023680E900D930D99277E2B680722C905B5
:100DA00045D59B1893431A0008322A601A685B687D
:100DB000A264E3640122E56CA66C6B005B080F93F0
:100DC0005242AC4B30000F99FFF702FA002830D1A5
:100DD0000122A84B524230000F99FCF73DFF00283A
:100DE00027D10022002330002900FCF72BFF002828
:100DF00003D023002D2243331A709F4D472F00D874
:100E00009E4D032300260D9A236101339A432260ED
:100E10000B9B13AA009321000A9B099800F0F4F998
:100E2000431C00D093E00120404215B0F0BD0733D1
:100E3000B8E732002B0030002900FFF7C9F900287D
:100E400004D08F4D472FDCD88E4DDAE780230D99E3
:100E50006268DB000B43511C43D10732626012AA67
:100E60000021059211AA0392232223600691019387
:100E700008A9636852180292009332002B0004976D
:100E80000998FFF7D9FE20233A0005009A43472A24
:100E900007D1119BDA1C02DB6268934245DD023FF9
:100EA000FFB21199652F25D8200001393A00503042
:100EB0001191FFF725FF129A060013182361012AEA
:100EC00002DC2268D20701D501332361232308AA5B
:100ED0009B181B78002B9BD023002D2243331A70C4
:100EE00096E7672F00D176E1472FB8D1002AB6D117
:100EF0000122B3E7662F19D1636800290CDD216157
:100F0000002B02D12268D20702D501335B1823617E
:100F1000119B0026A365D9E7002B03D1012221688C
:100F2000114200D09A1C2261F2E76727119B129AA6
:100F3000934205DB22682361D207E9D50133E6E756
:100F40000121002B01DC4918C91A5218EBE722686D
:100F5000530508D423692A000A9909980B9DA847CC
:100F6000431C29D15FE7652F00D8E0E0A06CE16C5D
:100F700000220023FCF760FE002834D00123424AFF
:100F80000A9909980B9DA847431C00D14BE7119B78
:100F9000129A934202DB2368DB070DD50B9D0E9B53
:100FA0000C9A0A990998A8470025431C00D13AE7F2
:100FB000129B013BAB420ADC23689B0700D508E18A
:100FC000139BE068984200DB2FE718002DE7220012
:100FD00001231A320A9909980B9EB047431C00D18D
:100FE00021E70135E4E7119B002B2DDC0123264A84
:100FF0000A9909980B9EB047431C00D113E7119B37
:10100000002B05D1129B002B02D12368DB07D3D51F
:101010000B9E0E9B0C9A0A990998B0470026431C18
:1010200000D100E7119B5B42B34201DC129B92E7C7
:10103000220001231A320A9909980B9FB847431CD2
:1010400000D1F0E60136EDE7A36D129F9F4200DD6F
:101050001F00002F08DD3B002A000A9909980B9E0B
:10106000B047431C00D1DEE600230D93FB43DB17A2
:101070000F9318E0FFFFEF7FB35D0100AF5D01004C
:10108000BB5D0100B75D010026380100220001238D
:101090001A320A9909980B9EB047431C00D1C2E648
:1010A0000D9B01330D930F9BA66D0D9A3B40F31AD8
:1010B0009342EBDC119B129AAD19934210DB23682B
:1010C000DB070DD4129F119BBE1BFF1AB74200DD38
:1010D0003700002F0DDCFE43F31700250C931CE0B6
:1010E0000E9B0C9A0A9909980B9FB847431CE9D1AB
:1010F00099E63B002A000A9909980B9DA847431CD2
:10110000E9D190E6220001231A320A9909980B9E30
:10111000B047431C00D186E60135119A129B0C9909
:101120009B1A3A000A409B1AAB42EBDC44E7129B45
:10113000012B02DC01231A4232D001232A000A9932
:1011400009980B9FB847431C00D16CE60E9B0C9A84
:101150000A9909980B9F0135B847431C00D162E6F4
:10116000A06CE16C129B00225F1E0023FCF764FD63
:101170003B00002814D000250AE0220001231A3287
:101180000A9909980B9FB847431C00D14BE60135DB
:10119000129B013BAB42F0DC220033005032DBE615
:1011A0002A000A9909980B9DA847431CF4D13AE6F6
:1011B0002200012319320A9909980B9EB047431C5B
:1011C00000D130E60135E368139A9B1AAB42EFDC9D
:1011D000F6E60025F7E7002A00D189E6002106910E
:1011E00012A9059111A90391232108A809182360C8
:1011F000019300922B000497029132000998FFF7A7
:101200001BFD050045E6C046F7B5150001938A6849
:101210000B6900900C00934200DA130022002B604F
:1012200043321278002A01D001332B6023689B06D9
:1012300002D52B6802332B60062723681F4027D076
:10124000230043331B785A1E93412268920630D400
:101250002200019943320098089EB047431C25D0D4
:10126000062320682A68E16803400025042B03D187
:101270008D1AEB43DB171D40A3682269934201DD01
:101280009B1AED180027BD4220D1002010E0013745
:10129000E3682A689B1ABB42D2DD2200012319327F
:1012A00001990098089EB047431CF0D101204042AC
:1012B000FEBD3020E1184331087021005A1C453131
:1012C0000978A218433202331170C1E722000123CA
:1012D0001A3201990098089EB047431CE6D00137A6
:1012E000D1E70000F0B589B004920A0043320593BB
:1012F000039002920A7E0C000E9B6E2A00D186E0BB
:101300001FD8632A33D008D8002A00D18CE0582A8D
:101310004DD0250042352A7030E0642A01D0692A78
:10132000F7D1196825680A1D280629D508681A60AA
:10133000002803DA2D23029A404213706B4E0A27CD
:101340004FE0732A74D008D86F2A1FD0702AE0D1DA
:10135000202209680A43226003E0752A16D0782A01
:10136000D7D12200782145321170614E22E025004C
:101370001A684235111D196013682B70012365E04E
:1013800008681A606906D3D500B2D1E719682568E4
:10139000081D186008682E0605D5544E08276F2AC8
:1013A0001BD00A2719E06D06F7D580B2F5E7453165
:1013B0004E4E0A7018682268011D006819601506F3
:1013C00021D5D30702D520231A43226010270028F5
:1013D00003D1202322689A43226023000022433352
:1013E0001A706368A360002B58DB042221689143C4
:1013F0002160002854D1029D002B5AD0250033785B
:1014000042352B7055E05506DBD580B2D9E71A6816
:101410000D68101D4969186013682E0601D5196002
:1014200002E06D06FBD519800023029D23614FE089
:101430001A68111D1960156800216268280001F002
:101440005FFB002801D0401B6060636823610023BC
:10145000029A13703CE023692A0004990398059DC1
:10146000A847431C3ED023689B0715D4079BE06820
:10147000984239DA180037E0220001231932049922
:101480000398059EB047431C2CD00135E368079AAA
:101490009B1AAB42F0DCE9E70025F7E70028ADD066
:1014A000029D3900FCF7BAFA735C013D2B700028ED
:1014B000F7D1082F09D12368DB0706D563682269B5
:1014C000934202DC3023013D2B70029B5B1B2361A6
:1014D000059B07AA00932100049B0398FFF794FE45
:1014E000431CB8D10120404209B0F0BDBF5D0100EE
:1014F000D05D01000D4B70B51C680500A36B002B7F
:101500000FD11820FFF772F9094BA0630360094B54
:1015100001224360084B83600B2383810023026117
:1015200043610022A36B1D615A6170BDA4000020BD
:101530000E33CDAB34126DE6ECDE0500124B10B568
:101540001C68A36B002B0FD11820FFF74FF90F4B2E
:10155000A06303600E4B012243600E4B83600B239C
:101560008381002302614361A46B0B4A2069616996
:101570000A4BFCF7D3FB012200238018594120615C
:1015800061614800400810BDA40000200E33CDABBF
:1015900034126DE6ECDE05002D7F954C2DF451588C
:1015A000002370B5064C05000800236002F078F8AF
:1015B000431C03D12368002B00D02B6070BDC046B4
:1015C000EC2F00200CB430B5164B9DB00C1E1D68DE
:1015D00008DA8B2301202B6040421DB030BC08BCD0
:1015E00002B01847822302A99B008B81002302903E
:1015F00008619C4200D0631E8B604B6101235B42FB
:10160000CB81209A21AB2800019301F003FE431CFB
:1016100001DA8B232B60002CDFD00023029A137099
:10162000DBE7C046A40000200EB400B50B499CB017
:101630001DAB02900690079104910948094904CB1B
:101640000591006802A9019301F0E4FD0023029ACC
:1016500013701CB008BC03B01847C046FFFFFF7FE3
:10166000A40000200802FFFF020010B51378541CEC
:10167000002B05D1CC5CD4540133002CFAD110BD21
:101680002200F3E7C9B20378002B04D08B4200D1CB
:1016900070470130F7E74B42594149420840F7E7AC
:1016A00002780B78002A03D0013001319A42F7D03A
:1016B000D01A70470023C25C0133002AFBD1581EA8
:1016C0007047002330B59A420AD0013AC45CCD5C21
:1016D000AC4204D1934202D00133002CF6D1631BFB
:1016E000180030BD30B50500002A00D130BD0C789F
:1016F000013A6B1C2C700131002C05D19A189A42CA
:10170000F4D01C700133FAE71D00EDE710B5037843
:10171000002B0FD10B785A4253415B42184010BD49
:101720000023CA5C002AFAD0C45C944201D1013380
:10173000F7E701300378002BF2D11800EFE7000043
:10174000F0B51F000E0087B00590019102920C9831
:101750003478FFF747F8082200194378751C1340C6
:1017600036D12D2C36D1B51C74780126002F62D0CD
:10177000102F09D1302C07D120222B789343582BDE
:1017800054D110276C7802352D4B3900F31818000E
:101790000393FCF743F9049101210023494202001D
:1017A0008C4618002100303909291AD80C00A742AC
:1017B00023DD591C09D06346824206D302D1049925
:1017C000A14202DB0123784320182C780135E9E798
:1017D0002E00BCE72B2C01D01E00C7E7B51C747887
:1017E000FAE721004139192901D8373CDFE7210008
:1017F0006139192901D8573CD9E75A1C08D1059AF3
:1018000023331360029B0398002B09D107B0F0BD6E
:10181000002E00D04042029A002AF7D0002B01D0BF
:101820006B1E0193029B019A1A60EFE73024002F90
:10183000AAD10827A8E7302C9ED00A27A4E7C046E3
:10184000FFFFFF7F37B51300064A05001068046AE2
:10185000002C00D1044C0A0000942900FFF770FF0F
:101860003EBDC046A400002008010020F8B50500D8
:101870000E001400002804D08369002B01D101F070
:1018800033F8224B9C422DD16C68A369A360A389D5
:101890001B0731D52369002B2ED023682269F7B2AC
:1018A000981A6369F6B2834205DC2100280000F033
:1018B000ADFF002826D1A3680130013BA360236857
:1018C0005A1C22601F706369834204D0A389DB071E
:1018D0001AD50A2E18D12100280000F097FF002801
:1018E00012D00FE00A4B9C4201D1AC68CDE7094B06
:1018F0009C42CAD1EC68C8E72100280000F018F823
:101900000028CAD0012676423000F8BD105F0100E1
:10191000305F0100F05E01000B1E04D0FF2A04D9E5
:101920008A2303608B3B180070470A700123FAE793
:10193000364B70B51D6806000C00002D05D0AB6954
:10194000002B02D1280000F0CFFF314B9C420FD179
:101950006C680C23E25E93B219072DD4D90611D41A
:1019600009230120336037331343A381404270BD04
:10197000284B9C4201D1AC68EBE7274B9C42E8D155
:10198000EC68E6E75B0713D5616B002908D02300FC
:101990004433994202D03000FEF768FF00236363AE
:1019A0002422A3899343A3810023636023692360D6
:1019B0000823A2891343A3812369002B0BD1A02103
:1019C0008022A389890092000B40934203D021001A
:1019D000300001F051F80123A289134011D00023F7
:1019E000A36063695B42A361002023698342BED187
:1019F0000C23E25E1306BAD540231343A3810138BA
:101A0000B5E7920700D46369A360EDE7A400002066
:101A1000105F0100305F0100F05E010010B506208C
:101A200001F020FD012001F051FEF0B503690C69C1
:101A300089B0070005910026A34265DB0B00013C3D
:101A40001433A50003935B1904930300143302932A
:101A50005D19049B28681B68591C0193FBF758FF0C
:101A60000190B04229D0039B02989C46069662469C
:101A700008CA9446019A99B251431B0C53438919E1
:101A80000A0C9B1807931E0C036889B29AB2069B36
:101A9000D2180368521A190C6B469B8BCB1A11147F
:101AA0005B18191492B21B041A43049B069104C0DC
:101AB0006345DCD22B68002B2DD00599380001F04E
:101AC00041FA00281FDB0025019B0298013303998E
:101AD0000193026808C992B255199AB2AA1A056808
:101AE0001B0C2D0CEB1A15145B191D1492B21B0460
:101AF000134308C0049B8B42EBD2029AA300D31875
:101B00001A68002A11D0019E300009B0F0BD2B6880
:101B1000002B04D1013C029B043DAB42F7D33C6156
:101B2000CBE71A68002A04D1013C029A043B9A428E
:101B3000F7D33C61E7E70000F0B516001F00446AE8
:101B40009BB00290239D06960797002C08D1102089
:101B5000FEF74CFE029B5862446084600460C460DF
:101B6000029B5B6A196800290BD05A6801239340D5
:101B70004A608B60029801F008F80022029B5B6AC1
:101B80001A60002F20DA01232B607B005B0807938B
:101B9000079CB24B220017931A409A4217D1B04BC0
:101BA000229A1360069B002B03D1240301D100F07D
:101BB00087FDAC4B249A0893002A02D0AA4B249AA2
:101BC000136008981BB0F0BD00232B60E0E7069E71
:101BD000079F0022002330003900FCF72DF8051E76
:101BE0000BD00123229A1360A04B249A0893002A59
:101BF000E7D09F4A24990A60E3E718AB019319AB39
:101C0000009332003B00029801F01AFA630003903F
